:020000040800F2
:1000000000200010A53A030879020308154B0008E8
:1000100075020308710203086D0203080000000066
:10002000000000000000000000000000690203085A
:100030006502030800000000610203084D5D00082E
:100040000D3B03080D3B03080D3B03080D3B030864
:100050000D3B03080D3B030841EE00086DEF00085F
:1000600031EF0008F5EE0008B9EE00085D28000841
:100070004D2800083D2800082D2800081D280008EC
:1000800009280008F52700080D3B03080D3B03086D
:10009000210703080D3B03080D3B03087DEE000814
:1000A0000D3B0308E554000885540008F55400088A
:1000B000D5540008C5540008B55400080D3B03088A
:1000C0000D3B03080D3B03080D3B03080D3B0308E4
:1000D0000D3B0308D15E0008555E0008D95D00089D
:1000E00005EE00080D3B0308510203080D3B030811
:1000F000955400080D3B0308A55400080D3B030868
:100100000000000000000000000000000D3B03089C
:100110000D3B03080D3B0308D93C0108BD3C010819
:10012000E1270008CD270008B9270008A527000807
:10013000912700080D3B03080000000000000000AC
:100140000D3B03080D3B03080D3B030800000000B6
:10015000000000000000000000000000000000009F
:1001600000000000000000000D3B03080D3B0308E9
:100170000D3B03080000000000000000000000002C
:08018000000000000D3B030824
:10018800F8B50568037B2A6802269E4032420DD1E5
:10019800296804229A40114218BF6A602968082217
:1001A80002FA03F3194218BF6B60F8BD1749184AE1
:1001B8000B684FF6FE7423400B6013899F07FCD52C
:1001C800134B1A891406FCD41B89D90718D4114972
:1001D8000F4A0B684FF6FE773B400B606E609388C2
:1001E80023F0030304461B040B481B0C9380006890
:1001F8000EF0D0FD094A2568237B00211170C7E75E
:10020800034B9A891A89D207E1D5FAE70804024014
:10021800003C00401C040240AC5D00204D3600202C
:100228004FF40063838270474FF400638382704702
:100238004FF4805383827047012380F8453070471C
:1002480070B40468037B2268022101FA03F31A429E
:1002580013D042690A495C2000FB02124FF6FE7671
:1002680050685289C5680068296831402960C168AA
:10027800D24392B20A40C260636070BC704700BF4C
:100288006C56002030B40A4B1D7875B1094B00201C
:1002980003EBC5051A6899885062D4682143D16078
:1002A800083323F8040CAB42F4D130BC704700BFCC
:1002B8004C5900205059002010B40268047B116882
:1002C8000223A340194209D00649406800240C7053
:1002D80001684FF6FE742140016053605DF8044BDD
:1002E800704700BF074D0020F0B5836983B005460D
:1002F80013B11A689B8813856869264F8389C324BC
:100308004FF47A734FF0060E6E464FF6FF710137C1
:1003180003E0013B9BB28B421DD002899207F8D5BE
:1003280004734FF47A7302E0A3B28B4213D00289AC
:10033800D20703F1FF34F7D5027BD2B20EB1327087
:100348000136BEF1000F08D00EF1FF3EFF24002F4A
:10035800E3D03C78DBE70EF091FEAB6913B11A6885
:100368009B8893619DF805009DF801609DF8021037
:100378009DF803409DF804209DF8063041EA0621C7
:1003880043EA002342EA0422012029876A87AB87CF
:1003980003B0F0BDE050030810B490E80600047BF9
:1003A80040690223A3404B6013685DF8044B4FF685
:1003B800FE710B40136005F0C5BD2DE9F0472B4FCA
:1003C8002B4D2C4C8246386889460EF0DDFC012006
:1003D80005F01AFC0026A8464AFA06F3DA07206850
:1003E8003DD50EF0D7FC28680EF0D4FC012005F0AE
:1003F8000BFC28680EF0C8FC0136012005F004FC4F
:10040800042EE9D120680EF0C5FC28680EF0C2FC65
:10041800012005F0F9FB28680EF0B6FC012005F074
:10042800F3FB002529FA05F3DB0720681AD50EF03F
:10043800B1FCD8F800000EF0ADFC012005F0E4FB9B
:10044800D8F800000EF0A0FC0135012005F0DCFB17
:10045800142DE7D13868BDE8F0470EF09BBC0EF0CC
:1004680093FCC0E70EF090FCE3E700BFAC2A002045
:10047800B02A0020A82A0020028822F04002120494
:10048800120C0280028822F038031B041B0C59B19D
:1004980041F48071002991FAA1F2B2FA82F108BF01
:1004A8004FF0FF310139C9000B439BB20380038829
:1004B8009BB243F040030380704700BF08B540F289
:1004C800E93300E09BB10289013B12F0020F9BB2B5
:1004D800F8D0017340F2E93300E043B10289013BEF
:1004E80012F0010F9BB2F8D0007BC0B208BD0EF02D
:1004F800C5FDC0B208BD00BFF8B53E4C20680EF07F
:1005080043FC3D4B1B78012B65D050D3022B46D1C1
:100518003A4D08232B704FF4C373394E394F33804B
:10052800022100200FF0ACFD20680EF02DFC2D7884
:1005380035480021FFF7C2FF29463348FFF7BEFFC1
:10054800324B31481D780221FFF7B8FF29462E4863
:10055800FFF7B4FF2E4B2C481D780321FFF7AEFFA1
:1005680029462948FFF7AAFF2A4B27481D78042166
:100578000D43FFF7A3FF29462348FFF79FFF206895
:100588000EF008FC32882448002134F036FD3B7810
:1005980063B1224B1B7823B300233B70F8BD174D82
:1005A8002B785B06B7D54FF4F073B6E7F8BDA021FA
:1005B8001548124DFFF782FF00211348FFF77EFF11
:1005C80000F00603022B03D000F0050001280DD02F
:1005D80008232B709FE7094D48232B704FF4F073C5
:1005E8009BE70FF0D7FC00233B70F8BD48232B7026
:1005F800D9E700BFAC5D0020B05D0020F20100200B
:10060800F001002000000020003C0040B75D002001
:10061800B85D0020A83C0020703800205938002020
:100628002DE9F04F85B090F855300190002B40F03F
:100638007185019B1B7C022B00F0C885BB4CBC4D0F
:10064800DFF8F492BB48DFF8F4E24FF0640A4FF0A9
:10065800100C4FF47A76D9F80430C3F30803002B52
:1006680040F05684EFF31183002B40F05184216849
:10067800826800BF23689942F9D12F6806FB07F307
:100688009B1AB3FBF7F306FB013101270091D9F858
:100698000430C3F30803002B40F00084EFF3118308
:1006A800002B40F0FB832368816800BF22689342D7
:1006B800F9D1D5F800B006FB0BF2521AB2FBFBF2E7
:1006C80006FB0323009A9B1AB3F57A7FDFD3BAF1AE
:1006D800010AC0D1019B1B7C022B00F05B86DFF86E
:1006E80058929448DFF854E24FF0640A4FF0100C27
:1006F8004FF47A76D9F80430C3F30803002B40F09E
:10070800EB83EFF31183002B40F0E68321688268C6
:1007180000BF23689942F9D12F6806FB07F39B1A9B
:10072800B3FBF7F306FB013101270091D9F8043038
:10073800C3F30803002B40F09483EFF31183002BDD
:1007480040F08F832368816800BF22689342F9D103
:10075800D5F800B006FB0BF2521AB2FBFBF206FB0F
:100768000323009A9B1AB3F57A7FDFD3BAF1010A03
:10077800C0D1019B1B7C022B00F0E885DFF8B89103
:100788006C48DFF8B8E14FF0640A4FF0100C4FF4F2
:100798007A76D9F80430C3F30803002B40F0648458
:1007A800EFF31183002B40F05F842168826800BF5B
:1007B80023689942F9D12F6806FB07F39B1AB3FB0C
:1007C800F7F306FB013101270091D9F80430C3F390
:1007D8000803002B40F02883EFF31183002B40F02F
:1007E80023832368816800BF22689342F9D1D5F832
:1007F80000B006FB0BF2521AB2FBFBF206FB032316
:10080800009A9B1AB3F57A7FDFD3BAF1010AC0D1F7
:10081800019B1B7C022B00F08185DFF81C91454869
:10082800DFF818E14FF00F0A4FF0100C4FF47A760A
:10083800D9F80430C3F30803002B40F0F883EFF332
:100848001183002B40F0F3832168826800BF23687E
:100858009942F9D12F6806FB07F39B1AB3FBF7F30C
:1008680006FB013101270091D9F80430C3F30803CE
:10087800002B40F0BC82EFF31183002B40F0B782CD
:100888002368816800BF22689342F9D1D5F800B087
:1008980006FB0BF2521AB2FBFBF206FB0323009A8B
:1008A8009B1AB3F57A7FDFD3BAF1010AC0D1019957
:1008B80091F84F200B7C042A34BF18261A26022BE5
:1008C80000F01585DFF870901A48DFF870E04FF0F7
:1008D8000F0A4FF0100C4FF47A76D9F80430C3F3AE
:1008E8000803002B40F0F983EFF31183002B40F04D
:1008F800F4832168826800BF23689942F9D12F6880
:1009080006FB07F39B1AB3FBF7F306FB013101273C
:100918000091D9F80430C3F30803002B40F04A8251
:10092800EFF31183002B40F0458209E0385C00208A
:100938003C5C002010E000E000ED00E0345C0020AA
:100948002368816800BF22689342F9D1D5F800B0C6
:1009580006FB0BF2521AB2FBFBF206FB0323009ACA
:100968009B1AB3F57A7FD4D3BAF1010AB5D1019BAA
:100978001B7C022B00F0A384DFF8DC92B448DFF87C
:10098800D4E24FF00F0A4FF0100C4FF47A76D9F8F2
:100998000430C3F30803002B40F08383EFF3118383
:1009A800002B40F07E832168826800BF236899424B
:1009B800F9D12F6806FB07F39B1AB3FBF7F306FB85
:1009C800013101270091D9F80430C3F30803002B43
:1009D80040F0D381EFF31183002B40F0CE812368E0
:1009E800816800BF22689342F9D1D5F800B006FBB0
:1009F8000BF2521AB2FBFBF206FB0323009A9B1A76
:100A0800B3F57A7FDFD3BAF1010AC0D1019B1B7C11
:100A1800022B00F03A84DFF840928D48DFF834E288
:100A28004FF00F0A4FF0100C4FF47A76D9F80430D3
:100A3800C3F30803002B40F0A482EFF31183002BCB
:100A480040F09F822168826800BF23689942F9D1EB
:100A58002F6806FB07F39B1AB3FBF7F306FB01317C
:100A680001270091D9F80430C3F30803002B40F0A4
:100A78006781EFF31183002B40F06281236881685E
:100A880000BF22689342F9D1D5F800B006FB0BF2FB
:100A9800521AB2FBFBF206FB0323009A9B1AB3F52A
:100AA8007A7FDFD3BAF1010AC0D1019B1B7C022BEC
:100AB80000F0D283DFF8A0916548DFF898E14FF0A5
:100AC800640A4FF0100C4FF47A76D9F80430C3F367
:100AD8000803002B40F03982EFF31183002B40F01C
:100AE80034822168826800BF23689942F9D12F684F
:100AF80006FB07F39B1AB3FBF7F306FB013101274B
:100B08000091D9F80430C3F30803002B40F0FB80B0
:100B1800EFF31183002B40F0F6802368816800BF53
:100B280022689342F9D1D5F800B006FB0BF2521AAD
:100B3800B2FBFBF206FB0323009A9B1AB3F57A7FFC
:100B4800DFD3BAF1010AC0D1019B1B7C022B00F054
:100B58006C83DFF804913E48DFF8F8E04FF00F0AA5
:100B68004FF0100C4FF47A76D9F80430C3F3080329
:100B7800002B40F04082EFF31183002B40F03B82C2
:100B88002168826800BF23689942F9D12F6806FB63
:100B980007F39B1AB3FBF7F306FB0131012700911A
:100BA800D9F80430C3F30803002B40F08F80EFF32B
:100BB8001183002B40F08A802368816800BF226877
:100BC8009342F9D1D5F800B006FB0BF2521AB2FBEA
:100BD800FBF206FB0323009A9B1AB3F57A7FDFD357
:100BE800BAF1010AC0D1019B1B7C022B00F00683DD
:100BF800DFF864801649174F4FF00F094FF0100EB9
:100C08004FF47A70D8F80430C3F30803002B40F08F
:100C1800D481EFF31183002B40F0CF8122688E68D6
:100C280000BF23689A42F9D1D5F800C000FB0CF345
:100C38009B1BB3FBFCF300FB023300930126D8F89F
:100C48000430C3F308032BBBEFF3118313BB05E098
:100C580010E000E0345C002000ED00E02368D1F8EB
:100C680008A000BF22689342F8D1D5F800B000FB75
:100C78000BFCACEB0A0CBCFBFBFC00FB03C3009AAF
:100C88009B1AB3F57A7FDAD3B9F10109BAD105B065
:100C9800BDE8F08FEFF3118A8EF312888A680B682B
:100CA800DB0344BF3E608A682368D7F800C05FFA58
:100CB8008AFA8AF31188D5F800A09C4400FB0AF34D
:100CC8009B1AB3FBFAF300FB0C33D8E7EFF3118858
:100CD8008CF3128881680368DB0344BFCEF8007088
:100CE80081682368DEF800205FFA88F888F31188A5
:100CF800D5F800801A4406FB08F35B1AB3FBF8F337
:100D080006FB023367E7EFF311888CF312888168DA
:100D18000368DB0344BFCEF8007081682368DEF8FF
:100D280000205FFA88F888F31188D5F800801A4403
:100D380006FB08F35B1AB3FBF8F306FB0233FBE68A
:100D4800EFF311888CF3128881680368DB0344BFD2
:100D5800CEF8007081682368DEF800205FFA88F812
:100D680088F31188D5F800801A4406FB08F35B1A4B
:100D7800B3FBF8F306FB02338FE6EFF311888CF32D
:100D8800128881680368DB0344BFCEF8007081686D
:100D98002368DEF800205FFA88F888F31188D5F810
:100DA80000801A4406FB08F35B1AB3FBF8F306FB52
:100DB800023323E6EFF311888CF312888168036805
:100DC800DB0344BFCEF8007081682368DEF800209A
:100DD8005FFA88F888F31188D5F800801A4406FB72
:100DE80008F35B1AB3FBF8F306FB0233B7E5EFF33E
:100DF80011888CF3128881680368DB0344BFCEF83E
:100E0800007081682368DEF800205FFA88F888F3AC
:100E18001188D5F800801A4406FB08F35B1AB3FB67
:100E2800F8F306FB02333AE5EFF311888CF31288E6
:100E380081680368DB0344BFCEF8007081682368CB
:100E4800DEF800205FFA88F888F31188D5F800806A
:100E58001A4406FB08F35B1AB3FBF8F306FB0233EC
:100E6800CEE4EFF311888CF3128881680368DB0302
:100E780044BFCEF8007081682368DEF800205FFA6E
:100E880088F888F31188D5F800801A4406FB08F31F
:100E98005B1AB3FBF8F306FB023362E4EFF3118845
:100EA8008CF3128881680368DB0344BFCEF80070B6
:100EB80081682368DEF800205FFA88F888F31188D3
:100EC800D5F800801A4406FB08F35B1AB3FBF8F365
:100ED80006FB0233FFF7F6BBEFF311828CF312889F
:100EE80087680368D90303D50123CEF800308768E3
:100EF8002368DEF80010D2B282F311882A681944F8
:100F080006FB02F3DB1BB3FBF2F306FB01310BE438
:100F1800EFF311828CF3128887680368D90303D52D
:100F28000123CEF8003087682368DEF80010D2B2BB
:100F380082F311882A68194406FB02F3DB1BB3FB12
:100F4800F2F306FB0131FFF7A0BBEFF311828CF33C
:100F5800128887680368D90303D50123CEF80030C7
:100F680087682368DEF80010D2B282F311882A68F5
:100F7800194406FB02F3DB1BB3FBF2F306FB01315A
:100F8800BDE5EFF311828CF3128887680368D903F3
:100F980003D50123CEF8003087682368DEF80010F7
:100FA800D2B282F311882A68194406FB02F3DB1BCC
:100FB800B3FBF2F306FB013152E5EFF311868EF332
:100FC8001288D1F808C00B68DA0303D501233B6007
:100FD800D1F808C023683A68F6B286F311882E68FB
:100FE8001A4400FB06F3A3EB0C03B3FBF6F300FB78
:100FF8000233009322E6EFF311828CF3128887689C
:101008000368D90303D50123CEF800308768236825
:10101800DEF80010D2B282F311882A68194406FB60
:1010280002F3DB1BB3FBF2F306FB0131B6E5EFF38A
:1010380011828CF3128887680368D90303D50123CA
:10104800CEF8003087682368DEF80010D2B282F349
:1010580011882A68194406FB02F3DB1BB3FBF2F381
:1010680006FB0131FFF7FEBBEFF311828CF3128808
:1010780087680368D90303D50123CEF80030876851
:101088002368DEF80010D2B282F311882A68194466
:1010980006FB02F3DB1BB3FBF2F306FB0131FFF7A0
:1010A80092BBEFF311828CF3128887680368D90327
:1010B80003D50123CEF8003087682368DEF80010D6
:1010C800D2B282F311882A68194406FB02F3DB1BAB
:1010D800B3FBF2F306FB013173E4EFF311828CF3F7
:1010E800128887680368D90303D50123CEF8003036
:1010F80087682368DEF80010D2B282F311882A6864
:10110800194406FB02F3DB1BB3FBF2F306FB0131C8
:10111800FFF7FDBB1D09013D052D03F00F0300F28C
:101128005181964A32F8150040FA03F2D40740F18B
:101138004981012404FA03F3013B184032F02AFBE9
:101148008F4B904A5B5D184412EBC00500F03A8162
:1011580052F83000AE88038A33407FF46AAA00F15F
:1011680038428949EB71920A8A5C02F01F035209DE
:101178002021022A04FA03F3A97100F03681032A18
:1011880000F02E81012A00F02681002302A9039392
:1011980002961BF0B7FA01997C4B41F80C3F2846A0
:1011A80028F08AF9AB88B3FA83F3C3F11F03581CFC
:1011B8003FF43FAA012202FA03F375490A68134370
:1011C8000B60019B1B7C022B7FF438AA019B9B6957
:1011D80013B11A689B881385019C6B216069FFF71E
:1011E8006DF980216069FFF769F9A369002B3FF465
:1011F80025AA1A689B889361FFF720BA019B9B690F
:1012080013B11A689B881385019E38217069FFF70E
:1012180055F901217069FFF751F9B369002B3FF4C3
:10122800E7AC1A689B889361E2E4019B9B6913B160
:101238001A689B881385019E37217069FFF73EF96C
:1012480010217069FFF73AF9B369002B3FF481ACBC
:101258001A689B8893617CE4019A936992F85060BC
:1012680013B11A689B881385019F19217869FFF7C4
:1012780025F931467869FFF721F9BB69002B3FF45E
:1012880019AC1A689B88936114E4019A936992F8DF
:101298004E6013B11A689B881385019F1A217869DB
:1012A800FFF70CF931467869FFF708F9BB69002B9D
:1012B8003FF4B1AB1A689B889361FFF7ACBB019B05
:1012C8009B6913B11A689B881385019E1C2170695C
:1012D800FFF7F4F818217069FFF7F0F8B369002BED
:1012E8003FF44AAB1A689B889361FFF745BB8B694B
:1012F80013B11A689B881385019F1B217869FFF732
:10130800DDF831467869FFF7D9F8BB69002B3FF45F
:10131800D9AA1A689B889361FFF7D4BA019B9B6985
:1013280013B11A689B881385019E6B217069FFF7BA
:10133800C5F801217069FFF7C1F8B369002B3FF4C4
:101348006CAA1A689B889361FFF767BA019B9B692F
:1013580013B11A689B881385019E6B217069FFF78A
:10136800ADF800217069FFF7A9F8B369002B3FF4C5
:1013780005AA1A689B889361FFF700BA5871030899
:1013880064710308905E0020807003084102000821
:1013980000040140019B9B6913B11A689B8813855F
:1013A800019E68217069FFF789F807217069FFF7C6
:1013B80085F8B369002B3FF492A91A689B8893615A
:1013C800FFF78DB901990B4B41F80C3F002028F02D
:1013D80073F80123F1E6084A51690B435361D4E6D7
:1013E800054AD1690B43D361CFE6034A91690B43A0
:1013F8009361CAE641020008001002402DE9F04F4F
:101408004269B24C1388DFF8D082B14E23F0400312
:101418001B041B0C138013889BB223F0380343F082
:101428003003138013889BB283B043F040031380CA
:10143800019004F043FBDFF8A4E2A6498446102794
:101448004FF47A750120DEF80430C3F30803002B4B
:1014580040F01D81EFF31183002B40F018812368C1
:10146800D1F8089000BF22689342F8D1D8F800A0BC
:1014780005FB0AF2A2EB0902B2FBFAF205FB032311
:101488009C45E0D0019D2846FFF7CAF8AB6913B127
:101498001A689B881385019B586940F2E93302E07A
:1014A800002B00F038810289013B12F0020F9BB239
:1014B800F6D06A23037340F2E93302E0002B00F010
:1014C8002A810289013B12F0010F9BB2F6D0037BFF
:1014D800019B586940F2E93302E0002B00F01E81BD
:1014E8000289013B12F0020F9BB2F6D0102303735E
:1014F80040F2E93302E0002B00F010810289013B41
:1015080012F0010F9BB2F6D0037B019B9B6913B1CC
:101518001A689B889361DFF8C4916E486C4F4FF04E
:10152800640A4FF0100E4FF47A75D9F80430C3F3FB
:101538000803002B40F0D480EFF31183002B40F018
:10154800CF802168826800BF23689942F9D1D8F812
:10155800006005FB06F39B1AB3FBF6F305FB0131AC
:1015680001260091D9F80430C3F30803002B56D1A3
:10157800EFF31183002B52D12368816800BF2268E2
:101588009342F9D1D8F800B005FB0BF2521AB2FB1E
:10159800FBF205FB0323009A9B1AB3F57A7FE1D38C
:1015A800BAF1010AC1D1019B4A4D5A69484F1388C3
:1015B80023F040031B041B0C1380138823F038030B
:1015C8001B041B0C138013889BB243F04003138049
:1015D80004F074FADFF804C181464FF0100E4FF49E
:1015E8007A760120DCF80430C3F30803002B31D1EC
:1015F800EFF3118373BB2368A96800BF2268934285
:10160800F9D1D8F800A006FB0AF2521AB2FBFAF296
:1016180006FB03239945E5D003B0BDE8F08FEFF34F
:10162800118C8EF3128881680368DA0344BF3E6028
:10163800816823683A685FFA8CFC8CF31188D8F8C3
:1016480000C01A4405FB0CF35B1AB3FBFCF305FB63
:101658000233A0E7EFF311818EF31288D5F808A0C2
:101668002B68DB0344BF3860D5F808A023683A68C4
:10167800C9B281F31188D8F800101A4406FB01F3A7
:10168800A3EB0A03B3FBF1F306FB0233C2E7EFF364
:10169800118987F31288D1F808A00B68DB0344BFCF
:1016A8003060D1F808A0236832685FFA89F989F3B5
:1016B8001188D8F800901A4405FB09F3A3EB0A0334
:1016C800B3FBF9F305FB0233DAE600BF385C002010
:1016D800345C002010E000E03C5C002000ED00E0FD
:1016E800EFF311828EF3128886680368D90302D556
:1016F80001233B60866823683968D2B282F3118877
:10170800D8F80020194405FB02F39B1BB3FBF2F346
:1017180005FB013124E70DF0B1FCD9E60DF0AEFC74
:10172800F3E600BFF8B584894FF6FF764FF47A7474
:101738002BB311B30F78013101E0B44217D00589FA
:10174800013CAD07A4B2F8D507734FF47A7402E0F0
:10175800BCB2B4420BD00589ED0704F1FF37F7D5C9
:10176800057BEDB20AB115700132013BE0E70DF0DF
:1017780085FC003018BF0120F8BDFF27DFE70120F6
:10178800F8BD00BF037C022B01D00020704770B564
:10179800836982B013B11A689B881385044640F2A6
:1017A800E933406901E0002B35D00289013B12F092
:1017B800020F9BB2F7D0C323037340F2E93300E072
:1017C8004BB30289013B12F0010F9BB2F8D0037BA7
:1017D800606906236A460021FFF7A4FFA36913B1D5
:1017E8001A689B8893619DF804009DF800609DF835
:1017F80001109DF802509DF803209DF8053041EA3C
:10180800062143EA002342EA052201202187628754
:10181800A38702B070BD0DF031FCD9E72DE9F04F78
:1018280090F8553085B00646002B7FD1904B1B7839
:10183800002B00F0D7807069038823F040031B0455
:101848001B0C038003889BB223F0380343F0380352
:10185800038003889BB243F040030380B36996F882
:101868004E4013B11A689B88138540F2E93302E0B1
:10187800002B00F027840289013B12F0020F9BB273
:10188800F6D01A23037340F2E93302E0002B00F08C
:1018980019840289013B12F0010F9BB2F6D0037B39
:1018A800706940F2E93302E0002B00F008840289F5
:1018B800013B12F0020F9BB2F6D0047340F2E933F9
:1018C80002E0002B00F0FB830289013B12F0010FBC
:1018D8009BB2F6D0037BB36913B11A689B889361F6
:1018E80004F0ECF8044604F0E9F88442FBD070698F
:1018F800038823F040031B041B0C0380038823F098
:1019080038031B041B0C038003889BB243F040037D
:101918000380337C022B00F03283B6F93A305BB295
:10192800013300F0FB8205B0BDE8F08F1D09013DD1
:10193800052D03F00F0300F2EC834E4A32F8150030
:1019480040FA03F2D20740F1E483012404FA03F3D6
:10195800013B184031F01EFF474B484A5B5D184475
:1019680012EBC00500F0D58352F83000AF88038A27
:101978003B407FF45BAF00F138424149EB71920A7A
:101988008A5C02F01F0352092021022A04FA03F399
:10199800A97100F0CC83032A00F0B683012A00F075
:1019A800C183002302A9029703931AF0ABFE3146C4
:1019B800344B41F80C3F284627F07EFDAB88B3FA3C
:1019C80083F3C3F11F035F1C3FF430AF012202FA17
:1019D80003F32D490A6813430B60254B1B78002B32
:1019E8007FF429AF7069038823F040031B041B0CA4
:1019F800038003889BB223F0380343F03803038045
:101A080003889BB243F040030380B36913B11A689B
:101A18009B88138540F2E93302E0002B00F05683DF
:101A28000289013B12F0020F9BB2F6D06B230373BD
:101A380040F2E93302E0002B00F048830289013BC1
:101A480012F0010F9BB2F6D0037B706940F2E933C4
:101A580002E0002B00F03D830289013B12F0020FE7
:101A68009BB2F6D08023037340F2E93311E000BF44
:101A7800901B00205871030864710308905E0020D1
:101A8800807003084102000800040140002B00F0A8
:101A980020830289013B12F0010F9BB2F6D0037B31
:101AA800B36913B11A689B8893619623AA4CAB4D0E
:101AB800DFF8B0A2AA48DFF8B0C201964FF01008CC
:101AC8004FF47A779946DAF80430C3F30803002B09
:101AD80040F0D882EFF31183002B40F0D3822368C3
:101AE800816800BF22689342F9D12A6807FB02FE89
:101AF800AEEB010EBEFBF2FE07FB03EE0126DAF8A1
:101B08000430C3F30803002B40F08182EFF3118304
:101B1800002B40F07C822368816800BF22689342D2
:101B2800F9D1D5F800B007FB0BF2521AB2FBFBF261
:101B380007FB0323A3EB0E03B3F57A7FDFD3B9F1D9
:101B48000109C0D1019EB36913B11A689B88138536
:101B580068217069FEF7B2FC03217069FEF7AEFCDC
:101B6800B36913B11A689B8893619623DFF8F4A1CF
:101B78007B48DFF8F4C101964FF010084FF47A77EC
:101B88009946DAF80430C3F30803002B40F05D826D
:101B9800EFF31183002B40F058822368816800BF5F
:101BA80022689342F9D12A6807FB02FEAEEB010EC8
:101BB800BEFBF2FE07FB03EE0126DAF80430C3F39E
:101BC8000803002B40F00582EFF31183002B40F04F
:101BD80000822368816800BF22689342F9D1D5F852
:101BE80000B007FB0BF2521AB2FBFBF207FB032310
:101BF800A3EB0E03B3F57A7FDFD3B9F10109C0D1A6
:101C0800019EB36913B11A689B8813856B217069AB
:101C1800FEF754FC03217069FEF750FCB36913B159
:101C28001A689B8893610F2003F094FFB36913B17E
:101C38001A689B881385706940F2E93302E0002B2B
:101C480000F04A820289013B12F0020F9BB2F6D0E3
:101C58006A23037340F2E93302E0002B00F03C8270
:101C68000289013B12F0010F9BB2F6D0037B706929
:101C780040F2E93302E0002B00F031820289013B97
:101C880012F0020F9BB2F6D01023037340F2E9332F
:101C980002E0002B00F023820289013B12F0010FC1
:101CA8009BB2F6D0037BB36913B11A689B88936122
:101CB8000F2003F04FFFB36913B11A689B8813858F
:101CC800706940F2E93302E0002B00F00B820289D0
:101CD800013B12F0020F9BB2F6D06C23037340F263
:101CE800E93302E0002B00F0FD810289013B12F08C
:101CF800010F9BB2F6D0037B706940F2E93302E032
:101D0800002B00F0F2810289013B12F0020F9BB216
:101D1800F6D00023037340F2E93302E0002B00F011
:101D2800E4810289013B12F0010F9BB2F6D0037BDC
:101D3800B36913B11A689B8893610F2003F00AFFF7
:101D4800B36996F8504013B11A689B881385706977
:101D580040F2E9330DE000BF385C00203C5C002015
:101D680010E000E000ED00E0345C0020002B00F003
:101D7800BF810289013B12F0020F9BB2F6D01923F2
:101D8800037340F2E93302E0002B00F0B1810289CD
:101D9800013B12F0010F9BB2F6D0037B706940F251
:101DA800E93302E0002B00F0A6810289013B12F022
:101DB800020F9BB2F6D0047340F2E93302E0002B25
:101DC80000F099810289013B12F0010F9BB2F6D015
:101DD800037BB36913B11A689B8893610F2003F0E2
:101DE800B9FEB36913B11A689B8813851B21706902
:101DF800FEF764FB18217069FEF760FBB36913B145
:101E08001A689B8893610F2003F0A4FEB36913B18D
:101E18001A689B881385706940F2E93302E0002B49
:101E280000F06C810289013B12F0020F9BB2F6D0E0
:101E38001C23037340F2E93302E0002B00F05E81BB
:101E48000289013B12F0010F9BB2F6D0037B706947
:101E580040F2E93302E0002B00F053810289013B94
:101E680012F0020F9BB2F6D01023037340F2E9334D
:101E780002E0002B00F045810289013B12F0010FBE
:101E88009BB2F6D0037BB36913B11A689B88936140
:101E98000F2003F05FFEB36913B11A689B8813859E
:101EA80037217069FEF70AFB10217069FEF706FBFF
:101EB800B36913B11A689B8893610F2003F04AFE37
:101EC800B36913B11A689B88138538217069FEF7C6
:101ED800F5FA01217069FEF7F1FAB36913B11A68CE
:101EE8009B8893610F2003F035FE7269138823F0F5
:101EF80040031B041B0C1380138823F038031B04B6
:101F08001B0C138013889BB243F0400313800120FD
:101F180003F020FE884A012313708CE496F93830C8
:101F280001337FF400AD0A26322027F0C1FC4FF4BC
:101F3800FA7503F0C3FD044603F0C0FD001BB0F5BD
:101F48007A7FF9D3013DF4D1072027F01BFB4FF42A
:101F58007A7503F0B3FD044603F0B0FD001BB0F53D
:101F68007A7FF9D3013DF4D1013EDDD17349744B39
:101F78007448754A0860DA6005B0BDE8F08FB36947
:101F880013B11A689B881385C321FEF797FA0623B5
:101F980002AA00217069FFF7C5FBB36913B11A687B
:101FA8009B8893619DF80A509DF80B309DF8084076
:101FB8009DF809109DF80C009DF80D2043EA0523B3
:101FC8001BB241EA042142EA002273873187B287B3
:101FD800A5E4EFF3118188F31288D0F808B00368FC
:101FE800DB0344BFCCF80060D0F808B02368DCF805
:101FF8000020C9B281F3118829681A4407FB01F34C
:10200800A3EB0B03B3FBF1F307FB0233F0E5EFF3AC
:10201800118188F31288D0F808B00368DB0344BF45
:10202800CCF80060D0F808B02368DCF80020C9B20A
:1020380081F3118829681A4407FB01F3A3EB0B030A
:10204800B3FBF1F307FB023374E5EFF3118288F376
:10205800128881680368DE0303D50123CCF80030B9
:1020680081682368DCF80060D2B282F311882A689C
:1020780006EB030E07FB02F35B1AB3FBF2F307FB55
:102088000E3E99E5EFF3118288F3128881680368A0
:10209800DE0303D50123CCF8003081682368DCF81F
:1020A8000060D2B282F311882A6806EB030E07FBA0
:1020B80002F35B1AB3FBF2F307FB0E3E1EE50CF0CE
:1020C800DDFF08E40CF0DAFFFFF7EABB0CF0D6FFFF
:1020D800BBE40CF0D3FFE3E40CF0D0FFC7E50CF051
:1020E800CDFFE0E50CF0CAFF06E60CF0C7FF1FE6DF
:1020F8000CF0C4FF52E60CF0C1FF6AE60CF0BEFF1C
:10210800A5E60CF0BBFFBEE6104AD1690B43D361CC
:1021180047E431460E4B41F80C3F002027F0CCF93C
:10212800012356E4094A51690B43536139E4074ACC
:1021380091690B43936134E4901B0020FC9F0020BD
:1021480000ED00E0EFBEADDE0400FA05001002402D
:1021580041020008037A022B01D00020704770B5B5
:10216800036982B013B11A689B881385044640F24C
:10217800E933C06801E0002B35D00289013B12F039
:10218800020F9BB2F7D0BB23037340F2E93300E0A0
:102198004BB30289013B12F0010F9BB2F8D0037BCD
:1021A800E06806236A460021FFF7BCFA236913B1E9
:1021B8001A689B8893619DF804009DF800609DF85B
:1021C80001109DF802509DF803209DF8053041EA62
:1021D800062143EA002342EA05220120E182228304
:1021E800638302B070BD0CF049FFD9E7F0B55B4BD3
:1021F8005B4A97B01968914200AF00F0A380594933
:10220800594A00234FF47000C1F888003B607B6096
:10221800136843F48033136003E03B68B3F5A04FC1
:1022280009D0136803F400337B603B6801333B60DB
:102238007B68002BF1D04C4B1B6813F4003318BF9C
:1022480001237B607B68012B52D0464C464B474AA2
:10225800E260474A596A11605A6A42F080725A62CB
:102268005A6942F4FC025A610025032207F1080169
:10227800012341F6FF764FF09040FD60BE603A734F
:10228800BB731AF03FFA4FF6FF7307F1080139489C
:10229800BB601AF037FA07F108013748374E1AF0D1
:1022A80031FA07F1080136481AF02CFA07F108014B
:1022B80034481AF027FA07F1080133481AF022FACD
:1022C80007F108001AF077FABB683049304AA1FBD9
:1022D800031330499B0CF0204FF0070E5C370B605E
:1022E800566084F823009560C2F800E0BD46F0BD52
:1022F800294A1D4B122111605A685A605A685A605F
:102308005A6842F480625A605A6822F47C125A6011
:102318005A6842F4E8125A601A6842F080721A60E9
:102328001A689201FCD559680F4A21F003015960D7
:10233800596841F002015960536803F00C03082BF7
:10234800FAD182E700221A6062B6144B1B6883F345
:102358000888134B1B689847FEE700BFFC9F0020C6
:10236800EFBEADDE00ED00E0001002400005FA050A
:10237800E859002000040048000800483F190100FF
:10238800000C0048001000480014004883DE1B437E
:1023980010E000E03C5C00200020024000D8FF1F55
:1023A80004D8FF1F064A00235168814202F11C022B
:1023B80004D001330C2BF7D100207047D8B27047F6
:1023C8009800002070B50F4C0F4DC0EBC00004EB17
:1023D8008004686926693043686182B09209667B27
:1023E800A1600025012101A863618DF804608DF8C2
:1023F80005208DF806508DF807101AF04DF902B037
:1024080070BD00BF9800002000100240074BC0EBD1
:10241800C00030B403EB8000054C056963692B43A9
:1024280063610176427630BC704700BF9800002097
:10243800001002402DE9F04F554C54F8204083B06D
:10244800002C60D0A56D1F469046524B6A682265E5
:10245800A160236004F15E014FF4807304F5AF724C
:102468006161A261E36023610646287E26F008FDCB
:10247800E86858B1FFF796FF721CD2B20C21FFF73B
:10248800C5FF236DEA6862632433E364A86890B1EA
:10249800FFF788FF721C8146D2B20B21FFF7B6FF07
:1024A8002346EA7E3C494846FFF78CFF236DAA681D
:1024B800A2632833A36494F85D000CF013F88146F6
:1024C80094F85C000CF00EF83A07824695F819B0BB
:1024D8001DD5B9F1000F1AD017F0110F4FF00B03EB
:1024E80006F1010614BF4E213E2189F8063089F80D
:1024F80007605A4648460CF0B9F8FB0743D5636BAA
:102508006BB3A36B5BB3204603B0BDE8F08F17F045
:10251800010F0CBF2E274E2718F0020F0DD0B9F16E
:10252800000F0AD00B22731C89F8062089F807309F
:1025380048465A4639460CF099F818F0010FDED093
:10254800BAF1000FDBD001360C238AF807605A462F
:1025580039468AF8063050460CF088F8CFE72B7FCA
:10256800AA7E8DF804209B090021012201A88DF87C
:1025780005308DF806108DF807201AF08DF82046E2
:1025880003B0BDE8F08F48460CF0FEFBB7E700BF8C
:10259800542A0020E8500308A103000800B9704736
:1025A800F0B595B0054626F0D1FE6E4EC3680268B8
:1025B80032600446002B00F0C38028460BF092FFDF
:1025C800694B586018B1292200238271C371227A9D
:1025D800664D2E210CF04AF8306803F0FFF826F01B
:1025E8004FFC3068624A038823F001031B041B0C6C
:1025F800038014A91E232B8001270F230025138095
:1026080021F84C7D2D230293ADF80C50ADF80650FF
:10261800ADF80E5026F048FEE379ADF8145060226C
:102628009907ADF816500695ADF81C50ADF81E5038
:10263800ADF82050ADF82250049200F1838013F0D9
:10264800010F14BF022200224FF48073ADF81470FA
:10265800ADF81C20ADF82030002304AA6179306859
:10266800069302F00FFD3068617926F0FDFD3068B1
:10267800436C43F40043436403889BB243F08003F4
:102688000380E3799B0768D56179026A04238B404C
:1026980022EA03020262026A134303623268354F78
:1026A80013889BB243F001031380207C0022292168
:1026B800FFF7ACFE3049207C00236022FFF782FE42
:1026C800E068386019F054FF386803684FF6FE7206
:1026D8001340036019F04CFF09A819F01DFF336877
:1026E8006279264938680A91343313440993802261
:1026F8001023002509A940F22A3E0E920B934FF4AD
:1027080000724FF400530D951095139511950F9283
:102718001293ADF830E019F00CFF627933680C2A97
:1027280098BF1749D86898BF31F812503A681549C8
:102738000543DD601368012043F00203136008704D
:1027480015B0F0BD13F0010F14BF08222A46042368
:10275800ADF81E20ADF816307EE7012261791EF033
:102768000FFB9BE744880020901B00203A8800203C
:102778003888002040880020C1020008604D0020F1
:10278800447003083C8800200348D0F83C3113B15A
:1027980000F59A7018477047980000200348D0F851
:1027A800203113B100F58C7018477047980000204D
:1027B8000348D0F804310BB1FC301847704700BF0C
:1027C800980000200348D0F8E8300BB1E0301847F3
:1027D800704700BF980000200348D0F8CC300BB1F8
:1027E800C4301847704700BF980000200348D0F84D
:1027F800B0300BB1A8301847704700BF98000020D0
:102808000348D0F894300BB18C301847704700BF9C
:10281800980000200248836F0BB17030184770474A
:10282800980000200248C36D0BB154301847704718
:10283800980000200248036C0BB1383018477047E5
:10284800980000200248436A0BB11C3018477047B3
:10285800980000200248836803B11847704700BFFA
:1028680098000020F8B505015A4C5B4B6259611974
:102878009A4204EB050704BF01230B730646387A16
:1028880026F0FEFA3B7A03F01F015B090122022BB6
:1028980002FA01F278D0032B71D0012B67D06319AB
:1028A800013618790BF01EFEF6B2074610B1122356
:1028B800C6718371631958790BF014FE10B1132394
:1028C800C6718371631998790BF00CFE10B114234B
:1028D800C671837166190E21F27938460BF0C6FE6F
:1028E80070790BF0FFFDF2790E210BF0BFFEB07985
:1028F8000BF0F8FDF2790E210BF0B8FE6359374A58
:10290800934251D0344A934259D0354A934240D0E9
:102918002C44227B002A2FD1012002249A8822F4F9
:1029280080521204120C9A80998889B241F480511D
:1029380099801A8802F4415242F4457202432243B4
:102948001A809A8822F470621204120C42F4E0622F
:102958009A809A8B22F400621204120C07219A833F
:1029680019821A8892B242F040021A80F8BD1D4BB3
:10297800996A0A439A6292E700200446CEE7194B07
:1029880019690A431A618AE7164BD9680A43DA605B
:1029980085E702F5EA32116941F4004111611169D4
:1029A80021F400411161B3E702F56042D16841F4B6
:1029B8008051D160D16821F48051D160A8E702F537
:1029C800EC32116941F480411161116921F48041AF
:1029D80011619DE7782A002000380040003001404E
:1029E800003C0040001002401749184B184A19488B
:1029F80010B4D1F8884044F47004C1F888401C68C9
:102A080044F001041C605C6822405A601A6822F095
:102A1800847222F480321A601A6822F480221A60C2
:102A28005A6822F4FE025A60DA6A22F00F02DA6269
:102A38001A6B002410404FF0006218639C608A6093
:102A48005DF8044B704700BF00ED00E00010024045
:102A58000CC07FF8CCFC00FF2DE9F04FB0F908500E
:102A68000D81EDB2442D91B00C46174600F09282CC
:102A780006462FD9812D00F0DD8100F28280542D89
:102A880000F0B08040F2C3816E2D00F05182802D9D
:102A980040F00481AF4B1D780B3D15F0FF0512D0B7
:102AA800AD4F00220A2621683B88481C20600E7022
:102AB8002168FF2B02F10102A8BFFF23481CAA428C
:102AC80020600B70EFDB01252B462846638111B08F
:102AD800BDE8F08F052D00F04B821ED8022D79D06D
:102AE80040F28281032D00F01A82042D40F0D68036
:102AF8002A469A4920460CF08BFE002120460CF00D
:102B0800B7FE22680221531C0125236028462B4664
:102B18001170638111B0BDE8F08F242D58D040F2B8
:102B2800FA80282D00F0C081382D40F0B7800A685F
:102B38008B4B0125511C2160157022680521501905
:102B48002060117022680A215019206011702268D3
:102B580000215019206011702268197850192060DE
:102B6800117022685978501920601170226899787C
:102B7800531923602B4611702846638111B0BDE8B4
:102B8800F08FA02D12D040F20581B82D00F0C5813C
:102B9800FE2D40F08380734D05F1080635F8021BC1
:102BA80020460CF065FEB542F8D18CE76E4B08461E
:102BB80019680CF045FE6D4B204619680CF040FE74
:102BC8006B4B1968204601250CF03AFE2B467CE732
:102BD800684BF6E704226849204601250CF018FEE8
:102BE8002B46C9E70B68654A654F581C11212060C0
:102BF800197023681278591C21601A70236897F895
:102C08005520591C21601A70236897F85420591CC4
:102C180021601A70B7F8501020460CF029FE23687E
:102C28000022591C21601A7023682822591C21602F
:102C38001A70B7F8521020460CF01AFEBD1E07F1A4
:102C48004E0635F8021F20460CF012FEB542F8D1A8
:102C580022684C4B0D21501C20605D1811702268B1
:102C680013F8011F501C9D4220601170F7D1236892
:102C78000222591C21601A70B7F8561020460CF031
:102C8800F7FDB7F8581020460CF0F2FD0125B7F80B
:102C98005A1020460CF0ECFD2B466DE721462846DD
:102CA8000DF06EFB00287FF40EAF742D00F0B58098
:102CB800772D0CD1336872689A421BBF5A1C326058
:102CC80001461978304A20462DF024FAFBE6F52D06
:102CD80000F06881392D376801F0388200F2EE8102
:102CE800212D01F04382292D40F090827B1C336016
:102CF8003B780A2B01F08282502B40F05A873046ED
:102D08000CF074FD214F388030460CF06FFD012522
:102D180078802B4630E7202DC0D10B681C4D591CFC
:102D28006A7821601A7023682A78591C21601A7001
:102D38002368AA78591C21601A70298920460CF04A
:102D480097FD23686A79591C21601A702268A9794D
:102D5800D9E600BF2A3E0020702200204E600020E5
:102D6800B1860020803E0020ACF7FF1FB0F7FF1FA0
:102D7800B4F7FF1F10880020287A0308B45D0020EC
:102D88007C630020D96300207DF6020860220020C1
:102D980060400020822D81D10B68B14AB14D117875
:102DA800B14A581C20601970118920460CF060FD4A
:102DB800AE4B22681B88FF2B02F10101A8BFFF233D
:102DC80021601370A96881F3100189B220460CF0C4
:102DD8004FFD296801F30F0189B220460CF048FD28
:102DE800A34B226819788EE6012D7FF457AF0B6844
:102DF8000022591C21601A7023685A1C22601D7019
:102E080022682521531C23602B461170B4E6522DED
:102E18007FF444AF2268002175E6336872689A42ED
:102E28001BBF5A1C326001461978924A20462DF081
:102E380071F948E6904B1E780A3E16F0FF063FF4FB
:102E480042AE8E4B8E4F1E4403F101080A2314E054
:102E5800502B00F00181002529462268501C206073
:102E6800204613700CF004FD294620460CF000FDA6
:102E7800B0453FF428AE18F8013B0A2BE8D1814A47
:102E88009568116805EB85054FF6FF726D00954250
:102E9800A8BF15469142A8BF114625EAE57521EA63
:102EA800E171ADB289B2D8E70B68DFF80882764ED7
:102EB800591C022221601A70236806275A1C2260B6
:102EC8001F7023680A22591C21601A702368012583
:102ED8005A1922601D70B8F8001020460CF0C8FC82
:102EE800B8F8021020460CF0C3FC23685A19226077
:102EF8001F7023685022591921601A702368002214
:102F0800591921601A70318820460CF0B1FC71887B
:102F180020460CF0ADFC2B462EE65C4B51E60B68C8
:102F28005A1C0A601D700B685A1C0A601D7071E7F4
:102F38004E4B0A681B884B4DFF2BA8BFFF23511C23
:102F480021601370A96881F3100189B220460CF042
:102F58008FFC4F4B204619880CF08AFC296801F336
:102F68000F0189B2204601250CF082FC2B4603E6AE
:102F78000B22484920460CF04BFC082246492046C3
:102F88000CF046FC01250722444920460CF040FC81
:102F98002B46F1E5002A3FF496AD414B136001251D
:102FA8002B46E9E5336872689A4241F0FF803D4B51
:102FB800FF221A704FF000093B4D20F057FC49469C
:102FC80020223A4885F8009032F017F88DF80090E2
:102FD8009DF80030072B01F27381DFF8DC80334E57
:102FE8004A469DF8003003EB430308EBC3035B7CC0
:102FF800E3B19DF8003003EB430308EBC303202142
:103008005B699BB19DF8003003EB430308EBC303F6
:10301800586946F822000BF0FBFC2B7856F8230081
:103028000BF0B8FE2A780132D2B22A709DF800302F
:103038000133DBB28DF800309DF80030072BD0D972
:103048002368591C21601A70002F3FF43CAD184BBF
:103058003B6001252B468FE5BD68396812E700BF44
:10306800A23E002070400020604000208C3E0020DE
:1030780040640020DDF602082A3E002010510308B3
:10308800642200202C220020602200200C2E002028
:1030980008640020307A03083C7A0308487A030859
:1030A8000D010108D01B00208F5B0020505B002021
:1030B800F58702081431002084550020552D73D05F
:1030C800572D40F0A3807B1C336017F8375B0DF158
:1030D800FF320133336013F8011C02F8011FBB42B1
:1030E800F7D1444A1378002BFCD1DFF818A19AF8DD
:1030F8000070002FFDD1DFF810B13F4EDBF8000063
:103108004FF001088AF800800BF03EFE3B4B394631
:10311800304683F80080FDF7D1F939463046FDF78F
:10312800CDF909213046FDF7C9F929463046FDF7A2
:10313800C5F9E8466D460DF13609A5EB0807FFB25B
:103148000A213046FDF7BAF939463046FDF7B6F997
:1031580015F8017B0B213046FDF7B0F939463046AA
:10316800FDF7ACF900200AF029FE4D45E5D12248CB
:1031780008210546FDF7A2F9A0212846FDF79EF98A
:10318800A0212846FDF79AF900212846FDF796F96F
:1031980010F02006F4D1DBF8000001250BF0FAFD51
:1031A8008AF800602B46E7E47B1C336097F80080C0
:1031B800B8F1FF0F01F05780B8F1FE0F01F035802C
:1031C80030460CF013FB96E80C009B1A002B07DD29
:1031D800531C336013781BB9B8F10C0F41F23880D7
:1031E800B8F1270F00F29582054B012523F8180046
:1031F8002B46C1E44D360020003C004061380020D9
:103208007C63002059380020AC5D002072680B3DBB
:10321800D31BEF2D00F27D8201A151F825F000BFEC
:103228001F4100081B3700081B3700081B37000820
:103238001B3700081B3700081B3700081B3700081E
:103248001B3700081B3700081B3700081B3700080E
:103258001B3700081B3700081B3700081B370008FE
:103268001B3700081B3700081B3700081B370008EE
:103278001B3700081B3700081B3700081B370008DE
:103288008D4000081B370008054100081B3700085F
:10329800E34000081B3700081B3700081B370008ED
:1032A800493B00081B370008EF3A00081B370008A5
:1032B800813D00081B3700085B3D00081B370008EC
:1032C800493D00081B370008F53C00081B3700087B
:1032D800113C00081B3700081B3700081B37000883
:1032E8001B370008CF2A00081B370008E53B0008F9
:1032F8001B3700081B370008CB3B00081B370008AA
:10330800713B00081B3700081B3700081B370008F3
:103318001B3700081B3700081B3700081B3700083D
:103328001B370008A53E00081B370008573E000859
:103338001B3700081B370008173E00081B3700081A
:103348001B3700081B3700081B3700081B3700080D
:103358001B3700081B370008B33D00081B3700085F
:103368004F3F00081B370008E53E00081B370008E0
:10337800FD3F00081B370008C73A00087F3A0008DD
:10338800633A00081B3700081B3700081B37000882
:103398001B3700081B3700081B3700081B370008BD
:1033A8001B3700081B3700081B3700081B370008AD
:1033B8001B3700081B3700081B3700081B3700089D
:1033C8001B3700081B3700081B3700081B3700088D
:1033D8001B3700081B3700081B3700081B3700087D
:1033E8001B3700081B3700081B3700081B3700086D
:1033F8001B3700081B3700081B3700081B3700085D
:103408001B3700081B3700081B3700081B3700084C
:103418001B3700081B3700081B3700081B3700083C
:103428001B3700081B3700081B3700081B3700082C
:103438001B3700081B3700081B3700081B3700081C
:103448001B3700081B3700081B3700081B3700080C
:103458001B3700081B3700081B3700081B370008FC
:103468001B3700081B3700081B3700081B370008EC
:103478001B3700081B3700081B3700081B370008DC
:103488001B3700081B3700081B3700081B370008CC
:103498001B3700081B3700081B3700081B370008BC
:1034A8001B3700081B3700081B3700081B370008AC
:1034B8001B3700081B3700081B3700081B3700089C
:1034C8001B3700081B3700081B3700081B3700088C
:1034D8009D3A00081B3700084D3A0008233A0008B7
:1034E8001B3700081B3700081B3700081B3700086C
:1034F8001B3700081B3700081B3700081B3700085C
:103508001B3700081B3700081B3700081B3700084B
:103518001B370008C93900081B3700089139000813
:103528001B370008F5380008973800087B38000872
:103538001B370008613800081B37000839380008B5
:103548001B370008DF3700081B370008B1370008B1
:103558001B3700081B3700088F3700086137000841
:103568004D37000825370008FD360008DB3600080F
:103578001B3700081B3700081B3700081B370008DB
:103588001B3700081B3700081B3700081B370008CB
:103598001B3700081B3700081B3700081B370008BB
:1035A8001B3700081B3700081B3700081B370008AB
:1035B800C13600081B3700081B37000869360008A9
:1035C8001B3700081B3700081B37000803360008A4
:1035D8001B3700081B3700081B370008E9350008AF
:1035E800B14B1B78DB0700F19480012501F0C4FA88
:1035F80001F06AFB2B46FFF7BFBA30460CF0F6F82D
:103608003368ADF800001A46591C316012F8021BE5
:1036180032608DF802105A788DF80320DA1C326077
:103628009A788DF804201A1D3260DA788DF8052012
:103638005A1D32601B798DF8063068460023ADF8B4
:1036480008300CF02BF8994A994B1268801A4FF001
:10365800010561F10001C3E904012B46FFF78CBAAB
:103668007B1C33603B780F2B53D8BA1C3260C3EBFA
:10367800C303904A7978D154F91C31601344BA785D
:103688005A703A1D3260FA789A707A1D32603A7927
:10369800DA70BA1D32607A791A71FA1D3260BA7915
:1036A8005A7107F108023260FA799A71012528F0F7
:1036B80067FD2B46FFF760BA30460CF097F87E4F4F
:1036C800F88130460CF092F80125B8812B46FFF7B7
:1036D80053BA30460CF08AF8784F388230460CF0EE
:1036E80085F8788230460CF081F80125B8822B469F
:1036F800FFF742BA3B467A1C326013F8020B33607C
:10370800FB1C79783360BA7822F042F800287FF4FD
:10371800DAA94FF0FF352B46FFF72EBA3B467A1C45
:103728003260674A13F8021B11703360624A7B7873
:103738009370FB1C3360634BBA789A7001252B4653
:10374800FFF71ABA604B614918684E22012530F01C
:10375800C3FA2B46FFF710BA3A467B1C33605C4B22
:1037680012F8021B197032607A785A70FA1C3260AB
:10377800BA789A7030460CF039F8564B0125D88043
:103788002B46FFF7F9B930460CF030F8514F388026
:1037980030460CF02BF8788030460CF027F80125DD
:1037A800B8802B46FFF7E8B9DFF8388198F8003081
:1037B800002B3FF488A9484F002530460CF016F836
:1037C8001EF0A4F898F80030A7EC010A01359D42D4
:1037D800F3DBFFF778B90D2B9BD17B1C33603D7869
:1037E800072D96D8DFF8008130460C270BF0FEFF36
:1037F80007FB05F708EB0705A88030460BF0F6FF36
:10380800E88030460BF0F2FF336828811A46591CCD
:10381800316012F8021BA97232605B78EB72304695
:103828000BF0CCFF012548F807002B46FFF7A4B999
:103838007B1C33603878060600F1D9851A4B1B7853
:10384800DD073FF540A9032828BF0020012501F026
:1038580077F92B46FFF790B9134B1B78D8073FF53C
:1038680032A9012501F002FC01F02EFA2B46FFF7E0
:1038780083B90D4B1B78DA073FF525A9174A13784A
:10388800012543F0040313702B46FFF775B9064B67
:103898001B78D9073FF517A9114B4FF4C8720125BA
:1038A8001A802B46FFF768B90D3E0020385C0020CF
:1038B800D01B0020202D0020243100204456002059
:1038C8002054002034310020D4400020E06E03084A
:1038D8001C31002038460020342B0020E8630020EB
:1038E800724600202A3E0020602C0020092B7FF71A
:1038F80010AFDFF8F0833B467A1CD8F800503260EE
:1039080013F8022B2A7033607B78AB70FB1C336092
:10391800BB78642BA8BF64233A1D6B713260FB78B7
:10392800642BA8BF64237A1DAB7132603B79EB71BD
:10393800BB1D33607B79642BA8BF6423FA1D2B72EF
:103948003260BB79EB7007F108033360FB792B71A8
:1039580030460BF04BFF726833686881D11A002932
:103968000CDD591CD8F800003160521A002A197869
:10397800417203DD9A1C32605B78437001251EF0AA
:1039880025FE2B46FFF7F8B8C44B1868FB1C024607
:103998002137991E316013F8031C1170591E3160CC
:1039A80013F8021C5170336013F8011C9170033333
:1039B8009F4202F10302ECD128F0C6FFFFF783B85B
:1039C800C3F34705122D3FF6A4AEB5B110ABADF168
:1039D800020903EB4507C846423F30460BF006FF95
:1039E80028F8020FB845F8D1AD4B39F8022F23F863
:1039F800022FC845F9D1112D09D8AA4A6B00023BFC
:103A080013440021223223F8021F9A42FBD1A64A0E
:103A180001231D461370FFF7AFB87B1CA349336021
:103A28000A783B78002A40F04E8404220A70A04AA3
:103A38009B00138002F042F89E4B012598612B46AB
:103A4800FFF79AB89C4F002330463B600BF0B6FE58
:103A5800012538602B46FFF78FB87B1C33603B7815
:103A6800002B00F0CF844FF4004001250DF0AAFC94
:103A78002B46FFF781B8914B1B7813F001017FF4B7
:103A880048AE7B1C33603878012510F069F82B4666
:103A9800FFF772B83B467A1C326013F8025B33605A
:103AA800FB1C78783360B978002D00F0CD84012DA7
:103AB8007FF409A810F01AF92B46FFF75DB83B46CA
:103AC8007A1C32607E4A13F8021BD17033607D4A3B
:103AD8007B785371FB1C33607B4BBA78DA70012515
:103AE8002B46FFF749B87B1C784D33603B782B7227
:103AF80030460BF07BFEA88330460BF077FE288318
:103B080030460BF073FE32686883531C33601278BA
:103B1800EA747268D31A032B00F331843368D11A1C
:103B2800052900F31B84D21A002A7EF7CCAF5A1C51
:103B380032601B7885F8213001252B46FFF71CB829
:103B48007B1C3360624938780870D21A002A7EF7E5
:103B5800BAAFBB1C33607B78003318BF0123012543
:103B68004B702B46FFF708B87B1C3360584B3A78EC
:103B7800DFF874811A700023C8F8003030460BF063
:103B88001DFE3268D8F800305049524D0343501C8E
:103B9800C8F80030306013780B7230460BF026FE00
:103BA800286030460BF022FE686030460BF01EFE9F
:103BB800A86030460BF01AFE30460BF017FEFEF7F1
:103BC80082BF454B07F108020137376017F8011C1F
:103BD80003F8011FBA42F7D1FEF775BF3B46791CBF
:103BE80031603E4913F8020B88703360787848706A
:103BF80093423EF468AFFB1C33602E4BBA781A72BE
:103C080001252B46FEF7B8BF0722B3FBF2F2C2EB41
:103C1800C2055B1B7FF47DADD2B202F1FF385FFABB
:103C280088F8002A3EF44FAFDFF8B4A008F1010885
:103C38001D467B1C336097F90010294B002703E0D1
:103C48000137062F3FF465AD93F902208A4203F14C
:103C58000803F5D10AEBC709304689F802100BF0C2
:103C6800C5FD33682AF837001A46591C316012F826
:103C7800021B89F8031032605A7889F80420DA1C8C
:103C880032609A7889F806201F1D37600135DB7885
:103C980089F80530A845CCD1FEF715BFD4400020DF
:103CA800565A0020585A0020545A0020E231002069
:103CB80008640020D01B00200C2E00200D3E0020A0
:103CC800243100202C660020343100203C5D002087
:103CD8008C320020B42A00203B5D002044310020B3
:103CE800685D0020D8400020108800207B1C3360CD
:103CF8003B780E2B3FF60DADBA1C3260787803285E
:103D08003FF607ADAD49062202FB03F28B18FD1CF6
:103D180058713560B87888543A1D3260FA785A700C
:103D28007A1D32603A799A70BA1D32607A79DA70FF
:103D3800FA1D3260BA791A7101252B46FEF71CBFAD
:103D48007B1C33609E4B3A785A7501252B46FEF74B
:103D580013BF7A1C32603D781F2D3FF6DAAC052B75
:103D68007FF4D7AC30460BF029FD964B43F825007D
:103D780017F0BAFDFEF7A7BE924D05F14007304691
:103D88000BF034FD3368A5F88000591C1A463160E1
:103D980012F8021B85F8821032605B7885F8833050
:103DA8000435AF42EBD1FEF78EBE874B1B68002B64
:103DB8003EF489AE18F00EF8FF283EF484AE304683
:103DC8000BF014FD3F2840F22683804F00253D70FC
:103DD80033687268B880D21A012A7EF774AE1A4620
:103DE800591C316012F8021BB97010A83260002209
:103DF8005D7800F8402D17F0BFFF9DF80030AB420A
:103E08003EF461AE284617F0DBFFFEF75CBE704B50
:103E18001B78012B3EF657AE39467B1C3360DFF822
:103E2800CC8111F8023B88F802303160FB1C7878AD
:103E38003360D31A012BB97840F3FA8230460BF07D
:103E4800D5FC0125A8F800002B46FEF795BE7B1C83
:103E5800336097F80080B8F1110F3FF65AACBB1CDD
:103E680033605C4D7B7805F8183030460BF0BEFCAB
:103E780040F6CA039842A8BF184640F2EE2398427B
:103E880005EB4801B8BF18460125A0F2EE222B46E3
:103E9800192092FBF0F24A70FEF76EBE3B467A1C80
:103EA8004D4D326013F8022B2A7133607B786B71A9
:103EB80030460BF09BFC336828805A1C32601B7814
:103EC800AB7130460BF092FC336868805A1C326044
:103ED8001B78EB7101252B46FEF74EBE7B1C336029
:103EE8003E4DDFF80C813B7888F8053030462F6866
:103EF8000BF07CFC388430462F680BF077FC726836
:103F08003368F883D11A072900F3E281D11A03290B
:103F180000F35582D21A002A05DD591C2A6831603F
:103F28001B7882F8263000F031FE22F08FF82C4BF7
:103F38001B68002B00F0E3812868012528F0B4F9FC
:103F48002B46FEF719BE3B467A1C3260DFF8A0808C
:103F580013F8022B88F802203360224A7B7813700A
:103F6800FB1C3360204DBB782B713B1D3360FB7805
:103F7800092BA8BF09233046AB700BF037FC336818
:103F880072682880D11A012905DD30460BF02EFC15
:103F980033687268E8819A4240F05C8200F0F6FD6E
:103FA800336872689A423EF48EAD5A1C32601B78B0
:103FB800EB7001252B46FEF7DFBD00BF182E002051
:103FC8003C5D0020844B0020103E0020143E002061
:103FD80008880020C844002050460020D440002013
:103FE800743200201831002044560020EA63002073
:103FF8002054002030460BF0F9FB30460BF0F6FB5E
:1040080030460BF0F3FB30460BF0FCFB3368C14D38
:104018001946581C2A68306011F8020B82F82C00E7
:104028003160597882F83610D91C31609B7882F853
:10403800373030460BF0E6FB30460BF0E3FB3046FA
:104048000BF0E0FB30462F680BF0D0FB788730464A
:104058002F680BF0CBFB336872683887D11A0129B7
:104068000ADD591C2A6831601B7882F82E303046E8
:104078000BF0C8FB33687268D31A032B00F3AC81CA
:10408800286899E47B1C33603D78132D3FF641ABDB
:10409800BB1C336078782CF077F800283FF439ABF4
:1040A8009D4B027803F82520FA1C326003EB850348
:1040B800BA785A703A1D3260FA789A707A1D32606E
:1040C8003A79DA7000201EF0C1F9944B80F00100B3
:1040D800012518702B46FEF74FBD30460BF086FBC6
:1040E8008F4F386030460BF081FB786030460BF01C
:1040F8007DFB0125B8602B46FEF73EBD894F0023A6
:104108003B6030460BF05AFB3B68012503433B609C
:104118002B46FEF731BD844A102B4FF0000128BF13
:104128001023116051609160D1601174002B3EF42E
:10413800CAAC3168013A0B440131316011F8010C05
:1041480002F8010F8B42F7D1FEF7BDBC7B1C336030
:104158003B780A2B58D030460BF054FB30460BF016
:1041680051FB30460BF04EFBFEF7ADBC3B467A1CCC
:1041780032606E4D13F8022B6A7033607B782B70B7
:10418800FB1C3360BB78AB7030460BF02FFB3368F9
:104198002881591C1A46316012F8021B6971326075
:1041A8005B78AB7101252B46FEF7E6BC5A1C194615
:1041B80032605F4811F8022B027031605B784370FF
:1041C800042A04D9FF2A7EF425AEFEF7F3BE594926
:1041D8000978994205D8022A7EF41CAEFF2B7EF49A
:1041E80019AE236801255A1922601D70002F3EF46C
:1041F8006AAC514B3B602B46FEF7BEBC30460BF019
:10420800F5FA4E4FFEF77FBDBB1C33604C4B7A78F6
:104218001A70FA1C3260BA785A703A1D3260FA780D
:104228009A7001252B46FEF7A7BCBB1C33607D782E
:10423800022D3FF66EAA30460BF0D8FA414B03EB3D
:1042480045034FF0FF35A3F856002B46FEF794BC04
:104258003C4B0030984418BF0120012588F85E00C7
:104268002B46FEF789BCBB1C3360374B7A781A7033
:10427800FB1C3360DFF8CC80BB7888F855303B1DD9
:104288003360FB7888F8543030460BF0AFFAA8F862
:10429800500030460BF0AAFA30460BF0A7FA96E821
:1042A8000C009B1A012BA8F852007EF70CAC304684
:1042B8000BF09CFA0125A8F85A002B46FEF75CBCC7
:1042C8004A46FEF7BDBE042A7EF4FDABFFF7AFBB3E
:1042D80030460BF08BFAA8F80A0030460BF086FA45
:1042E800A8F80C0030462F680BF080FA7884304626
:1042F8002F680BF07BFA33687268B88406E61348B7
:104308001349144A144B036001250B6013602B46B4
:10431800FEF732BCD4400020B8430020CC02002075
:10432800B42A0020108800208A5000206040002015
:10433800D01B00202A3E002025010108143100204E
:10434800B18600207C630020B45D00201462002048
:1043580068620020D062002021DC00085A1C32600C
:104368001B78EB7230460BF029FA3368E8605A1C68
:1043780032601B782B7433687268FFF7D4BB304601
:104388000BF034FAA88430460BF030FA33687268C0
:10439800E884D11A03297FF7C2AB1A46591C316049
:1043A80012F8021BA97732605B7885F82030304616
:1043B8000BF01CFA336872686884FFF7B0BB3046AC
:1043C8000BF014FAA8F80E0030460BF00FFA336819
:1043D8007268A8F810009DE530462F680BF006FAC1
:1043E800788630462E680BF001FAB08648E600F071
:1043F8007F00032828BF002001250FF093FC2B46DF
:10440800FEF7BABB184A1368012523F4004313606A
:104418002B46FEF7B1BBC50800F007030135013391
:10442800EDB2124F284619467B7018F04BFCCEE4CB
:104438000F4B1A88012512FB00F22B4692FBF1F272
:10444800A8F80020FEF798BB012528F009F92B46AB
:10445800FEF792BB5A1C32601B78003318BF012349
:1044680088F807309AE500BFCC400020143E0020B1
:10447800822F002038B50B4C23688BB15A68821AFA
:10448800002A054604DA0CE05A68AA1A002A07DB53
:104498009A68226018461A6890472368002BF3D15F
:1044A80038BD38BD544300200B4B002210B40272B3
:1044B80003F17804012102E0072A09DC99798907C8
:1044C80002D51979815401329C4203F11403F3D1C6
:1044D8005DF8044B704700BF887003082B230370F6
:1044E800704700BF012310B4132110241222447016
:1044F8004171C27003720370037183705DF8044BDD
:10450800704700BF436A8269D154436A0169826B6C
:1045180001338B4228BF00234362002A2FD0EFF3D8
:104528001181502383F31288836B1A68D2072CD425
:1045380070B45E686EB9456A826A954217D084691C
:104548001444DC600ED9AA1A5A608562002280F8E9
:1045580054201A6842F00102C9B21A6081F3118826
:1045680070BC70470469A21A5A608662EEE701239C
:1045780080F85430C9B281F3118870BC7047026D5D
:10458800136843F0800313607047C9B281F3118840
:10459800704700BF426B10B462B1436CC268446993
:1045A800D11A013B615C5DF8044B08BF13464364B4
:1045B800C8B27047016A4369C4685B5C0131A142B3
:1045C80028BF114601625DF8044BD8B2704700BF9E
:1045D800836B13B190F854007047836A406A181AC5
:1045E800B0FA80F040097047416A836A99420AD359
:1045F800CB1A816B026961B14968501E0B44834232
:104608000AD2C01A704702691144CB1A816B00297B
:10461800F2D1501EC01A704700207047436B43B157
:10462800426C5B6893422FBF981AC0689B1AC018E7
:104638007047C269036A9A422FBFD01AC0688018AF
:10464800C01A70470A4B30B503F1140493F90020DF
:104658005D78072AC8BF143A811804330D7313F81C
:10466800025C855413F8012C0A76A342EED130BDC2
:10467800145103082DE9F0478C4B1B78DB070746DC
:1046880044D58B4B8B4D1C788B4E012C59D01CD3A9
:10469800022C07D189498A4A09881288914201D98E
:1046A80001241C70EB7AE3B12B89D3B1854B1B78BD
:1046B800BBB10FF059FB002800F09B802B7B834295
:1046C8002CBF0121002131700CE07C497E4A098809
:1046D80010886A7B801A8842E2DAEB7A0024002B81
:1046E800E2D131782A79632A06D8022C774E00F075
:1046F800BA803378002B5DD1754AAB7A8C4238BFCB
:104708000C461470002B4CD1BDE8F0876B4B694DFB
:1047180019885B88E878CB1A83EAE3728142A2EBB6
:10472800E3721DD32B788B421AD3614B1C78E01EA1
:10473800012861D96749097802294FD0012C5E4EBA
:10474800A5D15F4A5D491288687B0988121A91428F
:1047580039DD5D4A12888A42A4D200241C70A1E780
:10476800B1EB400FE1DC524B1C78E11E012940F20D
:104778009480022ADEDC57494F4E0878DFF84481DE
:10478800DFF844C1DFF838E100210324022834703F
:104798001C7088F80010ACF80010AEF8001081D139
:1047A8001FE0012C71D0022C0BD10720BDE8F04787
:1047B8002BF01CBB7068381A474B984258DD727052
:1047C8009AE7BDE8F08702241C706BE7022AD2DD65
:1047D8004049097802294FF0040464D13949364E1A
:1047E80009783E48022ACCBF00220122C28081807B
:1047F8004BE70221317075E7022A9BDC95F800C06F
:1048080091FBFCFC0CF1010CBCF1080FDFF8B4A023
:10481800304EA87895F801E096F800802A4CDFF829
:10482800A090254EA8BF4FF0080C8AF800C01FFAC8
:104838008CFA10FB0AF01EFB0AFE80B2DFF88CA08F
:104848002080A9F800E000244FF0640EB8F1020FB0
:1048580034701C70CAF804408AF801E07FF439AF5C
:104868000FFA8CF1BDE73078A0B901237760337077
:10487800C2F164021A4B00FB02F083FB0023C0174D
:10488800A0EBA3506430707036E70820BDE8F0470D
:104898002BF0ACBA7368F81A8EE7032C96D10D4941
:1048A800097802299AD0044EFCE600BF0D3E00208C
:1048B8009822002060400020A82200208C3E002082
:1048C8009C220020A23E00209A220020A022002044
:1048D800406400207C3E00207F969800803E0020A7
:1048E8006BCA5F6B2DE9F0470569C3681D4028D086
:1048F8000F4606464FF000484FF00009B5FA85F319
:1049080028FA03F2D2431B3B32611540042B16D818
:10491800DFE803F03129211903007B6A002B32D02C
:1049280003F1FF3A1FFA8AFAC7F824903C6A34B1B7
:1049380023682046514698476468002CF8D1002D1A
:10494800DCD1BDE8F0873868716B036889B2984795
:10495800002DD3D1F5E77868B16B036889B2984721
:10496800002DCBD1EDE7B868F16B036889B29847A1
:10497800002DC3D1E5E7F868316C036889B2984720
:10498800002DBBD1DDE7F36A1FFA83FACEE700BF3B
:1049980030B50446006D61710368A26823F0010315
:1049A800036087B0A379009213F004023DD04FF45E
:1049B800805213F00203019244D102934FF48063B2
:1049C8000022039311F00103059237D104930823C1
:1049D8008D07694648BF049318F0DEF86079236DA7
:1049E800A17900F00202002A15BF4FF440324FF4BB
:1049F80080324FF40034002410F0010F586808BFCB
:104A08002246CC074CBF024320EA02025A609A6849
:104A180009074CBF42F0080222F008029A601A689F
:104A280042F001021A6007B030BD13F00203019290
:104A38000BD04FF4005513460295C1E704230493A5
:104A48000C23C5E74FF40053B7E70293B8E700BF5C
:104A580010B50446006DA160036823F001030360EC
:104A6800A37986B013F00402009141D04FF480522C
:104A780013F00203019244D102934FF480636279E8
:104A88000393D1074FF000030493059345BF042314
:104A9800049308230C236946920748BF049318F02F
:104AA8007BF86079236DA17900F00202002A15BF16
:104AB8004FF440324FF480324FF40034002410F0A9
:104AC800010F586808BF2246CC074CBF024320EAB2
:104AD80002025A609A6809074CBF42F0080222F0A5
:104AE80008029A601A6842F001021A6006B010BD06
:104AF80013F00203019207D04FF4005113460291BC
:104B0800BDE74FF40053B7E70293B8E708B50121B2
:104B180002200AF04FF9094B1B7803F00503052B17
:104B280008D0002101200AF045F9002108460AF0C2
:104B380041F9FEE71CF0FEFFF3E700BF502A002012
:104B4800022828BF022010B4084C094B207000EB43
:104B58008002C0EBC20207495DF8044B013003EB49
:104B68004203C0B20B602BF027BA00BF4860002098
:104B7800C6860020D440002008B51AF05FF80AF075
:104B880069FBBDE808401AF041B800BF38B5434B8F
:104B98005A899989914224BF00225A81198ADA894F
:104BA800914224BF0022DA81DA788AB3072A2FD00B
:104BB8003B493C4D91F85300012400210A282C70F0
:104BC8009C70D9713DD00C2865D0DFED377A8ABB4F
:104BD800364C9FED370AA278002918BFF0EE407ACC
:104BE800062A04D8334901EB820191ED050A21799F
:104BF80059B3013A032A4DD8F7EE007A87EE800AB6
:104C08002FF03EFA2388984228BF1846208038BDE6
:104C1800D97921B198780428B8BF04209870204821
:104C280090F853000A280CD00C28CED1DFED227A58
:104C3800002ACDD0072ACBD00A282CD1DFED1F7A45
:104C4800C6E70A20DFED1E7AC1E79B78154A07EE12
:104C5800103A1178B8EEC77A27EE277A07EE901A3D
:104C6800F8EEE77A67EE877AB4EEE70AF1EE10FA23
:104C780010DDC0EE077AFDEEE77A17EE903A102BBA
:104C8800A8BF1023012BB8BF0123DBB28B4238BF6A
:104C98000B46137038BDDFED0B7A99E720540020DE
:104CA800A8510020183100206F1203394456002003
:104CB8006F120338145103080AD7A3390F506E3AFC
:104CC8005304E9386F12833A2DE9F047AA4FAB4EE7
:104CD80019F0B4FFBE421ED2DFF81C83DFF81C9324
:104CE8004446258862197DB14A450DD2052D0BD958
:104CF80033886188C3F30B03994200F0E2801446BD
:104D080025886219002DEFD17168304614360AF0F3
:104D18002DFABE42E4D39A4A1378A3F11701022967
:104D28000FD9984911F83300002840F0F680D800D0
:104D38000144497829B1944911F83330002B00F027
:104D48001481924B5A78022A40F2E180002290495D
:104D58005A701A788F48022A016000F2D48002EB58
:104D680082018D4BC2EBC10203EB4203998C5A8C32
:104D78008A4C9142236001D300225A84884B9A7846
:104D8800042A00F0E98032B91A88B2F5F07F84BFAE
:104D98004FF4F0721A80834DFFF7F8FE2B68824AB1
:104DA8001A40002A00F0E480D80700F1D0805904A6
:104DB80000F1C8801A0700F1C0809B0400F1B6809A
:104DC80025F04AFE10B979482AF05AFC80200AF0EA
:104DD80003FA4FF400700AF0FFF94FF400300AF0BC
:104DE800FBF94FF400100AF0F7F94FF000700AF0E1
:104DF800F3F94FF080600AF0EFF94FF000600AF025
:104E0800EBF91DF0E3FB00213022694830F0F5F89A
:104E1800206827F041FC674B276803F1500102E046
:104E2800043399426DD01A78002AF9D19C78D87841
:104E38008442F5D26049614B0D79614961480A7035
:104E4800614E624C0460C822642111FB05210022D6
:104E580059609A60DA601A615A619A61DA6183F876
:104E6800202083F82120376015F0A6FE584B9FEDCF
:104E7800595A1B88584A9FED596A5079584906EE85
:104E8800903AF8EEE66A1388C5EE265A07EE103A0D
:104E980053881279C1ED005A07EE903AB8EEC77AF6
:104EA800504BF8EEE77A18725A7227EE067A67EED8
:104EB800867ABDE8F04783ED017AC3ED007A19F0F0
:104EC800A5BE63799B077FF41AAF716894F804A0B4
:104ED80030460AF04BF93388BAEB133F04D0143646
:104EE800BE42FFF4FDAE16E773887068AA1FC3F3CD
:104EF8000B039A4204F10601A8BF1A462EF0ECFEF5
:104F0800EDE7012296E700221A70234B2EE720498D
:104F180002EB420201EB82011BE7D8000C1864681F
:104F2800002C7FF405AF1724147001E72E480AF00F
:104F380053F940200AF050F942E72C480AF04CF99E
:104F48002B683AE72A480AF047F92B6832E72948DC
:104F58000AF042F92B682AE79A8AB2F57A7FBFF4F9
:104F68001AAF4FF47A729A8215E718231370E8E69D
:104F780043F001032B6017E7A4B5030830B1030819
:104F88008C3200201C7403087C71030848600020E0
:104F9800D2870020D8400020C6860020D4400020B8
:104FA800445600201088002009600002685D002037
:104FB800E41C0020B843002050460020304D00205B
:104FC800CC020020281D0020181D00202A310020B6
:104FD800F01E0020C0C9FB48D41B002017B7D138E9
:104FE800F41E0020904500200940000201600002E4
:104FF800092000020860000202F00308000004080B
:1050080008B519F01BFE0AF025F919F0FFFDFFF7A6
:105018005BFE0120BDE808402AF0CEBF38B50C4C35
:105028000C4DAC4206D26168204614340AF09EF852
:10503800AC42F8D3084A094B094C146000220949CC
:105048001A705A7008480860BDE8384016F04CBC21
:1050580030B10308A4B50308D440002048600020FC
:10506800C6860020D8400020D287002008B5FFF768
:10507800D5FF19F0E3FD0AF0EDF8BDE8084019F096
:10508800C5BD00BFF0B50C292BD8DFE801F06F2AA9
:105098002A2A4C2A2A2A2B2A2A2A0700046AB2F822
:1050A8000CE097881668674D24F480540462036AFC
:1050B8004468C16923F4005343EA0E3321F4E641FE
:1050C800A84243EA073341EA062100F0B58005F516
:1050D8000065A84200F0B08092684460C161026433
:1050E8000362F0BD046A96899588D2F800E0554FAE
:1050F80024F480740462036A4468C16923F4007369
:1051080043EA062321F07301B84243EA052341EA42
:105118000E017ED04C4DA8427BD092684460C1619C
:10512800C2630362F0BD046A96899588D2F800E0EC
:10513800444F24F010040462036A4468816923F030
:10514800200321F0807143EA061321F4E641B842B6
:1051580043EA051341EA0E2148D03B4DA84245D009
:1051680092684460816182630362F0BD046A938936
:10517800B2F804E01768334E24F001040462056AAB
:105188004468816943EA0E0321F4803125F0020561
:105198009BB221F07301B04243EA050341EA0701DB
:1051A80014D0294DA84211D005F54065A8420DD06C
:1051B80005F58065A84209D005F58065A84205D0A7
:1051C80092684460816142630362F0BDD689158AA2
:1051D800578A23F0080333433D43D68824F44074A8
:1051E80023F00403ADB233432C43E9E7D589178A8A
:1051F800D68823F0800343EA051324F44064558AD3
:1052080023F0400344EA870443EA061344EA85048A
:10521800A6E7D589178AD68823F4006343EA0523CD
:1052280024F44054558A23F4806344EA071443EA7B
:10523800062344EA051470E7158A24F4804444EAF6
:10524800851449E7002C0140003401402DE9F04F56
:10525800F022002183B07948794CDFF80892794D23
:10526800794E7A4FDFF800822FF0C7FE78487949E7
:10527800DFF8F8E1DFF8F8C100221359834200F0A3
:10528800C280B3F1804F00F0CA80AB4200F0C98001
:10529800B34200F0C880BB4200F0C780734500F0FD
:1052A800C680634500F0C580434500F0C480DFF840
:1052B800C4A153457AD00AF5806A534508BF09232B
:1052C80075D014328C2AD8D15D4C634D634E614F32
:1052D80004F18C0802E01434A04564D0A379002BB3
:1052E800F9D023794FEA131909F1FF39B9F1050FFC
:1052F80003F00F03EFD835F8190040FA03F2D2078C
:10530800E9D54FF0010A0AFA03F3013B18402EF0E1
:1053180041FA16F809305249184411EBC002DAD0A4
:1053280051F83000DFF850E1217A00F138439B0A48
:105338001EF8033003F01F0E5B09022B0AFA0EFA5F
:1053480063D0032B66D0012B58D093880093B3FA0F
:1053580083F3C3F11F039BB2DA0800EB820203F068
:105368000703D2F820E09B004FF00F0C0CFA03FC67
:105378002EEA0C0EC2F820E0D2F820E001FA03F37E
:1053880043EA0E03136269460023022214348DF89F
:1053980004208DF805308DF806308DF8073017F0A9
:1053A800B1F9A0459AD103B0BDE8F08F082309EB05
:1053B800C3034FF0010B93F834A00AF01F034FEA20
:1053C8005A1ABAF1020F0BFA03F311D0BAF1030F0C
:1053D80008D0DA457FF475AFD1F814A043EA0A0380
:1053E8004B616EE7D1F81CA043EA0A03CB6168E77A
:1053F800D1F818A043EA0A038B6162E77B694AEA9D
:1054080003037B61A1E70023D1E7BB694AEA0303F1
:10541800BB619AE7FB694AEA0303FB6195E701234D
:10542800C5E70223C3E70323C1E70423BFE7052336
:10543800BDE70623BBE70723B9E700BF4C5C0020A4
:105448008870030800040040000800400010004075
:10545800002C0140001002405871030864710308D1
:10546800905E0020145103080040014000140040E1
:10547800003401400044014080700308014902489B
:10548800FFF730BA145D0020004801400149024886
:10549800FFF728BAEC5C00200034014001490248BB
:1054A800FFF720BAEC5C00200034014001490248B3
:1054B800FFF718BAC45C0020000800400149024800
:1054C800FFF710BA9C5C00200004004002494FF02E
:1054D8008040FFF707BA00BF745C0020014902480A
:1054E800FFF700BA4C5C0020002C0140014902483B
:1054F800FFF7F8B94C5C0020002C01402DE9F04181
:1055080004684E4DA30AAB427AD00AD94C4DAB423F
:105518005FD00535AB4277D0073DAB425DD0BDE8E3
:10552800F081B3F5801F67D0013DAB4259D14FF0F0
:10553800700E022647794FEA970C002968D0B00010
:10554800634685190227D4F80C809F400CEB45036D
:10555800BFB23C4D03F1040C47EA080745F8231095
:1055680045F82C20E760EFF31181502282F312886E
:10557800821905EBC2021369002B34D0136204337D
:10558800821905EBC202576917B11F6053690433CA
:10559800821905EBC202976917B11F60936904333A
:1055A800821905EBC202D76917B11F60D3690433AA
:1055B8000027CAB21F6082F31188304405EBC0008F
:1055C800036A9BB9E3684FF6FE721340E360BDE8D7
:1055D800F0814FF0C00E0426ACE74FF0200E0026F5
:1055E800A8E7BDE8F08105EB0E03C9E7E36843F0DF
:1055F8000103E360BDE8F0814FF0480E012699E70A
:105608004FF0980E032695E74FF0E80E052691E730
:10561800BF08022306FA03F0BB40DB43E768094DE5
:105628009BB23B4087190CEB470CE3600CF1040379
:1056380045F82C1045F8232095E700BF020010001C
:105648004D0010004C5C002030B503685C4D188894
:105658005C4CB4FBF2F20139013AAB4294B283B02C
:1056680089B282B266D05848834263D0B3F1804F82
:1056780060D0A0F5983083425CD000F5806083420A
:1056880058D0524883425BD000F5806083427DD079
:1056980022F4407200F58C3092B283421A80D962AB
:1056A8001C850ED0484A93420BD002F540629342C3
:1056B80007D002F58062934203D002F580629342DC
:1056C80001D100221A8601225A611A883C4992B2F5
:1056D80042F001028B421A8062D0B3F1804F61D050
:1056E8003B4A934260D002F5806293425ED002F555
:1056F800006293425CD002F5806293425AD002F570
:105708009032934258D002F54062934256D002F547
:10571800806293421ED002F58062934208BF09223C
:1057280019D002A84FF0012340F8043D16F0B4FF49
:1057380003B030BD254822F07002834292B2A3D153
:1057480001201A80D9621C8558611A8892B20243D6
:105758001A80C5E708221F4B03EBC20301A893F880
:1057680035408DF80440012300228DF805308DF86E
:1057780007308DF8062016F08FFF1B2CD8D1164B5A
:10578800019301A816F088FF03B030BD01201A80EC
:10579800D9621C8558611A8892B202431A809CE724
:1057A8000022D8E70122D6E70222D4E70322D2E773
:1057B8000422D0E70522CEE70622CCE70722CAE773
:1057C800002C014000A24A040034014000100040AF
:1057D800000400401451030819010001204B9842AD
:1057E8002DD0B0F1804F2CD0A3F5943398422AD015
:1057F80003F58063984228D003F50063984226D0C9
:1058080003F58063984224D003F59033984222D060
:1058180003F54063984220D003F58063984207D08F
:1058280003F58063984208BF092202D00020704720
:1058380008220C4B03EBC20393F834007047002294
:10584800F7E70122F5E70222F3E70322F1E7042252
:10585800EFE70522EDE70622EBE70722E9E700BFBD
:10586800002C0140145103082DE9F04F013085B098
:10587800C3B203930B4602918B4C8C4E002B00F065
:105888009A8032208A4D8B4FDFF82C9224F010F842
:105898004FF4FA7A4FF0100C4FF47A70D9F80430BC
:1058A800C3F30803002B40F0DE80EFF31183002BD5
:1058B80040F0D9802968A26800BF2B689942F9D1C5
:1058C800D7F800E000FB0EF39B1AB3FBFEF300FBD6
:1058D80001314FF0010E0191D9F80430C3F30803E8
:1058E800002B40F08780EFF31183002B40F082807B
:1058F8002B68A16800BF2A689342F9D1D7F800B095
:1059080000FB0BF2521AB2FBFBF200FB0323019AD5
:105918009B1AB3F57A7FDFD3BAF1010ABED1039B94
:10592800002B40F0BD804FF47A7ADFF88C91504616
:105938004FF0100CD9F80430C3F30803002B75D1CD
:10594800EFF31183002B71D12968A26800BF2B687F
:105958009942F9D1D7F800E000FB0EF39B1AB3FB8C
:10596800FEF300FB01314FF0010E0191D9F804302C
:10597800C3F3080313BBEFF31183FBB92B68A168CA
:1059880000BF2A689342F9D1D7F800B000FB0BF2A8
:10599800521AB2FBFBF200FB0323019A9B1AB3F5E0
:1059A8007A7FE3D3BAF1010AC4D1029B013B029387
:1059B800002B7FF466AF05B0BDE8F08FEFF31188D8
:1059C8008CF31288A1682368DB0344BFC6F800E0A3
:1059D800A1682B6832685FFA88F888F31188D7F8CD
:1059E80000801A4400FB08F35B1AB3FBF8F300FBD2
:1059F8000233D2E7EFF311888CF31288A168236889
:105A0800DB0344BFC6F800E0A1682B6832685FFA80
:105A180088F888F31188D7F800801A4400FB08F347
:105A28005B1AB3FBF8F300FB023370E7EFF3118264
:105A38008CF31288D4F808E02368D90303D501232E
:105A48003360D4F808E02B683168D2B282F3118849
:105A58003A68194400FB02F3A3EB0E03B3FBF2F31D
:105A680000FB01317FE7EFF311828CF31288D4F841
:105A780008E02368D90303D501233360D4F808E08C
:105A88002B683168D2B282F311883A68194400FB56
:105A980002F3A3EB0E03B3FBF2F300FB013118E7AB
:105AA800184623F06FFD3EE710E000E0345C00206C
:105AB800385C00203C5C002000ED00E0204B5B6877
:105AC800C3F3080330B4BBB9EFF31183A3B91D4B7B
:105AD8001D4C1868A16800BF1A689042F9D11B4B89
:105AE8001C684FF47A7202FB04F3591AB1FBF4F103
:105AF80030BC02FB00107047EFF31182102383F3D0
:105B0800128811498C680B6813F4803F104B02D03F
:105B1800012018608C680B49D2B20D68186882F3AE
:105B280011880A4B19684FF47A72284402FB01F372
:105B38001B1B30BCB3FBF1F302FB0030704700BF06
:105B480000ED00E0385C002010E000E03C5C002044
:105B5800345C00202DE9F84F8046FFF7AFFF254E53
:105B68002549DFF8A0E0254A254D844610274FF443
:105B78007A740120DEF80430C3F30803D3B9EFF3D5
:105B88001183BBB90B68D2F808A000BFD1F8009008
:105B98004B45F7D1D6F800B004FB0BF9A9EB0A097D
:105BA800B9FBFBF904FB0393A3EB0C034345E1D3D7
:105BB800BDE8F88FEFF3118A87F31288D2F808B09E
:105BC8001368DB0344BF2860D2F808B00B68D5F827
:105BD80000905FFA8AFA8AF31188D6F800A09944EF
:105BE80004FB0AF3A3EB0B03B3FBFAF304FB09333F
:105BF800DAE700BF3C5C0020385C002010E000E0E1
:105C0800345C002000ED00E02DE9F04FDFF830C1F2
:105C1800474A4849484E494D8046102718F1FF38F1
:105C2800C0F08480DCF80430C3F30803002B5CD197
:105C3800EFF31183002B58D10B68946800BF0868F4
:105C48008342F9D1D6F800904FF47A7000FB09FE30
:105C5800AEEB040EBEFBF9FE00FB03EEDCF80430ED
:105C6800C3F308034FF47A740120FBB9EFF31183EF
:105C7800E3B90B68D2F808A000BFD1F800904B45F3
:105C8800F7D1D6F800B004FB0BF9A9EB0A09B9FB68
:105C9800FBF904FB0393A3EB0E03B3F57A7FBDD2A4
:105CA800DCF80430C3F30803002BDFD0EFF3118ACC
:105CB80087F31288D2F808B01368DB0344BF286062
:105CC800D2F808B00B68D5F800905FFA8AFA8AF320
:105CD8001188D6F800A0994404FB0AF3A3EB0B0340
:105CE800B3FBFAF304FB0933D5E7EFF3118487F329
:105CF8001288D2F808901368D80303D501232B60C3
:105D0800D2F808900B682868E4B284F31188D6F8B2
:105D180000A04FF47A7400EB030E04FB0AF3A3EB24
:105D28000903B3FBFAF304FB0E3E97E7BDE8F08FD7
:105D380010E000E0385C00203C5C0020345C00206F
:105D480000ED00E030B4EFF31183102282F31288E3
:105D58000649074C0A680748013200250A60256091
:105D6800DBB2026883F3118830BC7047385C0020CE
:105D7800345C002010E000E00F4B1B88014643B95B
:105D88000E4B0F4A1B7810680BB981F0010109F01E
:105D980007B80C4B5A691AB118B91A6810605874C8
:105DA8007047094A18681188084A92FBF1F20121E4
:105DB80002605974704700BF105C0020125C00201C
:105DC800145C0020185C0020305C002020A1070033
:105DD8001D4B70B59C68236D626BDD69C2B1A36B06
:105DE8002BB12B0702D5236D08221A6270BD2A0633
:105DF800F7D5A26A616A8A4220D0511CA069A162C3
:105E0800825C2069266D81423285EAD3A362E8E785
:105E1800A906E4D5E26A22B1988C216B80B290473A
:105E2800DDE7E1699B8C6069DBB24E1CE661435497
:105E3800E169E368994228BFE261D0E7226D1368FF
:105E480023F080031360CCE7542A00201D4B70B563
:105E58005C68236D626BDD69C2B1A36B2BB12B0744
:105E680002D5236D08221A6270BD2A06F7D5A26AE8
:105E7800616A8A4220D0511CA069A162825C2069B3
:105E8800266D81423285EAD3A362E8E7A906E4D504
:105E9800E26A22B1988C216B80B29047DDE7E16914
:105EA8009B8C6069DBB24E1CE6614354E169E36890
:105EB800994228BFE261D0E7226D136823F080037E
:105EC8001360CCE7542A00201D4B70B51C68236D65
:105ED800626BDD69C2B1A36B2BB12B0702D5236DB1
:105EE80008221A6270BD2A06F7D5A26A616A8A4238
:105EF80020D0511CA069A162825C2069266D814274
:105F08003285EAD3A362E8E7A906E4D5E26A22B1BA
:105F1800988C216B80B29047DDE7E1699B8C6069C2
:105F2800DBB24E1CE6614354E169E368994228BF3D
:105F3800E261D0E7226D136823F080031360CCE799
:105F4800542A002070B4EFF31186502383F312888B
:105F5800836B1A68D20720D45D686DB9446A826A77
:105F6800944217D081691144D9600ED9A21A5A6097
:105F78008462002280F854201A6842F00102F1B2CB
:105F88001A6081F3118870BC704701698A1A5A60D7
:105F98008562EEE7012380F85430F1B281F311886D
:105FA80070BC704703685B6A03B11847704700BF4D
:105FB8002DE9F04FBF4B1E788BB0002E40F0BC800F
:105FC800BD4BBE4C1D78DFF814A3DFF81493DFF83F
:105FD800148305F00105A4F10A0B54F80A3CBBB17F
:105FE800CC2707FB06B7184607F0DAFE80B154F84D
:105FF8000A0C07F0CDFE14F8023C8BB9242831D0E6
:10600800F5B154F80A3C184607F0CAFE0028EED14C
:106018000136032E04F1CC04DFD10BB0BDE8F08FBC
:10602800012B23D0022B2BD0032B37D0042B67D086
:10603800052B40D0062B4FD054F80A2C1346D2E734
:1060480054F80A3C23281A4600F087819C4991F8A5
:1060580032108142C7D19B4BCAF80090C3F80C801C
:106068001346C0E7012304F8023CCAE74D2854F858
:106078000A2C0CBF0223002304F8023C1346B2E7A3
:1060880000233C2804F8023C45D03E28D4D1012204
:10609800032304F8012C04F8023CB2E7C02814D802
:1060A8000022042304F8050C04F8040C04F8062C58
:1060B80004F8023CA5E714F8063C14F8052C9A42AB
:1060C8002FD814F8043C834203D0002304F8023C80
:1060D80097E7062304F8023C14F801ECBEF1000F20
:1060E80000F07E81BEF1010F00F0C281013600236D
:1060F800032E04F8023C04F1CC047FF46EAF8CE765
:1061080014F8043C04F8030C5840052304F8040C64
:1061180004F8023C75E7032204F8013C04F8022C59
:106128006FE714F8042CF9184240013304F8042CE2
:1061380004F8063C887264E7634B186800283FF44B
:106148006CAF08F0BDFFDFF8A0A1604DDFF89C91AF
:10615800DAF8000007F024FE00283FF45EAFDAF812
:10616800000007F015FE09281BD03F2819D02B681E
:10617800002B66D1042800F0A6810C2800F0E680E8
:106188007F28E5D0A0F12002D2B25E2AE0D80BB970
:106198002028DDD05A1C09F803002A6025F070FA7F
:1061A800D6E72C68002C5AD1494B264603F594783B
:1061B800002E08BF1E4608334345F9D1002E00F0D3
:1061C8007681A3F1080B3068DBF80020075D135DCA
:1061D8009F42204402EB040140F06781671E4F4450
:1061E80022460BB9FD2A5CD907F8013F01322A6023
:1061F80010F8013F11F801EF9E45F2D00AB1B345FE
:1062080012D0344825F044FAB34508D356F8080BA1
:1062180025F03EFA092025F033FA5E45F6D92E48D6
:1062280025F036FA2A680024944291D2661E4E441C
:1062380016F8010F25F024FA2B6801349C42F7D395
:1062480086E70C2800F082800A2851D00D284FD00C
:106258007F2800F0FA80FF2B3FF67AAF92E71C4FB9
:106268004FF0000B07F594785E4602E00837474583
:106278000DD022463968484609F042FA0028F5D17F
:10628800BB46002EF2D13E4608374745F1D1002ED5
:1062980099D1BBF1000F3FF45BAF0E4825F0F8F938
:1062A800B4E7511C202009F80200296009F80130E0
:1062B8000A46A4E7583800200D3E0020128200202C
:1062C800685D002000ED00E0542B00205C2C0020CD
:1062D8004C540308547A03085C7A0308FC9F002096
:1062E800EFBEADDE0400FA05582B00205C2B002021
:1062F80025F04FFA23217C482EF096FE002800F066
:10630800E080A0EB0900286088B1431E19F803104B
:10631800202940F0E68009EB030204E012F8011D91
:10632800202946D10346581E002BF7D12B604FF485
:106338008072002148462EF060FE6C4B1B78002BC3
:106348003FF46BAE6A4825F0A3F901E7694825F0E8
:106358009FF9674825F09CF9FAE667496748C978C4
:10636800674ADFF8CCE11360003118BF01210170E2
:1063780064495160402193601173557362496348C1
:106388000B600432CEF80020584A0123137025F020
:1063980005FB574825F07CF94FF400600BF012F824
:1063A8005B4B93F83230232B00F0938014F8023CB7
:1063B80040E62B60574C002204F5947809F8032036
:1063C80002E00834444578D0216848460FF03CFE86
:1063D8000028F6D0444570D2636898470023A5E7A3
:1063E8004D4BADF822E00FCB0DF1280C02AF87E83A
:1063F8000F004CF824ED14F8051C14F8033C06941F
:1064080004EB010E624639464FF0010C06A8CDF8A0
:106418001CE0ADF820308DF824C0FCF71DFBE8B96E
:10642800019F002304F8023C002F3FF4F1AD54F81B
:106438000A0C29F063F9013654F80A0CB847032E00
:1064480004F1CC047FF4C9ADE7E5013B00223348F1
:106458002B6009F8032025F01BF979E6029A304BE6
:1064680003923946A4F10A0002930DF0DFFED7E744
:1064780014F8053C14F8032C0694234407936E2A59
:106488004FF0000308930993ADF820207FF42EAE57
:1064980006A809F0B7F906A809F0A8F906A809F0AE
:1064A800A5F906A809F0A2F920E62246A6E61D48A5
:1064B800A3F1080B25F0ECF8A8E61B4825F0E8F84E
:1064C8008CE7286820E708480FF007FA0BB0BDE80A
:1064D800F08F164A14F8023CC2F80C80CAF80090F3
:1064E800A8E5034666E700BF5C2B0020583800206B
:1064F8005C7A0308647A030848600020202300209F
:10650800F81B0020D5D70008582B0020907A0308E4
:10651800685D00204C540308945103088C7A0308E2
:106528006C890020547A0308707A030800ED00E0B3
:10653800542B00202DE9F04F2DED068BA74BA84AD0
:106548001C7897B000F59C41203181460B91116071
:10655800002C00F0EC86A34A1268904240F2E680D4
:10656800A14A06921668A149A14A0591013C1C70EE
:10657800A04B049206F480560893002E40F0E48065
:106588009D4B1B78022B01F03881042B01F0A6816A
:10659800012B01F05A81994B9945089B9B7800F291
:1065A8009785002B40F09885954B0793069B1E68AE
:1065B80016F4805740F08986DFF878A2049BB3F977
:1065C8000620059B5D8BAA42B4BF002501258D4B93
:1065D8001B68DC0040F1C280079B1B7813F00103A5
:1065E80000F0C3800599498C914241F35882002DEF
:1065F80040F0C280844C94F88C20002A40F0BC8083
:10660800824A8349106890F82D0000220A604A6087
:106618008A60804A002840F0B0801070002B40F05B
:10662800B1807D4B1A78002A40F014810599049CAA
:10663800488BB4F90070898BB4F90240B842B4BFF2
:106648008026002646F04003B942D8BF33469B084F
:1066580043F080068442C8BF3346049F43F0400697
:106668008C42B8BF33469B08B7F90440B7F90660B7
:1066780043F080078442C8BF3B4643F040078C4242
:10668800B8BF3B469B0843F080075F4C8642C8BFB3
:106698003B4643F0400794F88EE08E42B8BF3B4635
:1066A8009E4501F01D84A4F8902084F892205B494F
:1066B80084F88E300E78002E01F023835F2B01F0D2
:1066C80096836F2B01F0AD83079B1B78DE0700F1E3
:1066D800C18094F89210002940F0BC80B4F9903041
:1066E800322B40F3B78094F88E300120572B84F872
:1066F800920000F0A180069A1268550741F16D8258
:106708005A2B41F06A8294F89430002B41F0DB87D1
:1067180094F8963083F0010384F89630002B42F009
:106728002A800C2029F062FB3D4D94E02E4B069305
:106738001E682F4B2D4A049306F480562D4B059264
:106748000893002E3FF41CAF00212E4809F014FCDA
:1067580000287FF415AF1DF0C5F811E770023FF56A
:106768003BAF079B1B7803F00103274C002284F8FA
:106778008C20002D3FF444AF264A01211170002BD4
:106788003FF44FAFF1067FF54CAF264B1B78DA0686
:106798003FF547AF002F7FF444AF1BF0A5FE00285C
:1067A8007FF43FAF1D4B1B78002B01F093871E4BE6
:1067B8009B78002D41F0D1873BB11C4A1C4B1268D5
:1067C8001B689B1A002BC1F2DC8710200E4C29F0A5
:1067D8000DFB012384F88D3023E700BF50430020D0
:1067E800F44200204C430020445400203C5D00202B
:1067F80014640020304D0020E2310020404B4C0052
:106808000D3E002004310020481C0020D440002008
:106818002C320020C01E0020F73C0020CC020020B3
:10682800D0400020E863002044310020385C00207C
:10683800744B002008440020874B884A19684FF49D
:106848007A73B3FBF1F3C3EB431103EB8103DB0072
:10685800A2F8A830824D069B1B685F0700F19B8653
:106868000DF150097F4E09950022C9F804203446DD
:10687800149240F6330B4FF0190840F28337049D09
:1068880002E00434544520D0A178E378994218FBFB
:106898000170F6D26178043118FB037335F91110D1
:1068A8005945A8BF5946B1F5617FB8BF4FF461712A
:1068B8008142E6DD9942E4DC21782729E1D848467F
:1068C800043409F049FB5445DED1674A099D137821
:1068D800664A99E8030082E80300002B40F04386EB
:1068E800634B1A78002A00F0BB85624B0A935F4815
:1068F800012109F041FB002840F0DE82089BDB788B
:10690800002B40F0D9825C4B09932B881FB227F0EB
:1069180001071FFA87F84345A5F8008000F0EC87C7
:10692800564F4FF002090E204FF0140A4FF0FF0B9C
:1069380087F8009087F801A087F802B029F056FA86
:1069480049464A48B5F8008009F016FB002841F08E
:106958001D8228F002039BB243452B800BD0474B86
:1069680002201421FF2218700E2059709A7029F005
:106978003DFAB5F80080424B424A197850680C93AA
:1069880018F0030F08BF81F00201C1F340010B9218
:1069980008F006FA2421354809F0EEFA30B9079ACA
:1069A80013785F0744BF23F004031370099B1B6827
:1069B80013F00A0F11D006212C4809F0DDFA00283F
:1069C80001F044802B88580641F1A8810721274807
:1069D80009F0D2FA002840F0B2870C21234809F0C8
:1069E800CBFA2A88002800F0478342F480739A4241
:1069F8002B8009D0214B022214211A700E20FF226D
:106A080059709A7029F0F2F91F4B1B78082B00F087
:106A18003F830E2B00F03C83069BD3F8008018F4CC
:106A2800806F6BD0194B1B79002B00F0308214213A
:106A38000E4809F0A1FA002840F02E8226F058FDF1
:106A4800012029F015F9002855D0DFF844A00027C7
:106A58004FF0CC0BA14620E034540020A851002070
:106A6800D0400020B84300206856002004310020A0
:106A780058380020D84000207C400020342F0020C7
:106A8800035C0020045C00208C320020943E00202F
:106A980008820020DFB2022F2CD80BFB07F87B1CE2
:106AA8005AF80840002CF5D1032290F902300294DC
:106AB8000192C278E24951F82220009218462246F3
:106AC8002346012128F0E4FE034607EB470000EBCC
:106AD8000010099353B121460AEB8000CC222EF016
:106AE8008CFA099B4AF808300137FFB224F0ECFA17
:106AF8000028D0D14C46069BD3F80080079B93F81A
:106B080000A0D04B1AF0010A00F0388201221A7056
:106B18000A9B04991B68B1F906105A89CA480127CB
:106B28009142077080F21082C84B4FF07E521A6073
:106B3800059BC74FB3F81890049B97F90420B3F945
:106B48000030387897F801C0002AA3EB090714BF72
:106B580001224FF0FF32002FB8BF7F42B7F5FA7F0E
:106B6800A8BF4FF4FA77B84280F2EB813F1A07EEDC
:106B7800907AF8EEE77AB74F9945C7ED007A03DDCA
:106B8800F1EE677AC7ED007A049BB3F902E0AEEB49
:106B98000903002BB8BF5B42B3F5FA7FA8BF4FF4D7
:106BA800FA73984280F2CA811B1A07EE903AF8EEFF
:106BB800E77AF145C7ED017A03DDF1EE677AC7EDB3
:106BC800017A049BB3F90400A0EB0903002BB8BFBA
:106BD8005B42B3F5FA7FA8BF4FF4FA736345CCBFA5
:106BE800A3EB0C03002302FB03F207EE902AF8EE56
:106BF800E77A4845C7ED027ABCBFF1EE677AC7ED80
:106C0800027A18F4805800F07681B1F5FA6F924B49
:106C1800A8BF4FF4FA61B1F57A7F1A78B8BF4FF47C
:106C28007A71A1F57A71002A41F080808B4ADFF8E9
:106C380044E282FB0130CB17C3EB6013581C6FF0A2
:106C4800630C3EF910003EF913E00CFB0313A0EBB4
:106C58000E0003FB00F382FB0312DB17C3EB621386
:106C68009E440FFA8EFE07EE90EAB8EEE78A87EDAB
:106C7800038AB8F1000F40F09C832B885A0640F134
:106C8800FB807749774A91ED018AD2ED019A92ED1E
:106C9800026A91ED034A92ED030A91ED029A92ED90
:106CA800007AD1ED005AD7ED011A97ED002A6E4A05
:106CB8006E4938EE445A79EEC63A77EE007A65EEB8
:106CC800233A75EEC96A75EE890A37EE401A66EE00
:106CD800A76AB0EE633AA0EE813A13F00303B0EE70
:106CE800665A78EE044A79EE867AA0EE815AF0EE7A
:106CF800638AA4EEA73AD4EEA78AA4EEE75A33EE45
:106D0800263AF0EE687AF0EE674AF6EE008A35EE3B
:106D180088AAE0EEC14A28EEC33A35EE635A77EE08
:106D2800293A77EEE67AAAEE233A25EE285A76EE45
:106D3800403A34EE49AAE0EE817A74EEA64AAAEE09
:106D4800235A34EE094A37EE697A64EEA84A63EEAC
:106D5800036AE4EE074A75EEC85A36EE006A67EE33
:106D6800A87AB0EE667A95EE057AE5EE056AE5EE64
:106D7800867AB1EE648AF0EE665AF0EE476AB1EEB2
:106D8800674AE8EE246A63EE270A67EEA43AE4EE5F
:106D9800275AB1EE450AB0EE609AB0EE631AA4EE37
:106DA800277A23EE244AE7EEA76AA5EE249AA0EEF6
:106DB800031AE8EE245AB0EE448A31EEA16AE0EEF6
:106DC800240AA5EE278A66EEA16A72EE028AE5EE2B
:106DD800033A61EE211A26EE096AA4EEA47AA0EE1F
:106DE800274A0CBFD7ED022ADFED212A82ED005A8F
:106DF800A2EE256AE8EEA06AE2EE081A73EEA33A5C
:106E080027EE227A34EE044AF0EE005AE3EEA26A44
:106E1800A2EE846AA1EEA57AC7ED016AC1ED366AD1
:106E280081ED356A87ED006A81ED377A82ED013AA6
:106E3800C2ED027AC2ED034AF3B987ED027A1BE08C
:106E4800387303080E3E0020F81E0020741E002030
:106E58001C310020A43E0020A02200201F85EB51F9
:106E6800D002002084020020BC020020481C002020
:106E78000000000058460020BAF1000F40F01B81C6
:106E88001BF094FD17B0BDEC068BBDE8F08F079B97
:106E98001B78D9077FF5D2AD4FF40F7028F066F94B
:106EA80000283FF428AE0DF025FA4FF40F7028F0B3
:106EB800FFF80028F7D11EE69A4B09931B689B0739
:106EC8007FF523ADB5F8008018F0010F7FF441ADD0
:106ED80048F0010398452B803FF43BAD924B0222CA
:106EE80014211A700E20FF2259709A7028F07EFF24
:106EF800B5F800802DE5059B5A8B9142C0F2A2841B
:106F0800B1F5FA6FD4BFC2EB0101C2F5FA614FF4D3
:106F18007A7303FB01F185480378C2F5FA62B1FB85
:106F2800F2F1002B3FF482AE4378814A01FB03F172
:106F380082FB0123C917C1EB631177E6DFED7D7A88
:106F480037E6DFED7C7A16E6B1F5FA6F80F24E840B
:106F5800187A8B1A03FB00F3C2F5FA6293FBF2F37B
:106F6800C3F1640307EE903AF8EEE77A9FED727A80
:106F7800724B67EE877AC3ED007AD9E51B780693E2
:106F8800002B7FF4C5AD6E4A1268002A3FF4C0ADED
:106F98006C4A079212F8030CDFF8E0B11146D71ECD
:106FA8001BF078FA9BF80090079A002800F0BC853F
:106FB800069BB9F1000F53D107F1080178791BF04E
:106FC80069FA002841F075835F49B87A1BF062FAC4
:106FD800002800F0BC85B9F1020F41F066835B49D7
:106FE800F87B1BF057FA002841F05B835849387D3D
:106FF8001BF050FA002800F0BC85B9F1040F41F0ED
:107008004C835449787E1BF045FA002841F04183AF
:107018005149B87F1BF03EFA002800F0BC85B9F151
:10702800060F41F032834D4997F823001BF032FADE
:10703800002841F026834A4997F828001BF02AFACD
:10704800002800F0BC85B9F1080F41F016834549C6
:1070580097F82D001BF01EFA00283FF459AD0923BC
:107068001A4602EB820217443F4A7878B9788BF8BF
:107078000030107051704BE522F480739BB29A4235
:107088002B807FF4B7AC394B1B78082B7FF4C1AC4D
:107098002A8822F040039BB29A422B803FF4BCAC72
:1070A800214B022214211A700E20FF2259709A7067
:1070B80028F09CFEB0E40C9B19780B9B01F00101B1
:1070C800186807F06DFE17B0BDEC068BBDE8F08FB1
:1070D80013B9089A01239370254B089A1D7892F8E2
:1070E800214007931B201BF00DFA012C05F0010825
:1070F800814600F0938605F00205089A1D4E92F825
:107108002030DFF87CA01C4F09959346052B00F230
:107118002587DFE813F0BF00B5003700FD00FF004A
:10712800F20000BF7C400020342F0020A022002065
:107138001F85EB51000000000AD7233C741E002075
:10714800103E0020022F00200C2F0020112F0020BD
:10715800162F00201B2F0020202F0020252F002075
:107168002A2F00202F2F0020143E00208C320020D0
:107178000D3E002050460020CC4000201500002085
:10718800CC020020012C04BF05238BF82030B8F175
:10719800000F12D0059B3088B3F91810002213464F
:1071A80061F30F0260F31F4261F30F03049861F368
:1071B8001F4303600323426009939E4DDBF81410BC
:1071C8002A68914280F08D8547F230510322CBF82E
:1071D8001C108BF8202002200AF0F4F81CF082FB27
:1071E8002968DBF81C200A440421CBF818208BF806
:1071F8002010012C40F0F8862A68DBF8181091421C
:1072080080F0AC869AF8000020B91BF07BF90028C2
:1072180040F0A4863A6822F002023A602A6873882D
:10722800642101FB03234FF480600022CBF8103067
:107238008BF820208BF803200AF094F89BF8203074
:1072480064E71BF065F9012807D17A4D72882B682D
:10725800642101FB0233CBF81030B9F1000F02D0E2
:10726800B379002B4BD1012C00F07886714DDBF8F7
:1072780010102A689142C0F0C48601238BF8203090
:10728800012C3AD0F379012B46D01BF0C1F89BF8BA
:1072980020303BE7B8F1000FD3D1099D4FF480604F
:1072A800B9F1000F00F048830AF074F8089A002337
:1072B8001361002D3FF47AA9284628F097FD069B14
:1072C8001E6816F480573FF477A91D215A4808F024
:1072D80053FE00287FF470A9584B03F1500A03E0CD
:1072E80004339A4500F040861A78262AF8D199780E
:1072F800DA789142F4D2FFF761B94E4D8EE71BF070
:1073080087F803224FF47A738BF82020CBF81C30CF
:10731800484D60E7474D6CE71BF07AF8032240F6CA
:10732800B8338BF82020CBF81C30424D53E7444F3C
:107338003B78002B01F00A81424BDFF81881DFF817
:1073480018B1DFF818A1059345465E4604909946A2
:107358000EE019F804109847032C28DC88B93B780C
:107368002AF8020F01349C4205F1040580F23881A5
:10737800072CE1B23046DBF80430EADD984700B26A
:10738800EDE738F824206B88801A4FF47A719B1A3D
:1073980001FB00F040F6CA0290FBF3F0084490426B
:1073A80040F2EE23A8BF10469842B8BF184600B274
:1073B800D5E71D21204808F0DFFD28B100F0A8BD61
:1073C8000436A6423FF459AC31782629F8D1B27870
:1073D800F3789A42F4D2089BDB78002B7FF44DAC0B
:1073E800154808F0C9FDDFED187A002801F0B680CD
:1073F80038EE678A154A1649FDEEC87ACDED047A4B
:10740800BDF910301B0382FB0302DB17C3EBA2128A
:10741800C9F57A731BB203FB02F343F30F334B44F2
:1074280007EE903AF8EEE77A0123C7ED037A0B707E
:1074380023E400BF385C002004310020B84300205A
:10744800804400203C5D002000007A44D34D621047
:10745800EC1E002094440020E0420020461C00203E
:10746800DFF82C93DFF82CA3B84F099209F15A08DA
:107478004FF0010B494619F8010C1BF00BF800B34B
:1074880099F8040099F8023099F803E000EB4001FC
:1074980007EB8101013BD1F8A02003EB43035344E0
:1074A80093420ED097F8CC20C1F8A0300BFA00F028
:1074B80022EA0000099B81F89CE0C1F8A43087F813
:1074C800CC0009F10609C145D4D1A14BA14A0A93C0
:1074D8001946A14BDFF8C0A2126809681B780B9106
:1074E8000993AAF19C094FF0000B9046DAF8043092
:1074F80083B31F7877B3DAF80820A8EB0202002AD2
:107508000CDB99F8CC20012101FA0BF122EA0102E7
:1075180008F5FA7189F8CC20CAF80810099ACAB196
:107528009AF8002059780432D2B2002940F0BD827E
:1075380005990498098B30F9122001F1C80082429C
:1075480040F3248599F8CC109A7841FA0BF3D807C0
:1075580040F1AE850BF1010BBBF1040F0AF10C0AE7
:10756800C4D1FFF7C4B97D4B03E004339C423FF418
:10757800B7A919782329F8D19878DA789042F4D203
:10758800774808F0F9FC00283FF4AAA9142028F04D
:107598002DFCFFF7A5B96D4C94F896305BB1079BAD
:1075A8001B78DE0707D5049BB3F90620059B5B8B88
:1075B8009A4200F36F851121694808F0DDFC002824
:1075C80000F05B8294F89A302BB994F8943013B990
:1075D8003223A4F89830012384F89A30FFF740B991
:1075E800DDF810905F4A06925F49126842F2010A7C
:1075F800A1FB091B12EA0A0A4FEA9B1B00F03A8218
:107608005A4D5B48544C5B492E78007826700870B8
:107618001EB158490E7886F001064C4C0F2184F8AB
:107628002410002B00F08583059D534BB5F826C028
:10763800B5F824E0059D109318462D8B00784F4B24
:10764800129594F8255009954D4D0495A3FB0053C8
:107658005B0803EB4303C31ADBB20F90CDF834C0C9
:1076680002F480520C9304F128000BF59673CDF8C0
:10767800449097F80080DDF82490DFF820C1099441
:107688003F4C0E91139200210A930896CDF81CE006
:10769800089B002B00F0C782099B079D33F9112036
:1076A8001FFA82FEAE454FEA410303D30D9DAE4556
:1076B80040F2FE825CF82120934580F0BE82E25EB3
:1076C800BAF1000F40F0D38201314145E25200F196
:1076D8000600DDDB0E9A099C2A4B84F824200F2A29
:1076E80049460CBF01220022DDF8449084F8251099
:1076F8001A7000F02583244B1D491E4ADFF854B048
:1077080008931C46042001230B70137009F05AFEDD
:10771800DBF80030A1686268E3605B1A934284BFBB
:10772800002384F82130069B3C781E68002C00F06A
:107738001187059A154DB2F824E0178B104916F4F5
:107748008056284640F0358332463AE0481C0020EF
:10775800D8400020385C0020014D0020B8430020AC
:107768000431002044540020D34D6210BC42002054
:1077780074020020750200206D430020ABAAAAAA5B
:107788001464002098320020304D0020C8440020A6
:10779800192E0020A4510308E41C00207043002087
:1077A8006F12833F437803EB830303EB830303F2F6
:1077B800EE239BB20132A24221F8023B00F1020003
:1077C8000ED015F81230002B00F07682022BE9D08B
:1077D80001320B8821F8023BA24200F10200F0D1ED
:1077E800109A137801331370FEF7C7BE1B7AC3F1E2
:1077F800640307EE903AFFF7B7BB059A0499537DE7
:10780800D27D013B31F913301AB1C3F53B6308331C
:107818001BB2A3F57A7307EE903A1FED1F7AAD4AB3
:10782800F8EEE77A40F2FF3167EE877AFCEEE77A06
:10783800CDED077ABDF81C308B4228BF0B4613806C
:10784800FEF7A9BE4146FFF766BBA34CD4F88830C3
:10785800A9EB0303002BFEF69EAEA04AA04B527C78
:10786800059933F812308A7DDFED9E6A9FED9E6A96
:10787800C97D9BB207EE102A07EE903AB8EEC77A98
:10788800F8EEE77A27EE267A67EE867A0B9AC4F83E
:107898008820C7EE876A40F2FF32FCEEE67ACDED2B
:1078A800077ABDF81C30934228BF134609B1D31A92
:1078B8009BB28E488E4D01788E4C35F81160226847
:1078C80025F81130921B13440131824D236001F0D9
:1078D8000F021B0902702B80FEF75DBEFEF7EEF863
:1078E800854B864A1B68C31A93427EF754AE794B80
:1078F80000221A80FEF74FBE0221814808F03CFBA7
:1079080000283FF426A82F8018F0020F7FF433A830
:1079180048F0020343452B803FF42DA8794B0222FF
:1079280014211A700E20FF2259709A7028F05EFAFE
:10793800B5F80080FFF71FB809F014FDB6E4724AE5
:10794800B2F90030002BB8BF5B42B3F5E17FBFF658
:1079580044A8B2F90230002BB8BF5B42B3F5E17F0F
:10796800BFF63BA8694B93ED096AD3ED076AD3EDDF
:10797800057A93ED037A76EE866A37EE277A76EE05
:10798800A66AF7EE007A37EEE66A37EE077AB0EEC7
:10799800C66AF0EEC75AB4EEE56AF1EE10FAB4BF63
:1079A800B0EE655AB0EE465AB5EE405AF1EE10FA0E
:1079B80040F04183DFED567A9FED560AB4EEE56A52
:1079C800F1EE10FA44BF9FED536A76EE677AB7EE90
:1079D800006AF4EEC66AF1EE10FAC8BFDFED4E6A2F
:1079E800B5EEC07AC8BF76EEE77AF1EE10FA48BF76
:1079F800F1EE677AB6EE008A27EEC88A38EE000AFA
:107A0800FDEEC07A17EE903A2033402B40F2818584
:107A18009FED420A424FDFED417A87ED000ABDEE45
:107A2800C87AC7ED017A17EE103A2033402BC7ED1C
:107A3800027A00F26A85B0EE480A08F0CFF80A2008
:107A480087ED030A28F0D2F9FEF7C7BF2A8822F08B
:107A580040039BB29A422B803EF4B8AF294B0222D6
:107A680014211A700E20FF2259709A7028F0BEF95E
:107A7800FEF7ACBF2B490E78CAE594F89430002B7A
:107A88003EF4EEAE079B1B7813F001037EF4E8AEDC
:107A9800012284F8943084F89520FEF7E1BE0E4C5C
:107AA800012284F88C20FEF767BE012900F0E484E7
:107AB80099F8CC20012303FA0BF30BF1010B1343C4
:107AC800BBF1040F89F8CC300AF10C0A7FF40EAD33
:107AD800FEF70DBF08640020481C0020945B0020BE
:107AE800B45B00200000C84200008044E33100205D
:107AF800E8310020E4310020E81B002060E3160094
:107B080004310020342F00208040002094020020FF
:107B1800A7DFA834DB0FC93FDB0F49400000000096
:107B2800D0020020014D0020511D78791AF0B2FCD6
:107B380000283FF449AAB9F1010F40F0BA8507F1CE
:107B48000D01B87A1AF0A6FC002840F0AE85C049AD
:107B5800F87B1AF09FFC00283FF448AAB9F1030FFC
:107B680040F09F85BB49387D1AF094FC002840F00E
:107B78009485B949787E1AF08DFC00283FF448AA0C
:107B8800B9F1050F40F08585B449B87F1AF082FC39
:107B9800002840F07A85B24997F823001AF07AFC59
:107BA80000283FF448AAB9F1070F40F06A85AD49AB
:107BB80097F828001AF06EFC002840F05E85AA4964
:107BC80097F82D001AF066FC00283EF4A1AFB9F131
:107BD800090F3EF49DAFFFF742BA5D2B00F09D847C
:107BE8005B2B00F06A825E2B00F01A85562B00F0A2
:107BF8001B85972B00F03885A72B00F009859B4D36
:107C08002A88920740F0DA84A3F1B702072A00F223
:107C18007482DFE812F06D02720272027202680268
:107C2800720263025E02079B002B3FD05CF82120A2
:107C380093454FEA4103FFF442AD8D4A8C4DD25C27
:107C480005EB030E002A00F09480022A47D19EF823
:107C5800012002EB820202EB820202F2EE2292B2D1
:107C6800032933DD12B2BAF1000F3FF42DAD0C9D9C
:107C780020F81520B9F1000F03D10F9D022D7FF6D2
:107C880023ADB0F802900288B0F804E04A44964464
:107C9800784A0FFA8EFE82FB0E52774DA2EBEE72F7
:107CA80025F803E012B24FF001090DE51A464B0022
:107CB8000A9D4CF8215003E5D3B2022B04D9032BBB
:107CC8007FF486AD734675E53B4673E5012505FAF5
:107CD80001FE0E9D25EA0E0512B20E95F0E4E25A59
:107CE800BEE7664A1278002A7FF46EAAB8F1000F40
:107CF8003FF46AAA012C40F031819BF82030FFF74D
:107D080005BA31465E4808F037F9002800F0C4800B
:107D180084F893601CF014FAFEF7D6BC43F04002D6
:107D280093422A807FF49AAEFEF750BE5B78FFF745
:107D3800FCB8544B544A109201221A70534B0493C6
:107D48001B214F4808F018F900287FF4D4AC504B99
:107D5800DFF840B108931946DBF80030CA688B6039
:107D68009B1AC82B00F21B84069B1E6806F48056DB
:107D780036E5CAB2022A40F27C83032AAFD1129AAE
:107D8800139D079E002D08BF324669E728F00102BF
:107D980092B242452A803FF4B7AD0E2087F8009092
:107DA80087F801A087F802B028F020F8B5F800801D
:107DB800AAE500220FE0437803EB830303EB830378
:107DC80003F2EE239BB20132A24221F8023B00F1FA
:107DD80002003FF405AD15F812301BB1022BEAD0B2
:107DE8000B88F0E7D3B2032BFAD83B46EBE7B2F5A2
:107DF800FA7FFEF62FAD94F89230002B7EF42AAD70
:107E0800079B1B78012213EA020584F8922000F0F0
:107E18006F831BF067FD154DFEF71DBD0025FFF7AD
:107E28006CB9B2F5FA7FFEF615AD94F89230002BD6
:107E38007EF410AD079A12780121D70784F89210C2
:107E480000F17F831CF07CF9084DFEF704BD00BFEC
:107E5800112F0020162F00201B2F0020202F00207C
:107E6800252F00202A2F00202F2F0020D04000206F
:107E7800C844002056555555B81C0020B01E002097
:107E880004310020983200206D4300201464002043
:107E9800304D0020385C0020079BC74A1B781060D3
:107EA800DB077EF516ACC54B1B78002B3EF4D2AC35
:107EB800089BDB78002B7EF4CDAC94F8933001332B
:107EC800DBB2032B84F893307EF6C4ACBC4B5B78F2
:107ED80013B9002D7EF4BEAC1BF004FDFEF7F4BB15
:107EE800B84AB9491068B4F99020C66981FB0601FF
:107EF8008911F617701A00F5FF407F3082423EF76D
:107F0800D6AB891B0A4412B2A4F89020FEF7CFBB67
:107F1800089BDB78002B7FF457AADFEDAC7AAA49DF
:107F280038EE678AC9F5FA63FDEEC87A1BB2CDED63
:107F3800047ABDF91020120381FB0201D217C2EBAB
:107F4800A11203FB02F343F30F334B4407EE903ABD
:107F5800B8EEE78A87ED038AFFF736BA099D002D48
:107F68003EF424ABFFF7A8B9994A059BD588049A33
:107F78001B8BB2F90620591B8A4240F388802B4498
:107F88009A42B4BF00250125FEF721BBC8398A42B1
:107F980042DA99F8CC109A7841FA0BF3D9073FF5F1
:107FA800D9AA524201200C9228F006F87B1E0C9A9E
:107FB800162B00F23781DFE813F0B801CC01A001DD
:107FC800F101E00105028B01760161014C013801E4
:107FD8003501F101270105028B017601EB00D7007D
:107FE800C50046022F021A02AB460899DBF80020AA
:107FF800CB69099D13448B61002D3EF4D7AAFFF786
:108008005BB91AF005FA032140F6B8328BF8201054
:10801800CBF81C20FFF7DFB899F8CC30012202FA20
:108028000BF223EA020308F5FA7289F8CC30CAF891
:108038000820FFF78FBAB4EEE56AF1EE10FA8CBFAC
:10804800B0EE654AB0EE464AC4EE054A9FED612A95
:108058009FED615ADFED611ADFED612A9FED613A0C
:10806800DFED613A9FED614AA4EE825AE4EEE12A1F
:10807800E4EE857AA4EEA23AB0EE675AF0EE637A9F
:10808800E4EE837AA4EEA74AC4EE057A94E40125C7
:10809800FEF79DBA0021564807F06EFF00287FF4CE
:1080A8008AAA322384F89600A4F89830FFF783BA96
:1080B800002A0CBF0120022075E74E4B0122022046
:1080C8004D4C4E4922700B604D4D27F075FFFEF761
:1080D800C2BB02200BF026FEFEF7BDBB03200BF04F
:1080E80021FEFEF7B8BB00200BF01CFEFEF7B3BB69
:1080F80001200BF017FEFEF7AEBB9E2B00F023838A
:108108009D2B00F01983AE2B00F00F83AD2B00F0F0
:108118000583EF2B00F0FF82FD2B00F0F982FB2B8B
:1081280000F0E882FE2B00F01583F72B00F0208387
:108138007B2B7EF490AB4FF4FA6102200BF010FD1C
:10814800FEF789BBD9F8D0002E4B81781144C82995
:10815800A8BFC82121EAE17181709B78002B40F00B
:10816800318324F0F1FBA3E4D9F8D000254B417802
:108178001144C829A8BFC82121EAE17141709B7840
:10818800002BEED013201AF007FAD9F8D000E8E750
:10819800D9F8D0001B4B01781144C829A8BFC821C1
:1081A80021EAE17101709B78002BDAD012201AF0D5
:1081B800F3F9D9F8D000D4E7784B0020014D00201E
:1081C800443100203C660020D34D621000007A4400
:1081D8003846002099FB243F69A2163E39094E3DD6
:1081E800E3B59E3E88FA163E45FE7F3FA7DFA834DA
:1081F800043100201487002048600020D44000206B
:10820800D0400020EA630020C64B0B989B78417948
:1082180011446429A8BF642121EAE1714171002B4E
:1082280040F0CA82D9F8D0009BE7D9F8D000BD4BFE
:10823800017A9B781144C829A8BFC82121EAE171B5
:108248000172002B8DD00B201AF0A6F9D9F8D000B6
:1082580087E7D9F8D000B34BC1799B781144C82976
:10826800A8BFC82121EAE171C171002B3FF479AFA1
:108278000A201AF091F9D9F8D00072E7D9F8D0009D
:10828800A84B81799B781144C829A8BFC82121EA45
:10829800E1718171002B3FF464AF09201AF07CF979
:1082A800D9F8D0005DE7D9F8D0009E4B417993F812
:1082B80002E01144C829A8BFC82121EAE17141712F
:1082C800BEF1000F40F08482112F7FF43EAF48E7E3
:1082D800D9F8D000934B017993F802E01144C829EA
:1082E800A8BFC82121EAE1710171BEF1000F40F079
:1082F8005982102F7FF43BAF33E70B99894B0F79E5
:108308000C931744642FA8BF642727EAE7770F71F7
:108318001AF05CF90C9B9B78002B83D0032039461C
:108328001AF03AF9D9F8D0001BE70B987D4B017881
:108338001144FA29A8BFFA2121EAE17101709B785A
:10834800002B3FF46FAF01201AF026F9D9F8D000BE
:1083580007E70B98734B817811446429A8BF6421FF
:1083680021EAE17181709B78002B3FF45BAF02201A
:108378001AF012F9D9F8D000F3E60B98694BC179D5
:108388009B78114481F30801C171002B3FF44AAF77
:1083980005201AF001F9D9F8D000E2E60B98614BF4
:1083A800817993F802E011446429A8BF642121EA85
:1083B800E1718171BEF1000F40F014820D2F7FF43E
:1083C80024AF2FE7D9F8D000564BC17893F802E0D4
:1083D8001144C829A8BFC82121EAE171C170BEF1C2
:1083E800000F40F0D5810F2F7FF4D5AEB9E6D9F84C
:1083F800D0004C4B90F836109B7811446429A8BFE4
:10840800642121EAE17180F83610002B3FF4A9AE0F
:1084180017201AF0C1F805E7D9F8D000414B90F8B9
:1084280037109B781144FE29A8BFFE2121EAE1718B
:1084380080F83710002B3FF494AE16201AF0ACF8F1
:10844800D9F8D0008DE60B98364B41781144B1F538
:10845800967FA8BF4FF4967121EAE17141709B782D
:10846800002B3FF4DFAE15201AF096F8D9F8D000AB
:1084780077E6129AFFF7F4BB04999B7831F912203A
:10848800B2F5617F4FF4966191FBF3F350DB40F650
:1084980033019142A8BF11460C2FA1F5617191FBE0
:1084A800F3F100F0C780182F7FF402ABC9B2C829D6
:1084B8000B46A8BFC823D9F8D020D77DD8B2B84278
:1084C8003FF4F6AADF1B174BD07548BF0737FF10DC
:1084D8009B780137FFB23BB9002F3FF4E9AA384631
:1084E80027F06AFDFFF7E4BA18201AF055F8F3E709
:1084F8000F2027F07BFCB4F8903084F89250FA3BB8
:10850800A4F89030084DFEF7A6B9B0EE670AFFF759
:1085180096BA07F063FBFFF77DBA044B00220120EF
:10852800CEE500BFEA630020D0400020C6860020C8
:108538000C2F00F09680182F7FF4BAAA00210B4662
:10854800B9E7AC4AAC4D1360FEF785B9AB4A059262
:10855800FFF748B806F48056FFF742B938EE678A45
:10856800A74BA8491870FDEEC87AC9F5FA63CDED96
:10857800047ABDF91020120381FB0201D217C2EB65
:10858800A1121BB203FB02F343F30F334B4407EE74
:10859800903AF8EEE77AC7ED037AFEF76EBB9A4A8F
:1085A800069B1E68136823F004031360089A0123CE
:1085B80006F4805682F82130FFF712B90022BB2B4F
:1085C800149258D0B72B7BD0BE2B76D0BD2B7FF41E
:1085D80094AD13464FF6FE728C49C8898E890344C0
:1085E80032448A81CB8116F029FB06F033FE16F05F
:1085F8000DFBFCF769FB012027F0DEFCB4F8903096
:108608000022FA3BA4F8903084F89220FEF723B9B0
:108618007F4A794D137843F004031370FEF71BB9B2
:108628007C4B022203204BE5FCF7EAFC94F88E30E1
:10863800FFF7DFBACFB2784B0D915B78BB423FF4BE
:1086480037AA764B0C9338460BF06CFB0C9B0D99B4
:108658009B781BB1C9B20C2019F09EFF0137FFB2FD
:108668003AE700273946E6E76D4B634D4FF4C87289
:108678001A80FEF7F0B80223AEE708231A46FEF781
:10868800F0BC07231A46FEF7ECBC06231A46FEF791
:10869800E8BC05231A46FEF7E4BC04231A46FEF795
:1086A800E0BC03231A46FEF7DCBC02231A46FEF799
:1086B800D8BC01231A46FEF7D4BC134602228BE726
:1086C8004FF6FE7388E784F8941084F895004A4DB5
:1086D800FEF762BF002D3EF478A8524C94F88D3016
:1086E800002B3DF49EAF27F065FB002384F88D3006
:1086F800FDF797BF002102200BF032FAB4F8903052
:108708000022963BA4F8903084F89220FEF7A3B894
:1087180000210120F0E700210846EDE7FF210020B5
:1087280014F096FA94F88E30F3E40121002014F046
:108738008FFA94F88E30E9E40021FF2014F088FACB
:1087480094F88E30DFE40021012014F081FA94F8C7
:108758008E30D5E400210320CEE7002BBDD032496E
:10876800324A09684FF47A7000FB03131360B4E7C8
:1087780000210420C0E70B2027F038FB1E4DFEF730
:108788006AB8284C1BF0AEF884F88D50FDF749BF45
:108798000F200D930C9219F0FFFED9F8D0000D9B15
:1087A8000C9A20E610200D930C9219F0F5FED9F8DA
:1087B800D0000D9B0C9A9CE50E2019F0EDFED9F81F
:1087C800D000CEE4142019F0E7FED9F8D000C8E4B0
:1087D80011200D930C9219F0DFFED9F8D0000D9BF3
:1087E8000C9A71E50D200D930C9219F0D5FE0D9B96
:1087F8000C9AE3E5784B0020D04000203C5D002037
:10880800EC1E0020D34D6210CC4000202431002003
:10881800E86300206287002048600020EA630020A7
:1088280072460020481C0020385C0020744B002051
:108838002DE9F047C74C636820469847002800F0A8
:10884800C380C54B1B780122042B84F83C2000F020
:10885800BD80B4F91610B4F91820B4F91A302163A0
:108868006263A363BD4B1B88002B69D0BC4DD4ED5C
:108878000C7AD5ED004A95ED050A95ED015A95ED6E
:10888800067AD5ED035A95ED026AF8EEE76AD5ED5A
:10889800047AA4EEA60AA5EE267A67EEC07AA5EEBB
:1088A800C07AE6EE267A85ED057AC5ED067A2BF0D4
:1088B800E7FBD4ED0D6AD5ED094A95ED0E0A95ED65
:1088C8000A5A95ED0F7AD5ED0D7AD5ED0C5A95ED3E
:1088D8000B6A2063F8EEE66AA4EEA60AA5EE267AED
:1088E80067EEC07AA5EEC07AE6EE267A85ED0E7AB6
:1088F800C5ED0F7A2BF0C4FBD4ED0E6AD5ED124A04
:1089080095ED170A95ED135A95ED187AD5ED167A67
:10891800D5ED155A95ED146A6063F8EEE66AA6EE91
:10892800A40AA6EE857A67EEC07AA0EE657AE6EE2E
:10893800867A85ED177AC5ED187A2BF0A1FBA0632E
:10894800884FA17F884812F0B9F83B88002B40F087
:108958008480864ED6F8E050854B1B685B0743D46D
:10896800B5F90070216B636BA06B824A824E92ED61
:10897800026AD2ED006AD2ED015AC91B2163B5F92A
:108988000270DB1B6363B5F904703568C01B07EE22
:10899800900AB8EEE75A07EE901AB8EEE77A07EEB3
:1089A800903AF8EEE77A36EE056A36EE877A77EE91
:1089B800A57A0135A06382ED026A82ED007AC2EDE4
:1089C800017A3560BDE8F087BDE8F0876B4BB4F9F4
:1089D8001600B4F91810B4F91A20188020635980C9
:1089E80061639A80A2633DE7B6F89820322A00F0C6
:1089F8008880002A66D196F89530002BB0D0604860
:108A0800D6F8FC205F4980FB0273D217C2EB231211
:108A18002A80D6F8002180FB0273D217C2EB2312FA
:108A28006A80D6F80431A78A80FB0302DB17C3EB00
:108A38002213DB1BAB800023CB6086F8953016F041
:108A4800FDF806F007FC16F0E1F8FCF73DF9012007
:108A580027F0B2FAD6F8E05082E7444E226BD6F8F7
:108A6800E050B3F5C87F4FF0000323632B803988AB
:108A780018BFD6F8E400B7F8008008BF0020B1F5A9
:108A8800C87F18BFD6F8E830616B02440B44002059
:108A9800B8F5C87F6063C6F8E420C6F8E830688097
:108AA80052D0D4F838E0D6F8EC10A0637144B8F18D
:108AB800010FA880C6F8EC1068D008F1FF38A7F8B5
:108AC800008049E7D6F8FC00236B00210344C6F870
:108AD800FC3021632980D6F80001636B616303448D
:108AE800C6F800316980A36BD6F80401A16303447A
:108AF800012AC6F80431A98075D0013AA6F8982051
:108B080079E72B8820491F48276BA6F8F030002307
:108B1800B5F802E0B5F804C0C0684B608B60236309
:108B2800C6F8FC702B80616BC6F8001163636B801C
:108B3800A16BC6F80411A363A6F8F2E0A6F8F4C086
:108B4800C6F8F800AB80D8E7A36BC6F8EC30A06392
:108B5800A880B2E7884000207C3E0020D435002061
:108B6800D835002072460020B8400020481C00205C
:108B7800445400208445002080450020803E002089
:108B88001F85EB5124310020441D0020DFF88CC0E4
:108B9800DFF884E0C8328CFB02A9C833D217C2EBD5
:108BA800E9128CFB03A9DB17C3EBE913C8316B800F
:108BB8002A808CFB013CA28ACB17C3EBEC139B1ACF
:108BC800AB80CEF80C0016F039F806F043FB16F02F
:108BD8001DF8FCF779F8404627F0EEF9B7F8008061
:108BE800D6F8E05069E70B2086F89A1086F89420AA
:108BF80027F0FCF8D6F8E050074BB6F8F020B6F8A6
:108C0800F270B6F8F400D6F8F8102A806F80A880C1
:108C1800B6F89820D96070E7243100201F85EB5101
:108C28002DE9F04F2DED0E8BDFF8A8B393B0DBF8EC
:108C38000420049058469047002876D0BBF8A840F6
:108C480000218BF85110002C41F05E84DBF848209D
:108C5800BBF93C70BBF93840DBF82060BBF93A003F
:108C6800DBF82450DFF870A3BB1A83EAE371A1EBA9
:108C7800E371A41BB1F5804FCBF82C40DBF82840FA
:108C88009BF85210DCBFCBF848703A46401B121BC9
:108C9800CBF83000B248CBF8342011F00FFFDAF8E7
:108CA8000020900041F14A85DBED0C5AAD4CDBED1C
:108CB8000B7AAD4994ED406AD4ED416A94ED427A5D
:108CC800D4F80C210968A94B0293B8EEE58ADBEDCC
:108CD8000D5AF8EEE77AF8EEE58A013277EE867AF1
:108CE80038EE268A78EE878A8A42C4ED407A84ED87
:108CF800418AC4ED428AC4F80C2102F01B8293F821
:108D080000E0BEF1140F03F043810023D4F814519E
:108D18000393062D01F29581DFE815F05A15C71463
:108D28000314DA1401091C166314904B8D4C1E7839
:108D38000293072E01F0D88194F82131069353B19C
:108D4800013B84F82131012E01F0AE8413B0BDEC53
:108D58000E8BBDE8F08F864A5279002A01F03882DE
:108D6800844A1278013AD2B2072E84F8212102F0FF
:108D7800A28200230793804BD4F82C21D3F800A0BB
:108D88007E4B0593049B9FED7E6AD4ED4A9A7D49FC
:108D9800C4F82C319A1A07EE902AF8EE677AB7EEE3
:108DA800007AC6EE278A0025774BDFF83092DFF885
:108DB8003082764F03932E46D1ED006A94ED49DA5E
:108DC8009FED739ADFED73AA9FED73CA9FED73AAA7
:108DD800DFED73BA9FED73BA77EE69CA6CEEA6CA77
:108DE800F4EEC7CAF1EE10FA88BFF0EE47CA6E4B30
:108DF80099ED008A2B44D3ED007AF5EE407AF1EE36
:108E080010FA17D0694B2B4493ED007A78EE476A35
:108E1800B0EEE66AF4EEC67AF1EE10FA08D5F5EE91
:108E2800C06AF1EE10FACCBF37EE878A37EE678A50
:108E380083ED008A5E4B1B889A0739D0022E37D003
:108E48009AF82E105B4A07EE901A2A4492ED007A9F
:108E58004A42F8EEE76A07EE902A26EE877AF8EE9D
:108E6800E77AB4EEE77AF1EE10FA0AD407EE901A30
:108E7800F8EE677AF4EEC77AF1EE10FA88BFF0EEF2
:108E8800477A4D4A4D4902EB460231F91600B2F9CC
:108E98000C20821A07EE102AB8EEC77AD807E7EE38
:108EA800497A41F12B81464B93ED008A27EE888A57
:108EB800059B94F860212B4493ED01EA78EE4EDA95
:108EC800002A00F0CF803F4AD4F864310499126830
:108ED800CB1A934240F3C6809AF84820022A02F03F
:108EE8003982022E04F05084374A1268920779D4E6
:108EF800364A87ED00CA12689A42C0F2AD80F7EE92
:108F0800007AF4EEE79AF1EE10FA40F1AB80059999
:108F18002F4BD1ED017A93ED007AF0EEE77AF4EE7B
:108F2800C77AF1EE10FA40F19D80D1ED027AF0EEA9
:108F3800E77AB4EEE77AF1EE10FA40F39380D1EDD8
:108F4800037AF0EEE77AB4EEE77AF1EE10FA40F33E
:108F580089801D4B1B689B077ED51849164A62E01D
:108F6800D4510020501D00209C3200207C3E00205F
:108F78002054002018310020D44000203454002010
:108F88000024744924630020203200202C32002061
:108F9800CDCCCC3DAE47813F000000000000C84268
:108FA80000003443610BB63B186300208C1E002080
:108FB800D0400020981E002024310020804000204E
:108FC800006300202C6300207C40002028630020E0
:108FD80034630020A851002044540020801E002043
:108FE80038320020D44AD549DFF8C0E331F916C039
:108FF8009EED008ADFF8B8E387ED00CA02EB460071
:1090080028EE098AB0F90C00A0EB0C0007EE900AD4
:10901800F8EEE77ADEF8000027EE888A984278EEC4
:109028004EDABFF66CAFB2F90C30B1F900E0C448C3
:10903800AEEB030E00688EEAEE73A3EBEE73834289
:1090480010DAB1F90230B2F90E209A1A82EAE27304
:10905800A3EBE273984205DD0023184684F86031DB
:10906800FCF78AFEB74B2B4493ED000A039B2DEEC9
:10907800000A022E20EE2D0AA3EC010A039304F045
:10908800E582B14BD7ED006A93ED007AAF4BD3ED93
:10909800007AAF4B93ED006AAE4B67EE277A2B440C
:1090A80027EEAC7AD3ED007A67EE277AF0EE665AAF
:1090B800EDEEA75AB1EE467AB4EEE57AF1EE10FA83
:1090C80008DCB4EEE56AF1EE10FA8CBFB0EE657A12
:1090D800B0EE467A94ED4A6AF7EE007AB4EEE76AA3
:1090E800F1EE10FAACBF0123002343B1F0EEE66ABB
:1090F800F0EEC77AF4EEE67AF1EE10FA01D587EDD4
:10910800007A022E04F05E82934A944B52F82600AD
:109118001B68B0EE4E0A9847914A924B52F82600C7
:109128001B6898479AF8373023B18F4B1B88002B60
:1091380001F0E380B0EE4C8A8C4B38EE400A2B44A9
:1091480093ED008A83ED000A9AF8483030EE480A19
:1091580020EE288A002B33D0854B1B7813F00103AF
:1091680000F0C786F7EE007AF4EEE79AF1EE10FA0F
:1091780094F86031C1F25685002B01F06E81D4F865
:109188006431049AD31A7B4A12689A4218DD7A4BE2
:10919800D3ED007AF0EEEDDAF4EEE7DAF1EE10FA5C
:1091A80042F1E180754B1A88002384F86031002A67
:1091B80000F0AB8672494A6912B10A6813604B74B1
:1091C800704B94F870212B4493ED000A2DEE000AA1
:1091D80020EE088A88ED008A32B9039B87ED00CA21
:1091E80003ED01CA88ED00CA0136032E09F104090E
:1091F80008F1040807F1040705F104057FF4F7AD49
:10920800029B1A78072A01F02385012A02F041807F
:109218000023059394F87821002A41F07982DFF839
:1092280094A1594BDAF800201968D50491F82C70EC
:1092380001F18F80DFF88091544AB9F81A3092ED25
:10924800006A534A534ED2ED005AD6ED036A524A89
:1092580084ED626A07EE103A504B92ED005AD3ED56
:10926800007AD3ED013AD3ED024A84ED606AB8EE94
:10927800C77A35EEC64A012236EEC77A84ED5F4AD0
:10928800C4ED635A84F89021C7EE055A0A8D5342FB
:1092980006EE103A424BDFED436A93ED005A424B1B
:1092A80093ED004AB7EE007AF4EEC75A35EE045A49
:1092B800F1EE10FA88BFF0EE475A35EE275AB8EEAD
:1092C800C66AF4EEE65AF1EE10FA07EE902AB4EE0A
:1092D800C65AB8BFF0EE665AF1EE10FAC4ED665AF7
:1092E800B8EE677A01F17C83B4EEC75AF1EE10FA52
:1092F80088BFB0EE475A2A4BDFED306AD3ED017ACA
:10930800294B93ED014A77EE847A25EE265A77EEBB
:10931800A37AB4EEE76AF1EE10FA08DCB4EEE77A65
:10932800F1EE10FA8CBFB0EE676AB0EE476A1C4BDC
:109338004A8DD3ED027A43E024310020804000209A
:1093480030630020D4620020180000201062002042
:1093580048630020E06200201862002014620020A8
:109368006C62002068620020D0400020B81E0020F7
:109378000D3E00202C63002038630020105C002084
:10938800185C0020EC620020D4400020AC2F0020A4
:1093980010310020A43E0020404600202C3200203E
:1093A8002032002000000000383200200063002036
:1093B80028630020445400203C5D00206F12833A4B
:1093C8001FED027A534204EE103A74EEA77AB8EE13
:1093D800C44A26EE076AF4EEC47AF1EE10FA0AD40B
:1093E80007EE102AB8EE474AB4EEE74AF1EE10FA53
:1093F80088BFB0EE674AEC4ADFEDEC7A527824EE8B
:10940800274A0AB9B1EE444A002F41F04386B7EE25
:10941800003AE74D2A78002A02F0CB85E549DFEDCE
:10942800E67AD1ED024AD1ED016A91ED037A66EE52
:10943800244AE5EE264AE4EE074A63EE244AF4EEAF
:10944800E74AF1EE10FAB4BFF0EE673AF0EE643A8C
:1094580098BFF0EE647A012ACDED0A4A02F0FC8545
:1094680091ED067AD1ED052AD1ED076A26EE077A45
:10947800A5EE227AA4EE267A23EE077AB4EEE77AEE
:10948800F1EE10FAB4EEE37A8CBFF0EE676AF0EE14
:10949800476AF1EE10FA88BFF0EE676AB4BFF0EEE3
:1094A800637AF0EE477A022A8DED0B7A00F0DE80BF
:1094B80091ED0A7AD1ED092AD1ED0B3A26EE077A19
:1094C800A5EE227AA4EE237A23EE077AB4EEE67AA2
:1094D800F1EE10FAB4EEE77A8CBFF0EE663AF0EEF1
:1094E800473AF1EE10FA98BFF0EE636AA8BFF0EEC3
:1094F800477A032A8DED0C7A00F0B88091ED0E7A48
:10950800D1ED0D2AD1ED0F3A26EE077AA5EE227A93
:10951800A4EE237A23EE077AB4EEE67AF1EE10FA97
:10952800B4EEE77A8CBFF0EE663AF0EE473AF1EE29
:1095380010FA98BFF0EE636AA8BFF0EE477A042AE3
:109548008DED0D7A00F09280D1ED123AD1ED112A0D
:1095580091ED137A66EE233AE5EE223AE4EE073A05
:1095680063EE233AF4EEE63AF1EE10FAF4EEE73A57
:109578008CBFB0EE667AB0EE637AF1EE10FA98BF5F
:10958800F0EE476AA8BFF0EE637A052ACDED0E3AF1
:109598006CD0D1ED163AD1ED152A91ED177A66EE19
:1095A800233AE5EE223AE4EE073A63EE233AF4EE84
:1095B800E63AF1EE10FAF4EEE73A8CBFB0EE667ACE
:1095C800B0EE637AF1EE10FA98BFF0EE476AA8BFE2
:1095D800F0EE637A062ACDED0F3A47D0D1ED1A3A6C
:1095E800D1ED192A91ED1B7A66EE233AE5EE223A7F
:1095F800E4EE073A63EE233AF4EEE63AF1EE10FAB7
:10960800F4EEE73A8CBFB0EE667AB0EE637AF1EE2C
:1096180010FA98BFF0EE476AA8BFF0EE637A072AFF
:10962800CDED103A22D091ED1E7AD1ED1D2AD1ED63
:109638001F3A26EE077AA5EE227AA3EE847A27EE61
:10964800037AB4EEE67AF1EE10FAB4EEE77A8CBF5C
:10965800B0EE666AB0EE476AF1EE10FA8DED117A57
:1096680098BFF0EE466AA8BFF0EE477A77EEE67A42
:10967800F7EE006AF4EEE67AF1EE10FAC4ED4A7AF3
:1096880043F3898586EEA77A022ADDED0B7A67EE29
:10969800244A67EE877ACDED0A4ACDED0B7A2DD0B4
:1096A800DDED0C7A67EE877A032ACDED0C7A25D0AA
:1096B800DDED0D7A67EE877A042ACDED0D7A1DD09F
:1096C800DDED0E7A67EE877A052ACDED0E7A15D094
:1096D800DDED0F7A67EE877A062ACDED0F7A0DD089
:1096E800DDED107A67EE877A072ACDED107A05D07E
:1096F800DDED117A27EE877A8DED117A2F49096809
:1097080011F0805801F04182F6EE005AC4ED665A15
:10971800002A02F071842A4B94ED636A29492A4F82
:109728001E78DFF8B0E094F9903194ED625AB7F9F9
:109738000670C878DAF80010DEED004A0397BDEE2F
:10974800C66A07EE103AB9F81A70204B079716EE5A
:1097580010EABDEEC56A06F0010C01F4805701F06D
:10976800100601F4800108911B78D4ED5F6AD4EDEE
:10977800607AB8EEC77A16EE101A002841F00E800B
:10978800002E41F063830B4E9DED0A5A96ED006A58
:109798000F4825EE866AA5EE076AB0EE675AA6EE70
:1097A800265ABDEEC56A17E08C3200206F12833A44
:1097B8002A3E0020B04500200000000004310020AF
:1097C8000D3E0020304D0020146400206856002013
:1097D80054320020AC45002016EE108A16EE107A9E
:1097E800F045A8BF77464145C8BF0F4606EE107A38
:1097F800B8EEC66A012A80ED006A00F0DC8096EDBA
:10980800046A9DED0B5A25EE866AA5EE076AB0EE4E
:10981800675AA6EE265ABDEEC56A16EE108A16EEEF
:10982800107AF045A8BF77464145C8BF0F4606EEF7
:10983800107AB8EEC66A022A80ED016A00F0BB8091
:1098480096ED086A9DED0C5A25EE866AA5EE076A24
:10985800B0EE675AA6EE265ABDEEC56A16EE108A15
:1098680016EE107AF045A8BF77464145C8BF0F46A7
:1098780006EE107AB8EEC66A032A80ED026A00F096
:109888009A8096ED0C6A9DED0D5A25EE866AA5EE36
:10989800076AB0EE675AA6EE265ABDEEC56A16EEFE
:1098A800108A16EE107AF045A8BF77464145C8BF22
:1098B8000F4606EE107AB8EEC66A042A80ED036AEF
:1098C80079D096ED106A9DED0E5A25EE866AA5EEC2
:1098D800076AB0EE675AA6EE265ABDEEC56A16EEBE
:1098E800108A16EE107AF045A8BF77464145C8BFE2
:1098F8000F4606EE107AB8EEC66A052A80ED046AAD
:1099080059D096ED146A9DED0F5A25EE866AA5EE9C
:10991800076AB0EE675AA6EE265ABDEEC56A16EE7D
:10992800108A16EE107AF045A8BF77464145C8BFA1
:109938000F4606EE107AB8EEC66A062A80ED056A6A
:1099480039D096ED186A9DED105A25EE866AA5EE77
:10995800076AB0EE675AA6EE265ABDEEC56A16EE3D
:10996800108A16EE107AF045A8BF77464145C8BF61
:109978000F4606EE107AB8EEC66A072A80ED066A28
:1099880019D096ED1C6A9DED115A65EE865AE7EEE0
:10999800055AE6EEA57AFDEEE77A17EE906AB64527
:1099A800A8BFB646B142D8BF714607EE901AF8EE86
:1099B800E77AC0ED077ABCF1000F00F0FC87D24AC5
:1099C8001268002A41F00480D04A127892B12878AF
:1099D80068B1CF4FDFF85C830026F0B2D8F80030CA
:1099E800B7EC010A9847287801368642F5DBC94A60
:1099F80012689047029B1A78072A01F018810025FF
:109A0800DAF80020530500F1EF87C34B1B78BBB190
:109A1800C24AB9F81A30B2F906209A4210DCC04B93
:109A28001B78012B01F05C84192B01F059840E2B53
:109A380006D0082B04D0BB4E0023B360C4F83831DD
:109A480094F8A26126B1B84B1B889F0741F00B849C
:109A580094F8A821002A40F0D28799F81E70002FA8
:109A680000F01886022F01F04683032F41F04A8345
:109A780099F82030C3EB431103EB8101C90089B287
:109A880099F81F300233DBB2002A00F05B86002908
:109A980000F05886A5480768B1FBF7F10FB2A4F8A3
:109AA800D871002B03F0AE8007EE907AF8EEE77AD3
:109AB800F7EE006A86EEA77A9A4E012BD4ED7B6A00
:109AC800D6ED007A77EEE67A67EE877AC4ED777A94
:109AD80021D0D6ED017AD4ED7C6A77EEE67A022BB6
:109AE80067EE877AC4ED787A15D0D6ED027AD4ED90
:109AF8007D6A77EEE67A032B67EE877AC4ED797A8A
:109B080009D0D6ED037AD4ED7E6A77EEE67A67EE71
:109B1800877AC4ED7A7A02990978092903F0B28123
:109B2800002F40F3BD859BB394ED7B7AD4ED777A13
:109B380077EE877A012BC4ED7B7AC6ED007A21D0C7
:109B480094ED7C7AD4ED787A77EE877A022BC4ED9F
:109B58007C7AC6ED017A15D094ED7D7AD4ED797AC8
:109B680077EE877A032BC4ED7D7AC6ED027A09D0A9
:109B7800D4ED7E7A94ED7A7A77EE877AC4ED7E7AA0
:109B8800C6ED037A013B022BB8BF0223DBB2069372
:109B9800069B002A18BF02239E46654BDFED6A6AC2
:109BA8001A68029B91781878137807EE903AF8EEC5
:109BB800E77AB0EE007A67EEA67AF4EEC77AF1EEAD
:109BC80010FA40F30987DFED5D6A37EEC77AB0EE29
:109BD800676AA7EE266AF0EE466A96ED007A9FED70
:109BE800586A27EE066AF0EEC65A84ED526AC4ED4A
:109BF800555A99B107EE101AB8EEC75A9FED527A26
:109C080066EE064A25EE075AB7EE007A37EE457A31
:109C180064EEA54AA4EE857A26EE076A9FED497A96
:109C2800537926EE877A27EE067ACBB1DFED466ABE
:109C38009FED466A65EEA65A06EE903AF8EEE66A99
:109C480066EEA56AF4EEC66AF1EE10FA01F3188220
:109C5800F7EE005A75EEE66A85EEA66A27EE067AF2
:109C68000C289FED3B8ADFED3B6A00F0B587B4EE28
:109C7800C87AF1EE10FA98BFB0EE478AB4EEE68AD9
:109C8800F1EE10FAB8BFB0EE668A84ED4C8ABEF1E8
:109C9800000F00F00881B0EE007AF4EEC77AF1EE1A
:109CA80010FA05DD37EEC77ADFED246AE7EE267A8B
:109CB80096ED017ADFED226A27EE267AF0EEC75A92
:109CC80084ED537AC4ED565A99B106EE901A9FED79
:109CD8001E6AF8EEE66A27EE075A66EE866AB7EE5F
:109CE800006A36EE666A25EE255AA5EE266A27EE44
:109CF800067ADFED146A937967EEA67A67EE877ABB
:109D0800002B3FD028E000BF0C62002090590020B3
:109D18005432002064560020CC0200201464002035
:109D28008C320020A43E0020D04000207432002055
:109D3800D84000205C5600200000C842D7A36841E4
:109D48006F12033B000048430AD7233CA4707D3FB1
:109D580000C0F94400C0F9C407EE103AB8EEC77A5B
:109D68001FED076A5FED076A27EE257A27EE067A68
:109D7800B4EEE67AF1EE10FA41F374815FED126AFF
:109D880067EEA67A0C2800F007875FED0F6A1FEDD3
:109D98000F7AF4EEE67AF1EE10FA88BFF0EE667A02
:109DA800F4EEC77AF1EE10FAB8BFF0EE477ABEF1DA
:109DB800010FC4ED4D7A76DD53785FED1D6A07EE2D
:109DC800903AF8EEE77AB0EE007A67EEA67A537A20
:109DD800F4EEC77AF1EE10FA05DD37EEC77A5FEDDB
:109DE800296AE7EE267A96ED027A5FED2B6A27EE6E
:109DF800267AF0EEC75A84ED547AC4ED575A9BB1CF
:109E080006EE903A1FED306AF8EEE66A27EE075A3A
:109E180066EE866AB7EE006A36EE666A25EE255A61
:109E2800A5EE266A27EE067A5FED3A6AD37967EEE1
:109E3800A67A67EE877AFBB107EE103AB8EEC77AD2
:109E48001FED3F6A5FED3F6A27EE257A27EE067A17
:109E5800B4EEE67AF1EE10FA01F30081B5EEC07ABD
:109E6800F1EE10FA02F1BB82B7EE006A36EE477ADD
:109E7800C6EE076A67EEA67A0C2800F0CB865FED7F
:109E88004C6A1FED4C7AF4EEE67AF1EE10FA88BFD0
:109E9800F0EE667AF4EEC77AF1EE10FAB8BFF0EE9B
:109EA800477AC4ED4E7A092800F0628699F8216055
:109EB800002E40F01786002384F8A83116F0CCFB5A
:109EC800002840F0FE83C44B1B7823B9C34B9B7812
:109ED800002B41F0C381029B1E78072E7EF433AF1E
:109EE800FBF7ECFDBE4B029A401B1678D880FEF7B4
:109EF8002ABF94F86021002A3FF462A9B94A84F87D
:109F080060311288002A7FF455A9B74AB74B1178F7
:109F1800186881F0010104F043FFFFF751B9B44A12
:109F28001178D4F81871B34B9FEDB37AFE009A19E3
:109F380082ED007A002979D0B048B0EE476AF0EE99
:109F4800476A0022F0EC017A013267EEA77A05EE43
:109F5800902AB4EEE77AF1EE10FAF8EEE55AB8BFB7
:109F6800B0EE677A8A4276EEA76AA7EEA56AE9D1CB
:109F7800F5EEC06A9A19F1EE10FA82ED007A55DD15
:109F8800C6EE265A9E4A9F490988F7EE007A75EE72
:109F9800E75AD2ED007A65EEA77AFDEEE77A17EE7A
:109FA800902A812A42F392818A42A8BF0A4607EE84
:109FB800902AF8EEE77A944AF01902EB800292EDC3
:109FC800057AD2ED003A92ED066A92ED014AD2ED99
:109FD800046AD2ED034A92ED025AA3EEA77AA4EEE0
:109FE800276A66EEC76AA7EE646ABDEEC77AE5EE31
:109FF800276A17EE100A812882ED056AC2ED066A03
:10A0080042F361818142A8BF014607EE901AF8EE3B
:10A01800E77AFCEEE77ACDED057ABDF814209919B8
:10A028008A801FB9BEF1130F03F0A380BEF1150F8C
:10A0380041F0C9821E446A4BB28823F81720D4F82D
:10A048001451724A013582FB05325119EA17C2EBE5
:10A05800A102C2EBC202AD1AC4F814516C48D4F87C
:10A068001C21049B6B4D01682D78C4F81C319A1A89
:10A0780011440160002D40F0DD8007EE902A664E05
:10A08800DFF8AC91654FB8EEE78A06F5F07506F58E
:10A098001378F6EC017A9BED070ADBF80832F8EE44
:10A0A800E77A284627EE800A9847A5F1E000DBF812
:10A0B80028319847A5F17000DBF898319847D6F811
:10A0C800EC00DBF8AC309847D7ED007AA9EC010A30
:10A0D800E0EE087A2435A845E7EC017AD9D1029B4D
:10A0E8001E78072E7EF428AEFBF7E8FC029A3C4B5C
:10A0F8001678049A801A1880FEF71EBE94ED557AD9
:10A10800B1F90000D4ED566AB1F902E0444AF4EE20
:10A11800C76A80EAE0738EEAEE71A3EBE073F1EEB2
:10A1280010FAA1EBEE71B8BFF0EE476A8B42B8BFE8
:10A138000B4607EE103A1378B8EEC77A27EE097A7D
:10A14800002B00F06181374B93ED005AB5EEC05AF1
:10A15800F1EE10FA40F31585334BD3ED004AF5EED6
:10A16800C04AF1EE10FA40F30C8534EEC77A66EE79
:10A17800CA5A87EE246AC5EE856AB7EE007AB4EE4D
:10A18800C76AF1EE10FA88BFB0EE476AB5EEC06A4A
:10A19800F1EE10FA76EE876AB8BFB0EE4C6A66EE5A
:10A1A800266AF4EEC76AF1EE10FA88BFF0EE476A45
:10A1B800F5EEC06AF1EE10FAB8BFF0EE4C6A1B4B30
:10A1C80093ED007A67EE877AA7EEA68AFEF770BE4F
:10A1D8000122FEF7C9BD00BF58380020EA630020FD
:10A1E800803E0020105C0020125C0020145C0020DF
:10A1F800A23200209835002000000000501D0020E9
:10A20800A4320020A0320020C034002093244992B8
:10A218007045002099320020D45100207445002058
:10A228000C630020086300201063002004630020F2
:10A238003854002007EE902A9D4B9E4D9E49DFF82A
:10A24800C0820594F8EEE78A039305F5B876994637
:10A2580000270C46029BDBED077A1B78172B6CD086
:10A2680095ED007AB8EEC78A082B28EE278A07D121
:10A27800B0EE480A069329F003FF069BA9F80000F0
:10A28800DAF8002091000BD5002F03F04082B0EEE1
:10A29800480ADBF8083206F170009847B0EE408AA9
:10A2A800B0EE480ADBF82831A6F170009847DBF8D1
:10A2B800983130469847029B1B78032BB0EE408AB2
:10A2C80036D0D5F8F000DBF8AC30B0EE480A984745
:10A2D800D8ED007AA4EC010AE0EE287A0137032FC2
:10A2E80006F1240609F1020905F10405E8EC017AF2
:10A2F800B0D1029B059C1E78F3E6704B704A2B4444
:10A3080093ED007AD2ED007A6E4B67EE277AF7EE7E
:10A31800006AF4EEE67AF1EE10FA93ED007A88BF5F
:10A32800F0EE667A67EE877A27EE888AFEF704BF32
:10A3380029F0A6FEA9F80000C3E795ED007A0BEB1B
:10A348004702B8EEC78A128FA9F8002028EE278A9C
:10A3580096E75D4BDFF8AC911A785C4ED0075CBF8E
:10A36800B9F81820A4F88421594AD6ED037A12883E
:10A3780007EE102AB8EEC77AF4EEC77AF1EE10FAB3
:10A3880041F2C3855348038807EE103AB8EEC77AFE
:10A39800F4EEC77AF1EE10FAC0F2AE874E4A4F4893
:10A3A80092ED006AD0ED006A94F99021C4ED626ADA
:10A3B80076EE665A012AC4ED606AC4ED5F5A84EDF0
:10A3C800636A01F07B84049BC4F89431002037EE63
:10A3D800C77AFCEEE77A424D84ED667A17EE902A4A
:10A3E800A4F88421012295ED005A84F890213D4A71
:10A3F800904241F2BA853C4BD3ED007AD3ED013A55
:10A40800D3ED024AFEF740BF384B93ED006AB4EE35
:10A41800EA6AF1EE10FA40F11C87F7EE005A75EE81
:10A42800C65A3BEEC77A65EE8B5A314BA7EE256AC2
:10A4380093ED007A26EE076AB5EEC06AF1EE10FADF
:10A4480040F29F83CAEE065AB7EE007AB0EE476A2A
:10A45800A6EEE56AF0EE466AA3E6264AD2ED007A51
:10A46800B0EEC87AB4EEE77AF1EE10FA7EF7A8AE4D
:10A47800214AD2ED007AB0EEED7AB4EEE77AF1EE49
:10A4880010FA7EF79DAE1D4AD9ED007A92ED007A5A
:10A49800F0EEE77AF4EEC77AF1EE10FA7EF590AEB8
:10A4A80001220499C4F8641184F86021FEF76BBE98
:10A4B800803E0020D451002038540020A41E0020E3
:10A4C800FC620020F86200200D3E0020A43E00201F
:10A4D8004446002046460020103100203046002027
:10A4E8004C4600208FD003002C320020146300203B
:10A4F800086300203C63002038630020406300208C
:10A50800744500203C5D0020944B954D95481A6891
:10A5180003954778B5F9060005934FF47A75B5FBAE
:10A52800F2F2C2EB421502EB8502D5008E4B029384
:10A53800ADB2AC421E7801F0CD86DBF87C30BBF9B9
:10A548003810DBF8602003F1010E07EE901A0A4478
:10A55800BEF1010FCBF87CE0CBF86020F8EEE77A8B
:10A5680001F0C586DBED1B5ADBED1D6A07EE10EA2C
:10A5780037EEE56AB8EEC75A012C86EE057A37EE53
:10A58800257A77EEC77A8BED1C7AE7EE866A8BED33
:10A598001B7AF0EE667ACBED1E6ACBED1D6A02F0EF
:10A5A8007D81DBF89030BBF93A10DBF8642003F1C9
:10A5B800010E07EE901A0A44BEF1010FCBF890E0A5
:10A5C800CBF86420F8EEE77A01F0AC86DBED205A90
:10A5D800DBED226A07EE10EA37EEE56AB8EEC75AF5
:10A5E800012C86EE057A37EE257A77EEC77A8BED61
:10A5F800217AE7EE866A8BED207AF0EE667ACBED6B
:10A60800236ACBED226A02F07181DBF8A430BBF932
:10A618003C10DBF8682003F1010E07EE901A0A449B
:10A62800BEF1010FCBF8A4E0CBF86820F8EEE77A8A
:10A6380001F09386DBED255ADBED276A07EE10EA79
:10A6480037EEE56AB8EEC75A012C86EE057A37EE82
:10A65800257A77EEC77A8BED267AE6EE276A8BEDB8
:10A66800257AF0EE667ACBED286ACBED276A02F000
:10A678006581039B3D4CD880BBF8A820029B013A1A
:10A688001E78ABF8A820059900224A608A60CA6043
:10A69800FEF74FBBA4F8D871002A3FF40FAC344E34
:10A6A8004FF0020EFFF779BA324B334A1968128815
:10A6B8002B4BC96919805A8013B0BDEC0E8BBDE8CD
:10A6C800F08F2E4C15F084FE6378022B00F0F8858D
:10A6D800032B7FF4F8AB41F2B813E35C002B41F095
:10A6E800E88241F2A403E35C002B41F0DD8241F2F1
:10A6F800E803E35C002B41F0D28241F22C13E35CC7
:10A70800002B3FF4E0AB1E4825F072FFFFF7DBBBE0
:10A718001C4B1D4D1A7812F0010F2A7840F0AC82BC
:10A72800002A00F0B184920018491948DFF864A0A3
:10A73800DFF8649029F0D0FAFFF741B90A4B029389
:10A748000A4C8BE4B4F8D871013F3FB2002FA4F84B
:10A75800D871A1DD064EFFF7E6B900BF34540020DA
:10A76800803E0020205400207C3E0020501D002008
:10A77800A43E00203C6600202E2B002054670020B9
:10A78800807800200D3E00202A3E0020342B002037
:10A7980054320020445400203C5D0020002E01F07B
:10A7A8003981BCF1000F42F03B82C34E002B42F0CE
:10A7B800DB8096ED006A9DED0A5AC04825EE866A50
:10A7C800FDEEE44AA5EE076AB0EE675AA6EE265AF1
:10A7D80014EE901ABDEEC56A16EE10CA16EE107A7F
:10A7E800F445A8BF77466145C8BF0F4606EE107A04
:10A7F800B8EEC66A012A80ED006A00F0DF8096EDA7
:10A80800046A9DED0B5A25EE866AA5EE076AB0EE3E
:10A81800675AA6EE265ABDEEC56A16EE10CA16EE9F
:10A82800107AF445A8BF77468C45B8BF0F4606EEA8
:10A83800107AB8EEC66A022A80ED016A00F0BE807E
:10A8480096ED086A9DED0C5A25EE866AA5EE076A14
:10A85800B0EE675AA6EE265ABDEEC56A16EE10CAC5
:10A8680016EE107AF445A8BF77468C45B8BF0F4658
:10A8780006EE107AB8EEC66A032A80ED026A00F086
:10A888009D8096ED0C6A9DED0D5A25EE866AA5EE23
:10A89800076AB0EE675AA6EE265ABDEEC56A16EEEE
:10A8A80010CA16EE107AF445A8BF77468C45B8BF93
:10A8B8000F4606EE107AB8EEC66A042A80ED036ADF
:10A8C8007CD096ED106A9DED0E5A25EE866AA5EEAF
:10A8D800076AB0EE675AA6EE265ABDEEC56A16EEAE
:10A8E80010CA16EE107AF445A8BF77468C45B8BF53
:10A8F8000F4606EE107AB8EEC66A052A80ED046A9D
:10A908005CD096ED146A9DED0F5A25EE866AA5EE89
:10A91800076AB0EE675AA6EE265ABDEEC56A16EE6D
:10A9280010CA16EE107AF445A8BF77468C45B8BF12
:10A938000F4606EE107AB8EEC66A062A80ED056A5A
:10A948003CD096ED186A9DED105A25EE866AA5EE64
:10A95800076AB0EE675AA6EE265ABDEEC56A16EE2D
:10A9680010CA16EE107AF445A8BF77468C45B8BFD2
:10A978000F4606EE107AB8EEC66A072A80ED066A18
:10A988001CD096ED1C6A9DED115A65EE865AE7EECD
:10A99800055AE6EEA57AFDEEE77A17EE906AB64517
:10A9A800A8BFB646B142D8BF714607EE901AF8EE76
:10A9B800E77AC0ED077A002A3FF401A892004049DF
:10A9C8003E4829F089F93F4A1268002A3EF4FCAF54
:10A9D80021F00AF8FEF7F8BFF0EE676AFFF7FDB856
:10A9E800B0EE465AFEF787BCDBF80830002B3FF480
:10A9F8000CA83549A1F14C009847FFF706B8334930
:10AA0800334BD1F8EC101B6844F620608142A8BF94
:10AA18000146B1F57A7FB8BF4FF47A7189B213F065
:10AA2800100FA4F8AA11DAF8003000F06084DB04F3
:10AA380041F1B185274BD3F800E0BEF832707F08AA
:10AA4800254E2648D4F8AC31D6ED037AA0FB010197
:10AA58008809642191FBF0F11429BDEEE77A04EB33
:10AA68004306A8BF142101339942C4F8AC3117EE4C
:10AA780010CADCBF0023C4F8AC3104EB4303A6F8CA
:10AA8800B0C1B3F9B03107EE103AB8EEC77A77EE35
:10AA9800C77AFDEEE77ACDED037ABDF90C1081EAAD
:10AAA800E173A3EBE173BB4201F3DC860C494FF081
:10AAB8007E530B60FEF7D1BFB04500205432002012
:10AAC800342B00200C620020F4510020EC020020FE
:10AAD80004310020D4400020A43E0020D34D621051
:10AAE800180000201E21CD4805F046FA00283FF442
:10AAF800E2A9CB4B1B885A063FF5DDA994F8FC3137
:10AB0800B34242F0E181C74B94ED800AD3ED018A4C
:10AB1800D4ED4E5A9FEDC46ADFEDC46A20EE657A23
:10AB280068EE007AA8EE287AE5EEA87AB4EEC67A3E
:10AB3800F1EE10FA88BFB0EE467AB4EEE67AF1EE9E
:10AB480010FAF4EEC67AB8BFB0EE667AF1EE10FAF3
:10AB580088BFF0EE467AF4EEE67AF1EE10FAB8BF66
:10AB6800F0EE667A84ED4C7AC4ED4E7AFFF7A3B91D
:10AB7800FDEEC87AAE4A17EE903A9780D380FFF779
:10AB880095B9DFEDAC6AFFF71ABBDAF80010490295
:10AB98003EF5BAADFEF7BCBD9FEDA37ADFEDA36A23
:10ABA800A349F4EEC77AF1EE10FA98BFB0EE677ACF
:10ABB800FDEEE77AB4EEE67AF1EE10FA17EE903A87
:10ABC800B8BFB0EE667ABEF1010F84ED4D7A4B80C6
:10ABD8003FF7F2A8FFF76AB9B4EEC87AF1EE10FAB7
:10ABE80098BFB0EE478ABDEEC77AB4EEE68ADFF8C2
:10ABF80040C2F1EE10FA17EE103AB8BFB0EE668A0E
:10AC080084ED4C8AACF80030BEF1000F7FF443A805
:10AC1800FFF74CB9BDEEE77A854B17EE102A9A80FC
:10AC2800FFF72DB9002B3EF4CBAAFEF7A8BAFAF726
:10AC380045FF029B7E491A78059B072AA0EB030073
:10AC480088807EF4DCAEFAF739FF0546FEF7D8BEF9
:10AC5800FAF734FF029A07991278754B0393401A52
:10AC6800012A588000F01783072A7EF4D1AAFAF740
:10AC780025FF0590FEF7CEBA002A00F00582D4ED34
:10AC8800563A94ED556AD4ED607A6B4994ED5F7A43
:10AC9800D1ED005A94ED534AD4ED524A674E6848B4
:10ACA800F4EEC63AF3EE046AF1EE10FA37EEA65A5D
:10ACB80000F1848396ED026A26EE446AF0EE674A54
:10ACC800E6EE074AF4EEC54A34EEE66AF1EE10FA0B
:10ACD80048BFB0EE656A012A80ED006A00F0D481B1
:10ACE80096ED066A26EE446AF0EE674AE6EE074AF3
:10ACF800F4EEC54A34EEE66AF1EE10FA48BFB0EE5B
:10AD0800656A022A80ED016A00F0BE8196ED0A6A42
:10AD180026EE446AF0EE674AE6EE074AF4EEC54AC4
:10AD280034EEE66AF1EE10FA48BFB0EE656A032A1F
:10AD380080ED026A00F0A88196ED0E6A26EE446A5C
:10AD4800F0EE674AE6EE074AF4EEC54A34EEE66AE4
:10AD5800F1EE10FA48BFB0EE656A042A80ED036A86
:10AD680000F0928196ED126A26EE446AF0EE674A88
:10AD7800E6EE074AF4EEC54A34EEE66AF1EE10FA5A
:10AD880048BFB0EE656A052A80ED046A00F07C8150
:10AD980096ED166A26EE446AF0EE674AE6EE074A32
:10ADA800F4EEC54A74EEE66AF1EE10FA48BFF0EE2A
:10ADB800656A062AC0ED056A00F06681D6ED1A6A52
:10ADC80066EEC46AF0EE674AE6EE874AB3EE046AB6
:10ADD800F4EEC54A74EEC66AF1EE10FA48BFF0EE1A
:10ADE800656A072AC0ED066A00F04E81D6ED1E6A34
:10ADF800DFF850A0DFF8509026EEC44AE4EE077A58
:10AE0800F4EEC57A77EEC67AF1EE10FA48BFF0EEA6
:10AE1800657AC0ED077AFEF7D2BD00BF0431002085
:10AE2800D04000201800002000C0F94400C0F9C438
:10AE3800803E002000000000AC450020B045002006
:10AE480054320020445400203C5D0020AF4E9DED5C
:10AE58000A5A96ED006ABCF1000F41F0318125EEE7
:10AE6800866AAB48A5EE076AB0EE675AA6EE265A80
:10AE7800BDEEC56A16EE10CA16EE107AF445A8BFE4
:10AE880077466145C8BF0F4606EE107AB8EEC66A27
:10AE9800012A80ED006A3FF491AD96ED046A9DEDBC
:10AEA8000B5A25EE866AA5EE076AB0EE675AA6EE3B
:10AEB800265ABDEEC56A16EE10CA16EE107AF4458B
:10AEC800A8BF77466145C8BF0F4606EE107AB8EEB0
:10AED800C66A022A80ED016A3FF470AD96ED086AF1
:10AEE8009DED0C5A25EE866AA5EE076AB0EE675A04
:10AEF800A6EE265ABDEEC56A16EE10CA16EE107AF0
:10AF0800F445A8BF77466145C8BF0F4606EE107ADC
:10AF1800B8EEC66A032A80ED026A3FF44FAD96ED9B
:10AF28000C6A9DED0D5A25EE866AA5EE076AB0EE0D
:10AF3800675AA6EE265ABDEEC56A16EE10CA16EE78
:10AF4800107AF445A8BF77466145C8BF0F4606EE9C
:10AF5800107AB8EEC66A042A80ED036A3FF42EAD73
:10AF680096ED106A9DED0E5A25EE866AA5EE076AE3
:10AF7800B0EE675AA6EE265ABDEEC56A16EE10CA9E
:10AF880016EE107AF445A8BF77466145C8BF0F464C
:10AF980006EE107AB8EEC66A052A80ED046A3FF418
:10AFA8000DAD96ED146A9DED0F5A25EE866AA5EE55
:10AFB800076AB0EE675AA6EE265ABDEEC56A16EEC7
:10AFC80010CA16EE107AF445A8BF77466145C8BF87
:10AFD8000F4606EE107AB8EEC66A062A80ED056AB4
:10AFE8003FF4ECAC96ED186A9DED105A25EE866A92
:10AFF800A5EE076AB0EE675AA6EE265ABDEEC56AF8
:10B0080016EE10CA16EE107AF445A8BF77466145C9
:10B01800C8BF0F4606EE107AB8EEC66A072A80ED5A
:10B02800066A3FF4CBAC96ED1C6A9DED115A65EEAD
:10B03800865AE7EE055AE6EEA57AFDEEE77A17EEB0
:10B04800906AB645A8BFB646B142C8BF8E4607EE5D
:10B0580090EAF8EEE77AC0ED077AACE4DFED2D6A06
:10B06800FEF708BFB5EEC07AF1EE10FA01F1B38130
:10B07800B7EE006A36EE477AC6EE076AFEF780BE7C
:10B088009FED246AFEF7EABDDFF8A0A0DFF8A090E4
:10B09800FEF795BC20494A79002A3EF4B8A91F4A10
:10B0A8001278002A3EF4B3A90B781D49DFED1D4A3A
:10B0B80007EE903A0B88B8EE677A07EE902A06EE0C
:10B0C800903AF8EEE77AF8EE666A67EE277AB7EE16
:10B0D800007A87EEA63AB4EEE43AF1EE10FA88BFA9
:10B0E800B0EE643AB4EEC73AF1EE10FAB8BFB0EE7B
:10B0F800473AFEF78EB9B4F8AA1101F57A7189B208
:10B10800FEF7BEBC084B5988FEF7BABCB045002014
:10B11800543200200000C84260400020A23E0020B7
:10B128008C3E0020713DAA3FE0420020445400209C
:10B138003C5D00209349039107EE102A08461978D0
:10B14800B0F904009BED070AB4F81061B8EEC77AAD
:10B15800F7EE006A0022132986EE879AC4F80C21BC
:10B1680001F04E81884A894901EB86070025C4F819
:10B178000051C4F8045167EE897A92ED001AD2EDB5
:10B18800053A92ED122A92ED173AD2ED091AD2ED4C
:10B198000E4A92ED016A92ED064A92ED0A7AD2EDD4
:10B1A8000F5AD2ED132AD2ED186A92ED045AD2ED55
:10B1B800030A69EE288A29EE088AE1EE273AA2EE08
:10B1C800283AE1EE884AA6EE274AE7EE085A92EDB9
:10B1D800167A92ED0D6A92ED021AD2ED0C1AC7EDAD
:10B1E800003AE2EEA86A25EE635A27EE437A92ED1A
:10B1F8000B2AD2ED152AC7ED204AA0EEE34A26EE27
:10B20800646AD2ED143A82ED054AA1EE275AF0EEAF
:10B21800477AE1EEE45AA2EE086AE2EEC36AE3EE88
:10B22800A87A82ED065AC2ED0E5A82ED0F6A87EDB2
:10B23800403AC2ED176AC2ED187AC4F80851039B68
:10B24800721C02F01F029880A4F81021029BFDF7DF
:10B2580056BD4F4B93ED006AFFF7EEB804980DF01A
:10B26800EFFAFEF738BE4B4B9FED4B7AD3ED087AD9
:10B27800F4EEC77AF1EE10FA00F2B5849FED477A42
:10B28800474ED6ED037A77EE877AC6ED037AFEF756
:10B29800DFBB3C4B0393FAF711FC4249D4F8742105
:10B2A80009680590821AC4F874010398511A8280BB
:10B2B800C180FDF7AFBFFAF701FC0790FDF75BBD52
:10B2C800A3784FF0010A072B3EF6FDADDFE813F037
:10B2D8001305FA050705FC04970580058A052B0563
:10B2E800314B9B7B002B3EF4A6ABFEF7A9BBD800E5
:10B2F8003FF59DABFEF7B1BBB4F88401904240F234
:10B30800BD8494F89C01002840F07C86274A284D8B
:10B3180092ED007AD5ED007A94F99021C4ED627A25
:10B3280077EE676A012AC4ED607AC4ED5F6A84ED3E
:10B33800637A01F03887049BC4F894311D4A9FED65
:10B34800177A92ED005A84ED667A012284F89021EA
:10B35800FFF74DB80120FAF70FFDD4F86431049ACD
:10B36800D31AFDF7BEBD144BD9ED007A93ED007AE0
:10B37800F0EEE77AF4EEC77AF1EE10FA7DF720AF37
:10B38800FDF710BF803E00202C350020C032002081
:10B3980008630020484500208FC2753C000000006B
:10B3A800A43E002074320020C05D0020103100202F
:10B3B800304600204C4600204063002096ED016A8C
:10B3C80026EE646AB0EE674AA6EE074AB4EEC54AAE
:10B3D80034EE666AF1EE10FA48BFB0EE656A012AEB
:10B3E80080ED006A3FF450AE96ED056A26EE646A79
:10B3F800B0EE674AA6EE074AB4EEC54A34EE666A6E
:10B40800F1EE10FA48BFB0EE656A022A80ED016AD3
:10B418003FF43AAE96ED096A26EE646AB0EE674AE2
:10B42800A6EE074AB4EEC54A34EE666AF1EE10FAA3
:10B4380048BFB0EE656A032A80ED026A3FF424AE85
:10B4480096ED0D6A26EE646AB0EE674AA6EE074AE4
:10B45800B4EEC54A34EE666AF1EE10FA48BFB0EEB3
:10B46800656A042A80ED036A3FF40EAE96ED116A10
:10B4780026EE646AB0EE674AA6EE074AB4EEC54AFD
:10B4880034EE666AF1EE10FA48BFB0EE656A052A36
:10B4980080ED046A3FF4F8AD96ED156A26EE646A0D
:10B4A800B0EE674AA6EE074AB4EEC54A74EE666A7D
:10B4B800F1EE10FA48BFF0EE656A062AC0ED056A9B
:10B4C8003FF4E2ADD6ED196A66EEE46AB0EE674A7B
:10B4D800A6EE874AB3EE046AB4EEC54A74EE466A2D
:10B4E800F1EE10FA48BFF0EE656A072AC0ED066A69
:10B4F8003FF4CAADD6ED1D6ADFF8C8A2DFF8C892DE
:10B5080066EEE44AE4EE877AF4EEC57A77EEC67A18
:10B51800F1EE10FAB8BFF0EE657AC0ED077AFEF7E3
:10B528004EBAA04ED4ED017A94ED006A3188726962
:10B5380077EEA77AF0EE006AB0EE677AA6EE267A82
:10B548004E1E04EBC601D6EE267A08391032F6EE06
:10B55800003A27EE237A67EEA37A84ED207AC4EDC9
:10B56800217A914C274604F1800091ED027A91ED01
:10B57800036AD7ED036AD7ED027A52ED014A12ED5C
:10B58800025A37EE674A76EEC65A77EE277AE4EE25
:10B59800845A013EA1F10801E5EE047A07F1080793
:10B5A80002F1080236EE267A00F10800E4EE877A06
:10B5B800E5EE475A67EEA37A25EEA37AC0ED007A46
:10B5C80080ED017AD1D1BEF1140F7EF43AADFAF7CD
:10B5D80075FA039A754B801A5880D4F81451FEF7FF
:10B5E80030BDD4F81891B4F810C1714ACCF12003D9
:10B5F800DBB20CEB491702EB87079A0801F0C68506
:10B60800013216016B486C4907EB060807F1100276
:10B6180012ED024A12ED035A12ED016A12ED047A94
:10B6280050ED024A50ED035A50ED016A50ED047A8C
:10B6380064EE244A65EE255A66EE266A67EE277A96
:10B648001032904541ED024A41ED035A41ED016A3D
:10B6580041ED047A00F1100001F11001D8D15748EA
:10B66800A6F110010F4400EB0108214413F0030276
:10B6780009D0B7EC017AF8EC017A67EE277A013A3B
:10B68800E1EC017AF5D1BCF1000F40F03287BEF150
:10B69800140F7EF4D6ACFAF711FA039A434BD4F898
:10B6A8001451801A5880FEF7CCBC3E4E3E48B26812
:10B6B800B18927F0EBFA029B93F800E0BEF1140F72
:10B6C80001F0D785D4F814510135C4F8145129E78D
:10B6D800DFF8F89099F800108F0801F09D86384E31
:10B6E80007F101084FEA481806EB080C06F120029A
:10B6F800A6F1700012ED076A52ED056A12ED037AA1
:10B7080052ED017A52ED025A12ED084A52ED064AFC
:10B7180012ED045A26EE066A66EEA66A27EE077A46
:10B7280067EEA77AA4EE046A20329445E4EEA46A90
:10B7380000F11000A5EE057AE5EEA57AF1EEC65AFD
:10B74800B1EEE66AF1EEC76AB1EEE77A40ED085A63
:10B7580000ED076A40ED066A00ED057ACAD1A8F146
:10B768002002324404EB071711F0030018BF083217
:10B778000FD052ED017A12ED027A67EEA77A0138FE
:10B78800E7EE077A02F10802B1EEE77AA7EC017A50
:10B79800EFD1BEF1140F01F05D850135C4F81451E5
:10B7A800FEF7BFBBA8320020501D0020803E0020BD
:10B7B800C032002050340020601D0020403400209A
:10B7C800D01D0020445400203C5D0020A2320020FF
:10B7D800894E318873684FEA51094FEA89005FEA58
:10B7E800D10C04EB000204EB810500F0A18000F10C
:10B7F80010010CF1010C814F02EB0C1C2944103292
:10B8080003F1100E05F1100050ED032A50ED043A33
:10B8180017ED043A17ED032A50ED026A10ED016A9C
:10B8280017ED020A17ED018A11ED044A11ED035ACA
:10B8380052ED044A52ED035A12ED027A52ED017AA2
:10B8480051ED020A11ED011A73EE238A72EE221AE3
:10B8580047ED048A47ED031A70EE268A78EE061A39
:10B8680047ED028A47ED011A74EE848A75EE851A4F
:10B8780042ED048A42ED031A77EE208A77EE811AA8
:10B8880042ED028A42ED011A73EE633A75EE655A8B
:10B898001EED035A32EE623A74EE644A65EE631A9C
:10B8A8001EED044A23EE052A64EE652AE3EE041A27
:10B8B8001032944524EE843AA3EE842A07F1100747
:10B8C8000EF1100EA5EE853A00F1100001F11001FD
:10B8D800E4EE852A40ED071A00ED082A01ED073A43
:10B8E80041ED082A5EED055A1EED065A70EE666AAD
:10B8F80038EE466A30EEC77A71EE677A26EE253A58
:10B9080065EEE63A25EE674A67EE054AE6EE053A41
:10B91800A6EE853AA7EE254AE7EEA54A00ED063AD7
:10B9280040ED053A01ED064A41ED054A7FF46CAF5A
:10B938001FFA89F91A46494631481EF08BFB72688E
:10B94800494628461EF086FB029B1A78142A7FF483
:10B9580044AE3CE6D4F818512A492B482B4BEA0050
:10B96800114415448A88196800EE102A643AC82AD6
:10B97800A8BFC822782AB8BF782207EE902AB8EE66
:10B98800C07AF8EEE77A00EB850577EE670A77EE7E
:10B99800876A67EE877A20EEA67AB8EE400AC7EE85
:10B9A800870A2846D5F81490D5F81880EF692E6ACA
:10B9B8001EF040FF029BC5F8149093F800E0C5F80C
:10B9C8001880BEF1140FEF612E6201F03884D4F8AC
:10B9D80018210F49D4F81451013281FB0213A3EB4B
:10B9E800E27909EB4903A2EB03090135C4F8189180
:10B9F800C4F81451F7E500BFA8320020601D0020EC
:10BA0800501D002098350020B453002034540020E5
:10BA180056555555C64E002B40F0D48596ED006A14
:10BA28009DED0A5AC34825EE866AFDEEE44AA5EE66
:10BA3800076AB0EE675AA6EE265A14EE901ABDEEC3
:10BA4800C56A16EE108A16EE107AF045A8BF77463A
:10BA58004145C8BF0F4606EE107AB8EEC66A012AFD
:10BA680080ED006A3DF4A7AF96ED046A9DED0B5A90
:10BA780025EE866AA5EE076AB0EE675AA6EE265A44
:10BA8800BDEEC56A16EE108A16EE107AF045A8BF0C
:10BA980077468845B8BF0F4606EE107AB8EEC66AF4
:10BAA800022A80ED016A3DF486AF96ED086A9DEDA5
:10BAB8000C5A25EE866AA5EE076AB0EE675AA6EE1E
:10BAC800265ABDEEC56A16EE108A16EE107AF045B3
:10BAD800A8BF77468845B8BF0F4606EE107AB8EE7D
:10BAE800C66A032A80ED026A3DF465AF96ED0C6ADA
:10BAF8009DED0D5A25EE866AA5EE076AB0EE675AE7
:10BB0800A6EE265ABDEEC56A16EE108A16EE107A13
:10BB1800F045A8BF77468845B8BF0F4606EE107AAD
:10BB2800B8EEC66A042A80ED036A3DF444AF96ED88
:10BB3800106A9DED0E5A25EE866AA5EE076AB0EEEC
:10BB4800675AA6EE265ABDEEC56A16EE108A16EE9C
:10BB5800107AF045A8BF77468845B8BF0F4606EE6D
:10BB6800107AB8EEC66A052A80ED046A3DF423AF60
:10BB780096ED146A9DED0F5A25EE866AA5EE076AC2
:10BB8800B0EE675AA6EE265ABDEEC56A16EE108AC2
:10BB980016EE107AF045A8BF77468845B8BF0F461D
:10BBA80006EE107AB8EEC66A062A80ED056A3DF4FC
:10BBB80002AF96ED186A9DED105A25EE866AA5EE3D
:10BBC800076AB0EE675AA6EE265ABDEEC56A16EEAB
:10BBD800108A16EE107AF045A8BF77468845B8BF98
:10BBE8000F46FDF7C6BEF0EEE76AB7EE005A35EE2F
:10BBF800665A9FED514ADFED515A9FED516A9FED0C
:10BC0800517A94ED690AF1EEC54AE6EE845AF5EEEA
:10BC1800C07AA6EEA56AF1EE10FAA6EE867A48BFBB
:10BC2800DFED497A27EE247A48BF37EEC77A27EE48
:10BC3800000A28F025FAB0F5617F00F3018607EEC7
:10BC4800900AB8EEE70ADFED417A20EE270A07EE00
:10BC5800906AB8EEE78AFDEEC07A17EE903A203384
:10BC6800402B40F2F3859FED3A0A28F009FA00B21A
:10BC780007EE900AB8EEE77AFFF702BB354A02F101
:10BC8800500003E00432824200F0BC811378262B76
:10BC9800F8D19578D3789D42F4D2FFF732BB2E487D
:10BCA80024F0A6FCFEF729BD2C4824F0A1FCFEF7E1
:10BCB8001EBD2B4824F09CFCFEF713BDD4F894015C
:10BCC800049B181AFEF783BB41F27013E35C002B48
:10BCD8003EF4F9A8234824F08BFCFEF7F4B8224B75
:10BCE80000930320A0703023052220491D4826F028
:10BCF80035F8FEF7E8B800230AAE3146184609229F
:10BD080014F042F901287EF4DEA80A9B93F8FE217C
:10BD1800552A01F0518241F2B41202210123A154A3
:10BD28006370FEF7D0B803236370FEF7CCB800BF8A
:10BD3800B045002054320020306E99BC2716983D3B
:10BD4800843459BEA40DC93FDB0F4940D06D393A40
:10BD580000000000B84300203C780020F87700205D
:10BD68000C790020C4780020550F0308987A03083E
:10BD780023690622652BA27034D92278032A14BFBE
:10BD88006FF0FF026FF07F02A3F1650303EA02037D
:10BD980003F1010314BF4FF4807280229A42236199
:10BDA80020D23A68E768023203EB0708904581F031
:10BDB8009583B24A6760D16FC4F80880490203FBD3
:10BDC80001F30521176042F81C3C42F8183CA170A9
:10BDD800A268AB49012025F0EDFD012841F0E88378
:10BDE8000623A3700021A74825F004FA012841F092
:10BDF800DF83A3780133DBB2A370FFF764BA22783C
:10BE0800237DA14FDFF87892032A14BF4FF480787E
:10BE18004FF08008002B41D0012BFBD19B4B62686F
:10BE28001968386800234FEA412E4FF0FF31B1FB03
:10BE3800FEF112EB010B43F1000C0021614500F10A
:10BE4800020008BF584538BF83465A469049022029
:10BE580014F0DAF9032801F2AC8101A353F820F0B9
:10BE6800CF9E000879BE0008CF9E000879BE000862
:10BE78006268A3682669991AB14284BFE2602161A9
:10BE880003283FF475AF0133B3FBF8F208FB123215
:10BE98000AB143449B1A0022636022753A684946F6
:10BEA8000232002014F0B0F9032801F2828101A3C4
:10BEB80053F820F0CF9E000807BF0008CF9E000867
:10BEC80079BD00080AAE41F2FC173146E05900235B
:10BED800092214F059F801287DF4F5AF00230A9AD5
:10BEE8002370B2F80B30B3F5007F01F0FC8241F209
:10BEF800B41203210123A1546370FDF7E4BF636802
:10BF080084F814A00133A36088E7624A6248D2ED3E
:10BF1800006A624A90ED006A1278C4ED626A84EDA4
:10BF2800636A002A00F0E08276EE665A94F990215E
:10BF3800C4ED5F5A0132C4ED606A00F06686049B66
:10BF4800C4F89431002037EE677AFCEEE77A544D56
:10BF580084ED667A17EE902AA4F88421FF2295EDE5
:10BF6800005A84F89021FEF742BADFED4E7A4E4B24
:10BF780094ED667AC3ED007AC3ED017AC3ED027AD7
:10BF88004A4BF0EE674AF0EE673A1968FDF77CB95C
:10BF9800F9F794FD029B039093F800E0BEF1140FAB
:10BFA80005BF434BD4F81451D4F814511D80FCF745
:10BFB800B0BE4049DFED407A0968C4ED4A7A11F015
:10BFC800805840F05E84DAF8001011F4800800F020
:10BFD800E9824FF00008B6EE007A67EE877AF4EE51
:10BFE800E57AF1EE10FAC8BFF0EE675A40F34984DB
:10BFF800C4ED665AFDF78CBB304B1E7806F0010C79
:10C00800FDF7D9BC234A2448D2ED007A234A90EDA3
:10C01800007A1278C4ED627A84ED637A002A00F01F
:10C028001B8477EE676A94F99021C4ED5F6A013248
:10C03800C4ED607A00F02087049BC4F89431002096
:10C048009FED187A164D84ED667AFF2295ED005A19
:10C0580084F89021FEF7CBB973EEE77AB7EE007A51
:10C06800F4EEC77AF1EE10FAC4ED4A7A41F3938000
:10C0780084EEA77A8DED0A7AFDF740BBE8780020B8
:10C0880058670020C47800205C790020647900207B
:10C098005C670020AC2F0020344600206856002042
:10C0A80048460020000000002C320020D440002028
:10C0B800803E002004310020000000800D3E00205A
:10C0C800002F00F03D8725EE866AC748A5EE076A6F
:10C0D800B0EE675AA6EE265ABDEEC56A16EE10CA2D
:10C0E80016EE107AF445A8BF77466145C8BF0F46DB
:10C0F80006EE107AB8EEC66A012A80ED006A3DF4B1
:10C108005EAC96ED046A9DED0B5A25EE866AA5EEA7
:10C11800076AB0EE675AA6EE265ABDEEC56A16EE55
:10C1280010CA16EE107AF445A8BF77466145C8BF15
:10C138000F4606EE107AB8EEC66A022A80ED016A4A
:10C148003DF43DAC96ED086A9DED0C5A25EE866AE5
:10C15800A5EE076AB0EE675AA6EE265ABDEEC56A86
:10C1680016EE10CA16EE107AF445A8BF7746614558
:10C17800C8BF0F4606EE107AB8EEC66A032A80EDED
:10C18800026A3DF41CAC96ED0C6A9DED0D5A25EE45
:10C19800866AA5EE076AB0EE675AA6EE265ABDEE85
:10C1A800C56A16EE10CA16EE107AF445A8BF77468F
:10C1B8006145C8BF0F4606EE107AB8EEC66A042A73
:10C1C80080ED036A3DF4FBAB96ED106A9DED0E5AC7
:10C1D80025EE866AA5EE076AB0EE675AA6EE265ADD
:10C1E800BDEEC56A16EE10CA16EE107AF445A8BF61
:10C1F80077466145C8BF0F4606EE107AB8EEC66AA4
:10C20800052A80ED046A3DF4DAAB96ED146A9DEDDB
:10C218000F5A25EE866AA5EE076AB0EE675AA6EEB3
:10C22800265ABDEEC56A16EE10CA16EE107AF44507
:10C23800A8BF77466145C8BF0F4606EE107AB8EE2C
:10C24800C66A062A80ED056A3DF4B9AB96ED186A10
:10C258009DED105A25EE866AA5EE076AB0EE675A7C
:10C26800A6EE265ABDEEC56A16EE10CA16EE107A6C
:10C27800F445A8BF77466145C8BF0F4606EE107A59
:10C28800B8EEC66A072A80ED066A3DF498AB96EDCB
:10C298001C6A9DED115A65EE865AE5EE075AE6EEE0
:10C2A800A57AFDEEE77A17EE902A9645A8BF96463E
:10C2B8008A42A8BF714607EE901AF8EEE77AC0EDF9
:10C2C800077AFDF77CBB8222FDF7A9BEDFED477A2E
:10C2D800FDF771BEBBF93820CBF8201007EE902A85
:10C2E8000121F8EEE77ACBF86020CBF87C10002229
:10C2F800012CCBED1C7ACBED1B7ACBF8742001F026
:10C308009080AC427EF44DA9BBF93A20CBF864206A
:10C3180007EE902A00210122F8EEE77ACBF82410E4
:10C32800CBF890200022012CCBED217ACBED207A9E
:10C33800CBF8882001F01E80AC427EF466A9BBF9D8
:10C348003C20CBF8682007EE902A00210122F8EE65
:10C35800E77ACBF82810CBF8A4200022012CCBEDEB
:10C36800267ACBED257ACBF89C207EF482A99FED26
:10C37800208A032E29D04FB107EE907AF8EEE77A9B
:10C38800F4EEC87AF1EE10FA01F1A180194A1A4CBC
:10C39800039B1168DBF86820D88094F8200102EB31
:10C3A800550292FBF5F50022CBF828508A620A6301
:10C3B800CA6228B1114A126832F480637EF45CA91B
:10C3C800012023F013FDFEF757B9B0EE480A27F015
:10C3D80057FE00B2CFE7F7EE006AFDF7D1BCF7EEE3
:10C3E800006AFDF747BD00BF543200200000024339
:10C3F800000000003C660020501D0020CC400020BA
:10C408006D4D6E4F95ED004A95ED057AD5ED014AD3
:10C4180095ED066AD5ED046A95ED035AD5ED025AF5
:10C4280067EE897A07EB8602A4EE277AA4EEA76A5C
:10C4380066EEC76AA5EE476AE5EEA76A20EE070A28
:10C4480085ED056AC5ED066A82ED007A29EE088A4F
:10C4580027F016FE69EE288AD5ED0E5AD5ED176A33
:10C4680095ED091AD5ED121A95ED0F5A95ED187A32
:10C4780095ED0A2AD5ED132A95ED0D6AD5ED167AB4
:10C4880095ED0C3AD5ED0B3A95ED154AD5ED144AD4
:10C49800E1EE085A002207EB8601E8EEA16A00B235
:10C4A800C4F80021A2EE085AC4F80421C4F80821EF
:10C4B800A8EEA27A26EE656A67EEE67AA3EE655ADA
:10C4C800A3EE886AA6EEC47AE8EEA47A85ED0E5A41
:10C4D800C1ED205A85ED0F6AC1ED406A85ED177AE6
:10C4E800C5ED187AFEF7ABBE76EEC65AF0EE466A90
:10C4F8001CE59F00314B03EBC9195FEA9C0300EB75
:10C508000708274400F0918701331B0109EB030654
:10C5180009F1100208F1100007F1100112ED024AAA
:10C5280012ED035A12ED016A12ED047A50ED024A37
:10C5380050ED035A50ED016A50ED047A64EE244A36
:10C5480065EE255A66EE266A67EE277A103296421D
:10C5580041ED024A41ED035A41ED016A41ED047A89
:10C5680000F1100001F11001D8D1103B994408EBFB
:10C5780003001F441CF0030C3FF489A8B9EC017AAE
:10C58800F0EC017A67EE277ABCF1010CE7EC017A4E
:10C59800F4D1FFF77CB80A4BD3F800E0BEF932704B
:10C5A800FEF74EBAB6EE007AF4EEC75AF1EE10FA7C
:10C5B8003FF711ADFDF7ACB82C350020C032002094
:10C5C800D440002096ED006A9DED0A4AE24825EE27
:10C5D800866AFDEEE43AA4EE076AB0EE674AA6EE74
:10C5E800264A13EE901AB4EEC45AF1EE10FAB0EEE1
:10C5F800446A88BFB0EE646ABDEEC66A16EE108A59
:10C6080016EE107AF045A8BF77464145C8BF0F46D9
:10C6180006EE107AB8EEC66A012A80ED006A3DF48B
:10C62800CAA996ED046A9DED0B4A25EE866AA4EE2A
:10C63800076AB0EE674AA6EE264AB4EEC45AF1EE8F
:10C6480010FAB0EE446A88BFB0EE646ABDEEC66AFE
:10C6580016EE108A16EE107AF045A8BF7746884580
:10C66800B8BF0F4606EE107AB8EEC66A022A80ED09
:10C67800016A3DF4A0A996ED086A9DED0C4A25EEE5
:10C68800866AA4EE076AB0EE674AA6EE264AB4EEBA
:10C69800C45AF1EE10FAB0EE446A88BFB0EE646A8C
:10C6A800BDEEC66A16EE108A16EE107AF045A8BFDF
:10C6B80077468845B8BF0F4606EE107AB8EEC66AC8
:10C6C800032A80ED026A3DF476A996ED0C6A9DED89
:10C6D8000D4A25EE866AA4EE076AB0EE674AA6EE12
:10C6E800264AB4EEC45AF1EE10FAB0EE446A88BF96
:10C6F800B0EE646ABDEEC66A16EE108A16EE107ABF
:10C70800F045A8BF77468845B8BF0F4606EE107AB1
:10C71800B8EEC66A042A80ED036A3DF44CA996ED8A
:10C72800106A9DED0E4A25EE866AA4EE076AB0EE01
:10C73800674AA6EE264AB4EEC45AF1EE10FAB0EEF5
:10C74800446A88BFB0EE646ABDEEC66A16EE108A07
:10C7580016EE107AF045A8BF77468845B8BF0F4651
:10C7680006EE107AB8EEC66A052A80ED046A3DF432
:10C7780022A996ED146A9DED0F4A25EE866AA4EE6D
:10C78800076AB0EE674AA6EE264AB4EEC45AF1EE3E
:10C7980010FAB0EE446A88BFB0EE646ABDEEC66AAD
:10C7A80016EE108A16EE107AF045A8BF774688452F
:10C7B800B8BF0F4606EE107AB8EEC66A062A80EDB4
:10C7C800056A3DF4F8A896ED186A9DED104A25EE25
:10C7D800866AA4EE076AB0EE674AA6EE264AB4EE69
:10C7E800C45AF1EE10FAB0EE446A88BFB0EE646A3B
:10C7F800BDEEC66A16EE108A16EE107AF045A8BF8E
:10C8080077468845B8BF0F4606EE107AB8EEC66A76
:10C81800072A80ED066A3DF4CEA896ED1C6A9DEDC8
:10C82800114A65EE865AE7EE045AE6EEA57AB4EEAA
:10C83800E75AF1EE10FAC8BFF0EE647AFDF7ABB82C
:10C8480007EE906A9FED450AB8EEE78A03F0C6F94D
:10C8580020EE080AFFF709BA77EEC76AF0EE477AC2
:10C86800FFF7E1BBBEF834309FED3D7A07EE903A12
:10C87800F8EEE77A3B4B67EE877AC3ED007AFDF76F
:10C88800ECB8B7EE007A77EE677AF4EEE75AF1EE95
:10C8980010FA88BFF0EE675AFFF7AABBBEF1010F86
:10C8A80040F3BF8507EE103AB8EEC77AC7EE876A3D
:10C8B800B1EEE68A032E13D04FB107EE907AF8EE68
:10C8C800E77AF4EEC87AF1EE10FA00F10086DBF8A8
:10C8D800602002EB550292FBF5F2CBF8202010E520
:10C8E800B0EE480A27F0CCFB00B2E5E7BEF1010F35
:10C8F80040F3408507EE103AB8EEC77AC7EE876A6C
:10C90800B1EEE68A032E13D04FB107EE907AF8EE17
:10C91800E77AF4EEC87AF1EE10FA00F1D885DBF880
:10C92800642002EB550292FBF5F2CBF8242003E5D4
:10C93800B0EE480A27F0A4FB00B2E5E7BEF1010F0C
:10C948007FF715AD07EE103AB8EEC77AC7EE876ADB
:10C95800B1EEE68A0DE500BF5432002084F9223F8B
:10C968006F12833A1800002096ED006A9DED0A4A7E
:10C97800A94825EE866AFDEEE43AA4EE076AB0EE11
:10C98800674AA6EE264A13EE907AB4EEC45AF1EE40
:10C9980010FAB0EE446A88BFB0EE646ABDEEC66AAB
:10C9A80016EE10CA16EE101AF445A8BF7146674570
:10C9B800C8BF394606EE101AB8EEC66A012A80EDDD
:10C9C800006A3DF4FBAF96ED046A9DED0B4A25EE37
:10C9D800866AA4EE076AB0EE674AA6EE264AB4EE67
:10C9E800C45AF1EE10FAB0EE446A88BFB0EE646A39
:10C9F800BDEEC66A16EE10CA16EE101AF445A8BFA8
:10CA08007146BC45B8BF394606EE101AB8EEC66A7C
:10CA1800022A80ED016A3DF4D1AF96ED086A9DEDDA
:10CA28000C4A25EE866AA4EE076AB0EE674AA6EEBF
:10CA3800264AB4EEC45AF1EE10FAB0EE446A88BF42
:10CA4800B0EE646ABDEEC66A16EE10CA16EE101A8B
:10CA5800F445A8BF7146BC45B8BF394606EE101A62
:10CA6800B8EEC66A032A80ED026A3DF4A7AF96EDD8
:10CA78000C6A9DED0D4A25EE866AA4EE076AB0EEB3
:10CA8800674AA6EE264AB4EEC45AF1EE10FAB0EEA2
:10CA9800446A88BFB0EE646ABDEEC66A16EE10CA74
:10CAA80016EE101AF445A8BF7146BC45B8BF394602
:10CAB80006EE101AB8EEC66A042A80ED036A3DF441
:10CAC8007DAF96ED106A9DED0E4A25EE866AA4EEBE
:10CAD800076AB0EE674AA6EE264AB4EEC45AF1EEEB
:10CAE80010FAB0EE446A88BFB0EE646ABDEEC66A5A
:10CAF80016EE10CA16EE101AF445A8BF7146BC45CA
:10CB0800B8BF394606EE101AB8EEC66A052A80ED97
:10CB1800046A3DF453AF96ED146A9DED0F4A25EE75
:10CB2800866AA4EE076AB0EE674AA6EE264AB4EE15
:10CB3800C45AF1EE10FAB0EE446A88BFB0EE646AE7
:10CB4800BDEEC66A16EE10CA16EE101AF445A8BF56
:10CB58007146BC45B8BF394606EE101AB8EEC66A2B
:10CB6800062A80ED056A3DF429AF96ED186A9DED19
:10CB7800104A25EE866AA4EE076AB0EE674AA6EE6A
:10CB8800264AB4EEC45AF1EE10FAB0EE446A88BFF1
:10CB9800B0EE646ABDEEC66A16EE10CA16EE101A3A
:10CBA800F445A8BF7146BC45B8BF394606EE101A11
:10CBB800B8EEC66A072A80ED066A3DF4FFAE96ED28
:10CBC8001C6A9DED114A65EE865AE7EE045AE6EEB8
:10CBD800A57AB4EEE75AF1EE10FAC8BFF0EE647A1F
:10CBE800FDEEE77A17EE901A8E45A8BF8E468F4263
:10CBF800D8BF774607EE907AF8EEE77AC0ED077A65
:10CC0800FDF7D9BE054EFCF786BFD4F89401049B06
:10CC1800181AFFF798B900BF54320020A43E00202C
:10CC2800002F00F03F83BD4E9DED0A4A96ED006A45
:10CC380025EE866AA4EE076AB0EE674AA6EE264A93
:10CC4800B0EE446A33B1B4EE445AF1EE10FAC8BFFC
:10CC5800B0EE646AFDEEE44ABDEEC66A14EE907A60
:10CC680016EE101A8F4214EE90CA00F32C84714508
:10CC7800A8BF714606EE101AA948B8EEC66A012A7E
:10CC880080ED006A3CF49BAE96ED046ADDED0B4A3C
:10CC980025EE866AA4EE876AF0EE674AE6EE264A33
:10CCA800B0EE646A002B00F00484B4EEE45AF1EEAE
:10CCB80010FA40F3FE8339467145A8BF714606EE67
:10CCC800101AB8EEC66A022A80ED016A3CF477AE03
:10CCD80096ED086ADDED0C4A25EE866AA4EE876AB1
:10CCE800F0EE674AE6EE264AB0EE646A002B00F0E2
:10CCF800D783B4EEE45AF1EE10FA40F3D183394603
:10CD08007145A8BF714606EE101AB8EEC66A032A26
:10CD180080ED026A3CF453AE96ED0C6ADDED0D4AE7
:10CD280025EE866AA4EE876AF0EE674AE6EE264AA2
:10CD3800B0EE646A002B00F0AA83B4EEE45AF1EE78
:10CD480010FA40F3A48339467145A8BF714606EE30
:10CD5800101AB8EEC66A042A80ED036A3CF42FAEB6
:10CD680096ED106ADDED0E4A25EE866AA4EE876A16
:10CD7800F0EE674AE6EE264AB0EE646A002B00F051
:10CD88007D83B4EEE45AF1EE10FA40F37783394626
:10CD98007145A8BF714606EE101AB8EEC66A052A94
:10CDA80080ED046A3CF40BAE96ED146ADDED0F4A93
:10CDB80025EE866AA4EE876AF0EE674AE6EE264A12
:10CDC800B0EE646A002B00F05083B4EEE45AF1EE42
:10CDD80010FA40F34A8339467145A8BF714606EEFA
:10CDE800101AB8EEC66A062A80ED056A3CF4E7AD6B
:10CDF80096ED186ADDED104A25EE866AA4EE876A7C
:10CE0800F0EE674AE6EE264AB0EE646A002B00F0C0
:10CE18002383B4EEE45AF1EE10FA40F31D83394649
:10CE28007145A8BF714606EE101AB8EEC66A072A01
:10CE380080ED066A3CF4C3AD96ED1C6ADDED114A3F
:10CE480065EE865AE4EE875AE5EEA67A002B00F0E6
:10CE5800FB82F4EEC57AF1EE10FA40F1F5823A461B
:10CE68007245A8BF7246944607EE90CAF8EEE77A74
:10CE7800C0ED077AFCF7A3BDD4F89401049B181AF7
:10CE8800FFF7DEB896ED000A0593039227F0F8F84D
:10CE98002449DFF8A4E0D1F8EC10DFF8A0C0039A29
:10CEA800ACF800008EFB013EC917C1EBAE1107EECE
:10CEB800901AF8EEE77A059BFDEEE77A17EE901ADE
:10CEC800ACF80210FCF72CBE07EE906A9FED167ABC
:10CED80084F8FC61B8EEE70ADFED147A20EE070A61
:10CEE80030EE277AFDEEC76A16EE903A2033402BD3
:10CEF80040F24A82DFED0E8A0E4BFDEEC07AC3ED9A
:10CF0800018A17EE903A2033402B00F23A8202F061
:10CF180065FE84ED800AFDF7FBBD00BFB04500202B
:10CF280054320020EC02002035FA8E3CDB0FC93F5A
:10CF38000000000018000020D34D6210803E002041
:10CF480025EE866AA5EE076AB0EE675AA6EE265A5F
:10CF5800BDEEC56A16EE100A814200F39D81704548
:10CF6800A8BF704606EE100AB8EEC66AB8F1000F00
:10CF780000F04083D248012A80ED006A3CF41FADDE
:10CF880096ED046A9DED0B5A25EE866AA5EE076AB2
:10CF9800B0EE675AA6EE265ABDEEC56A16EE107AAE
:10CFA800B94200F377817745A8BF774606EE107A35
:10CFB800B8EEC66AB8F1000F00F01183022A80EDBE
:10CFC800016A3CF4FCAC96ED086A9DED0C5A25EE1E
:10CFD800866AA5EE076AB0EE675AA6EE265ABDEE37
:10CFE800C56A16EE107AB94200F352817745A8BF98
:10CFF800774606EE107AB8EEC66AB8F1000F00F070
:10D008000F83032A80ED026A3CF4D9AC96ED0C6AD2
:10D018009DED0D5A25EE866AA5EE076AB0EE675AB1
:10D02800A6EE265ABDEEC56A16EE107AB94200F38E
:10D038002D817745A8BF774606EE107AB8EEC66A06
:10D04800B8F1000F00F0E182042A80ED036A3CF495
:10D05800B6AC96ED106A9DED0E5A25EE866AA5EEE1
:10D06800076AB0EE675AA6EE265ABDEEC56A16EEF6
:10D07800107AB94200F314817745A8BF774606EEC7
:10D08800107AB8EEC66AB8F1000F00F02D83052AB1
:10D0980080ED046A3CF493AC96ED146A9DED0F5A4A
:10D0A80025EE866AA5EE076AB0EE675AA6EE265AFE
:10D0B800BDEEC56A16EE107AB94200F3EF807745E7
:10D0C800A8BF774606EE107AB8EEC66AB8F1000F28
:10D0D80000F0FF82062A80ED056A3CF470AC96EDFC
:10D0E800186A9DED105A25EE866AA5EE076AB0EE1D
:10D0F800675AA6EE265ABDEEC56A16EE107AB942F0
:10D1080000F3C2807745A8BF774606EE107AB8EEDE
:10D11800C66AB8F1000F00F08E82072A80ED066A11
:10D128003CF44DAC96ED1C6A9DED115A65EE865A9D
:10D13800E5EE075AE5EEA67AFDEEE77A17EE902AB5
:10D14800914203DC7245A8BF7246114607EE901A59
:10D15800F8EEE77AB8F1000F7FF48AAE089B002B4F
:10D168007FF486AE039B079A9342B8BFF0EE647AC9
:10D178007EE69FED540A544B25EE800A1D4626F0A4
:10D188007FFFE880D4F81451FCF75BBF4F48504943
:10D198008046FEF76BBA4F49096811F080587EF453
:10D1A8001AAFFEF710BFD4F89401049B181AFEF7C3
:10D1B800C5B8237DFEF72EBE93F8FF21AA2A7EF478
:10D1C800AAADD3F8C61149B193F8C221A2F10B0058
:10D1D80001282DD902F0F702062A29D0D3F8D61152
:10D1E80049B193F8D221A2F10B00012820D902F00D
:10D1F800F702062A1CD0D3F8E61149B193F8E221C8
:10D20800A2F10B00012813D902F0F702062A0FD069
:10D21800D3F8F61100293EF47EAD93F8F231A3F16C
:10D228000B02012A04D903F0F703062B7EF473AD31
:10D2380041F2FC120123A150A370FEF744BEF8F797
:10D248003DFC029A204B92F800E0039A801A58801D
:10D25800FEF7BDBBF8F732FC029A1B4B92F800E0D0
:10D26800039A99F80010D4F81451801A9880FEF7A0
:10D2780094BAF8F723FC029A134B92F800E0039A49
:10D28800801A5880FEF71EBA0F463EE70F46D3E6CF
:10D298000F46AEE60F4689E6084663E60F4611E7F5
:10D2A8000F46ECE60AA9BDEEE46A01EB8202944659
:10D2B8000948034E09941A4616EE107A434627E0A9
:10D2C800543200200000C842803E00204034002034
:10D2D800501D002004310020B0450020000000004F
:10D2E800E4CB1641DB0F49C0DB0FC940E4CB16C1C4
:10D2F800DB0FC93FDB0F494092E741B99730083C43
:10D3080015A82ABE6145A6EC016A00F1100035D0C7
:10D3180090ED006AB1EC014A25EE866AA7EE046A30
:10D32800B0EE674AA6EE864AB0EE446A32B1B4EE71
:10D33800445AF1EE10FAC8BFB0EE646ABDEEC66A90
:10D3480016EE108A474506EE107A04DCF045A8BFB1
:10D35800F04606EE108AB8EEC66A002BD2D1089CB9
:10D36800002CCFD1039CA046079CA045B8BFB0EEC7
:10D37800646AC7E71FED278AFFF7C4BA099CFCF760
:10D388001EBB1FED2A0AC4E5B4EEE70AF1EE10FA57
:10D3980040F322811FED2C6A5FED2F6A01E0B0EEA9
:10D3A800677AB4EEE67AF1EE10FA77EE467AF6DCB2
:10D3B8001FED347AF4EEC77AF1EE10FA40F10981E4
:10D3C8001FED376A5FED376A01E0F0EE477AF4EE59
:10D3D800E67AF1EE10FA37EE867AF6D45FED3C7A0B
:10D3E800B4EEE77AF1EE10FA22DD5FED3E7A37EE21
:10D3F800C77A27EE076A5FED405A5FED406A5FED36
:10D40800407AE6EE256A67EE065AE6EE267AA5EE3B
:10D41800A77AF0EE478A6FE5CA4F07F18002FEF758
:10D42800A3B99FEDC98AFFF745BA4046FFF7A2B8EE
:10D43800DFEDC67AB4EEE77AF1EE10FA44BFDFED1D
:10D44800C47A37EEC77AD4E7FDEEE77A17EE902A6A
:10D45800BA42FFF609AD03E5BDEEC66A16EE101A2C
:10D46800B942BFF6DDAC3946DDE4BDEEC66A16EE5C
:10D47800101AB942BFF6B0AC3946B0E4BDEEC66A80
:10D4880016EE101AB942BFF683AC394683E4BDEEF6
:10D49800C66A16EE101AB942BFF656AC394656E4BB
:10D4A800BDEEC66A16EE101AB942BFF629AC394667
:10D4B80029E4BDEEC66A16EE101AB942BFF6FCABF7
:10D4C8003946FFF7FCBB14EE901AFFF7D3BB039B5A
:10D4D800ABF8A850D8809B4CFDF7D5B823F054FD85
:10D4E8002369FEF766BC137C022B7EF400AD92F82C
:10D4F800FE31552B7EF4FBAC92F8FF31AA2B7EF45B
:10D50800F6ACD689E759934B37441F6092F80DE083
:10D5180041F210210EF1FF337F2B44F801E03EF673
:10D52800E6ACCEF100033EEA03037EF4E0AC4FEA3A
:10D538004E2341F21821013B6350D08A00B9506A4A
:10D54800854941F20423E050B2F811305B0103F23F
:10D55800FF135B120B60B2F8131001B9116A400097
:10D568001E440644891B41F2082C40F6F476B1FBB0
:10D57800FEF1B14244F80C1040F2C5804FF6F47643
:10D58800B14240F2BC8003212170D26A73493B4406
:10D59800184441F20C2641F21C230978A051E250AC
:10D5A80009B926F067FBA3780133A370FCF78BBC9D
:10D5B80002287CF488AC41F2B4120123A3546370AE
:10D5C800FCF781BC94F87031002B7BF419AEFBF7A3
:10D5D80004BEB0EE677A01E7F0EE477AE8E6089B0A
:10D5E800002B7FF4EBAC039B079FBB42B8BFB0EEA8
:10D5F800646AE3E4089B002B7FF4BCAC039B0798A8
:10D608008342B8BFB0EE646AB4E4089B002B7FF491
:10D618001BAD039B079FBB42B8BFB0EE646A13E51E
:10D62800089B002B7FF4EDAC039B079FBB42B8BF60
:10D63800B0EE646AE5E4089B002B7FF46EAD039BB3
:10D64800079FBB42B8BFB0EE646A66E5444A454BE3
:10D6580010681B689847444BD7ED006A93ED007A31
:10D66800424BD3ED007A424B83ED020A414B67EE01
:10D67800277A2B4427EEAC7AD3ED007A3E4B67EE3F
:10D68800277AF0EE665AE7EEAD5A93ED006AB1EEEE
:10D69800467AB4EEE57AF1EE10FA08DCB4EEE56A03
:10D6A800F1EE10FA8CBFB0EE657AB0EE467A334BE5
:10D6B8001B78012B02D0192B7BF40CADDFED307AEF
:10D6C800F4EEE7DAF1EE10FACCBF01230023FBF702
:10D6D8000CBD089B002B7FF4FDAC039B079FBB424E
:10D6E800B8BFB0EE646AF5E4089B002B7FF4CFACBA
:10D6F800039B079FBB42B8BFB0EE646AC7E402222F
:10D708002270002242E701232370FEF7F0BB132B9F
:10D7180005D1B0EE480A26F0B3FC039B1880B0EEA2
:10D72800480ADBF8083217489847029B1B78132BE6
:10D73800B0EE408A7CF4B4AD26F0A2FC039B58807E
:10D74800FCF7AEBD501D002000000000DB0FC9BF74
:10D75800DB0F49C054790020747900203479002007
:10D76800BC620020D0620020106200201800002057
:10D7780020320020E062002048630020746100200D
:10D7880000009642B45300200E4AD2ED007AB1EE62
:10D79800677AF4EEC7DAF1EE10FA0FD4F4EEE7DAAE
:10D7A800F1EE10FA88BFF0EE67DA074A87ED00CA93
:10D7B80012689A42BBF6A3ABFBF7CBBBF0EE47DA95
:10D7C800F3E700BF446300202863002003682DE9C5
:10D7D800F041DF691FB13B46BDE8F0411847002A18
:10D7E800164611DD04460D460E4400E023689B688A
:10D7F800204698470028F9D0236815F8011B1B68B4
:10D8080020469847AE42F1D1BDE8F081002322229C
:10D81800027043708370C370704710B5074B03F1F3
:10D828000C0193F900205C78845402449C78D470ED
:10D83800DC78947104338B42F3D110BDEC510308AA
:10D84800002870B51EDB0928044620DD012303EB00
:10D8580083035B00B0FBF3F2092AF8D87BB10E4EC4
:10D86800B4FBF3F00928CCBF57223022A6FB03E50E
:10D87800024403FB1044EB0801F8012BF0D100230C
:10D888000B7070BD2D230B7040420131DBE7303047
:10D8980001F8010BF3E700BFCDCCCCCC884230B403
:10D8A8004FF001042ED301FB04F4B0FBF4F58D42D4
:10D8B800F9D284B1AAB901E0B0FBF4F5092DCCBFC7
:10D8C800572230222A4404FB150003F8012BB4FB2D
:10D8D800F1F4002CF0D100221A7030BC7047B0FB74
:10D8E800F4F5092DCCBF372230222A4404FB150059
:10D8F80003F8012BB4FBF1F4002CF0D100221A70CC
:10D9080030BC70470546002AEBD1D7E72DE9F04730
:10D9180014461D46064600234FF47A7220462946CF
:10D9280025F0E8FEDFF848814B4A4C4F88FB003170
:10D938000144C31782FB002EC3EB611188FB012849
:10D9480087FB00278644464AC3EBEE2EC1EB011C39
:10D9580082FB0E29A0EB8C0C0744424A86F806C0CD
:10D96800C3EB27474FEAEE7C08EB010ACCEBA90C86
:10D9780082FB07824FEAE1780CEB4C0CC8EB6A1883
:10D98800AEEBCC0EC8EB0818DFF8E8C086F804E068
:10D99800A1EB880171718CFB0010F917C1EBE21241
:10D9A80040F2B55101FB1272C3EBE050B2F5896F3A
:10D9B8004FEA80073FDA40F2DA239A4243DCB2F5B5
:10D9C800B77FB4BF4FF0000C4FF0010C4FEA4C0882
:10D9D800254B08EB0C0103EBC1031FFA8CFE588C96
:10D9E800224908EB0C0301EBC30116310B2301E0BC
:10D9F80031F8020D82421BDA013BF9D11A4BC444BB
:10DA080003EBCC0C0123BCF80C00B37007F2B2771F
:10DA18000132121ABE44F270A6F800E020462946E8
:10DA28004FF47A72002325F065FE3281BDE8F08755
:10DA38000133DBB2E9E74FF0030EF44640F29650AB
:10DA48004FF00608CCE74FF0020EF44640F22940AA
:10DA58004FF00408C4E700BFC5B3A29107452EC222
:10DA6800ABAAAA2A73B06D16EC510308F851030843
:10DA780089888888792D031103685A1C02601970F7
:10DA8800704700BF2DE9F047089C2578002B804699
:10DA980089460CBF4FF0200A4FF0300A661C35B398
:10DAA800002A29DD334601E0024698B113F8011B2C
:10DAB800501E0029F8D1971E60B13D46013D5146E0
:10DAC8004046C8476B1C002BF8DC257827EAE7702E
:10DAD800013055B1041B29464046C847301916F88D
:10DAE800015B002DF7D1BDE8F087BDE8F087002A7B
:10DAF80004DC2846BDE8F0870020EBE7571EDCE78A
:10DB080083684268D0ED037A00EB830101339342C6
:10DB180081ED040A836004BF0023836000EB830364
:10DB280093ED047A036870EE277A9A42C0ED037A7F
:10DB380077EEC77AC0ED037A0CDA013307EE103AB4
:10DB4800F8EEC76AB7EE007A87EEA60A036030EEF1
:10DB5800070A704707EE102AB8EEC77A87EE870AD9
:10DB6800704700BF90ED057A90ED004AD0ED066A47
:10DB7800D0ED014AD0ED047A90ED035AD0ED025A67
:10DB8800A4EE007AB0EE406AB0EE470AB0EE667ACC
:10DB9800A6EE247A67EEC07AA0EE457AE6EE257AFC
:10DBA80080ED057AC0ED067A704700BFD0ED057AA2
:10DBB80090ED013AD0ED003AD0ED064A90ED024AD8
:10DBC80090ED077A90ED035A90ED086AD0ED045A6B
:10DBD800C0ED067AF0EE406A27EE830AC0ED056ACA
:10DBE800A3EEA60A80ED087AA4EE240AA5EE470A59
:10DBF800A5EEC60A80ED070A704700BFD0ED007A8F
:10DC080090ED017A30EE670AE7EE007AB0EE670A27
:10DC1800C0ED007A704700BF704700BF0A449142C8
:10DC280014D030B40139551E41F2210211F8014FC8
:10DC3800082380EA042004044CBF82EA4000400024
:10DC4800013B80B2F7D18D42F0D130BC70472DE94D
:10DC5800F341056906460F467DBBD0F80080C8F33E
:10DC68000A0323B30023D6F8008001931DF082F93C
:10DC7800042819D1214C236943F001032361BBB265
:10DC8800A8F800301DF076F904282ED108F1020317
:10DC98000193019B3F0C1F801DF06CF92369042838
:10DCA80023F00103236125D06FF0010505E01DF085
:10DCB80061F9042805D04FF0FF35284602B0BDE8C9
:10DCC800F0810E4C236943F002032361C4F81480E9
:10DCD800236943F0400323611DF04CF923690428AC
:10DCE80023F002032361BDD0E5E7236923F0010394
:10DCF8002361D9E7336804333360DEE7002002404C
:10DD0800F8B504460D468E180027B54201D12069A2
:10DD1800F8BDE368591CE160234415F8012B1A7219
:10DD28000429F2D1A1682046FFF791FFE76020613E
:10DD3800EBE700BF03681B6A03B11847704700BFD1
:10DD480003682DE9F041DF691FB13B46BDE8F041AA
:10DD58001847002A164611DD04460D460E4400E019
:10DD680023689B68204698470028F9D0236815F84F
:10DD7800011B1B6820469847AE42F1D1BDE8F081EF
:10DD880003689B69184700BF03685B69184700BFB1
:10DD98000368DB68184700BF03689B68184700BF23
:10DDA80003685B68184700BF03681B68184700BF13
:10DDB800014B1868F8E700BFF81B0020054B53F823
:10DDC800203033B11A689B88918A0B4218BF1B0414
:10DDD80093617047045C002003682DE9F04F03F15C
:10DDE8003845644EAD0A0124755D05F01F066D09BE
:10DDF800022D04FA06F400F0A280032D00F0A4809E
:10DE0800012D52D08088B0FA80F4C4F11F04A4B266
:10DE1800E50803EB850504F007042E6AA4000F2724
:10DE2800A74026EA07062E622E6A01F0030702FAC7
:10DE380004F47A1E3443012AC1F3810CC1F300189B
:10DE48002C62C1F3411135D9C60700F197808507C7
:10DE580000F1A380440700F1B180020700F1BF8000
:10DE6800C60600F1CD80850600F1DB80440600F18E
:10DE7800E980020600F1F780C60500F105818505F5
:10DE880000F11381440500F12181020500F12F8181
:10DE9800C60400F13D81850400F14B81440400F182
:10DEA8005981020455D4BDE8F08F334D6E6934436F
:10DEB8006C61A7E7002422464FF0010E4FF00309DA
:10DEC80004E00132102A04F10204ECD00EFA02F642
:10DED80036EA0005F5D1D3F808A009FA04F5ED43B0
:10DEE8000AEA050AC3F808A0D3F808B00CFA04FA3D
:10DEF8004AEA0B0AC3F808A0B3F804A01FFA8AFA82
:10DF08002AEA06069E80B3F804A008FA02F646EA52
:10DF18000A06B6B29E801E682E401E60D3F800A086
:10DF280007FA04F646EA0A061E60D3F80CA001FABE
:10DF380004F605EA0A0A46EA0A05DD60C1E70E4D5D
:10DF4800AE693443AC615DE70B4DEE693443EC6177
:10DF580058E71A6822F040421A601A6842EA87773E
:10DF68001F60DA6822F0404242EA8171D960BDE858
:10DF7800F08F00BF80700308001002401A6822F07A
:10DF880003021A601A683A431A60DA6822F0030238
:10DF98000A438507DA607FF55DAF1A6822F00C0244
:10DFA8001A601A6842EA87021A60DA6822F00C02DC
:10DFB80042EA81024407DA607FF54FAF1A6822F01F
:10DFC80030021A601A6842EA07121A60DA6822F008
:10DFD800300242EA0112DA6002077FF541AF1A689F
:10DFE80022F0C0021A601A6842EA87121A60DA68D8
:10DFF80022F0C00242EA8112C606DA607FF533AF2A
:10E008001A6822F440721A601A6842EA07221A60F3
:10E01800DA6822F4407242EA01228506DA607FF566
:10E0280025AF1A6822F440621A601A6842EA872209
:10E038001A60DA6822F4406242EA81224406DA6011
:10E048007FF517AF1A6822F440521A601A6842EA3C
:10E0580007321A60DA6822F4405242EA0132DA6082
:10E0680002067FF509AF1A6822F440421A601A685E
:10E0780042EA87321A60DA6822F4404242EA813280
:10E08800C605DA607FF5FBAE1A6822F440321A60E2
:10E098001A6842EA07421A60DA6822F4403242EA11
:10E0A80001428505DA607FF5EDAE1A6822F4402258
:10E0B8001A601A6842EA87421A60DA6822F4402233
:10E0C80042EA81424405DA607FF5DFAE1A6822F43D
:10E0D80040121A601A6842EA07521A60DA6822F493
:10E0E800401242EA0152DA6002057FF5D1AE1A68A1
:10E0F80022F440021A601A6842EA87521A60DA6803
:10E1080022F4400242EA8152C604DA607FF5C3AEC7
:10E118001A6822F040721A601A6842EA07621A60A6
:10E12800DA6822F0407242EA01628504DA607FF51B
:10E13800B5AE1A6822F040621A601A6842EA87622D
:10E148001A60DA6822F0406242EA81624404DA60C6
:10E158007FF5A7AE1A6822F040521A601A6842EAA0
:10E1680007721A60DA6822F0405242EA0172DA60F5
:10E1780097E600BF036803F138422DE9F04F920A91
:10E18800584DAA5C02F01F0552090124022A04FA1C
:10E1980005F400F08C80032A00F08E80012A3CD020
:10E1A80001F003077A1E012AC1F3810CC1F300189C
:10E1B8008088C1F3411135D9C60700F197808507DA
:10E1C80000F1A380440700F1B180020700F1BF808D
:10E1D800C60600F1CD80850600F1DB80440600F11B
:10E1E800E980020600F1F780C60500F10581850582
:10E1F80000F11381440500F12181020500F12F810E
:10E20800C60400F13D81850400F14B81440400F10E
:10E218005981020455D4BDE8F08F334A55692C431F
:10E228005461BDE7002422464FF0010E4FF0030968
:10E2380004E00132102A04F10204ECD00EFA02F6CE
:10E2480036EA0005F5D1D3F808A009FA04F5ED433C
:10E258000AEA050AC3F808A0D3F808B00CFA04FAC9
:10E268004AEA0B0AC3F808A0B3F804A01FFA8AFA0E
:10E278002AEA06069E80B3F804A008FA02F646EADF
:10E288000A06B6B29E801E682E401E60D3F800A013
:10E2980007FA04F646EA0A061E60D3F80CA001FA4B
:10E2A80004F605EA0A0A46EA0A05DD60C1E70E4AED
:10E2B80095692C43946173E70B4AD5692C43D46163
:10E2C8006EE71A6822F040421A601A6842EA8777B5
:10E2D8001F60DA6822F0404242EA8171D960BDE8E5
:10E2E800F08F00BF80700308001002401A6822F007
:10E2F80003021A601A683A431A60DA6822F00302C5
:10E308000A438507DA607FF55DAF1A6822F00C02D0
:10E318001A601A6842EA87021A60DA6822F00C0268
:10E3280042EA81024407DA607FF54FAF1A6822F0AB
:10E3380030021A601A6842EA07121A60DA6822F094
:10E34800300242EA0112DA6002077FF541AF1A682B
:10E3580022F0C0021A601A6842EA87121A60DA6864
:10E3680022F0C00242EA8112C606DA607FF533AFB6
:10E378001A6822F440721A601A6842EA07221A6080
:10E38800DA6822F4407242EA01228506DA607FF5F3
:10E3980025AF1A6822F440621A601A6842EA872296
:10E3A8001A60DA6822F4406242EA81224406DA609E
:10E3B8007FF517AF1A6822F440521A601A6842EAC9
:10E3C80007321A60DA6822F4405242EA0132DA600F
:10E3D80002067FF509AF1A6822F440421A601A68EB
:10E3E80042EA87321A60DA6822F4404242EA81320D
:10E3F800C605DA607FF5FBAE1A6822F440321A606F
:10E408001A6842EA07421A60DA6822F4403242EA9D
:10E4180001428505DA607FF5EDAE1A6822F44022E4
:10E428001A601A6842EA87421A60DA6822F44022BF
:10E4380042EA81424405DA607FF5DFAE1A6822F4C9
:10E4480040121A601A6842EA07521A60DA6822F41F
:10E45800401242EA0152DA6002057FF5D1AE1A682D
:10E4680022F440021A601A6842EA87521A60DA688F
:10E4780022F4400242EA8152C604DA607FF5C3AE54
:10E488001A6822F040721A601A6842EA07621A6033
:10E49800DA6822F0407242EA01628504DA607FF5A8
:10E4A800B5AE1A6822F040621A601A6842EA8762BA
:10E4B8001A60DA6822F0406242EA81624404DA6053
:10E4C8007FF5A7AE1A6822F040521A601A6842EA2D
:10E4D80007721A60DA6822F0405242EA0172DA6082
:10E4E80097E600BF10B50409013C052C17D80D4B61
:10E4F80033F8142000F00F0042FA00F313F0010380
:10E508000DD0012303FA00F00138104025F042F93C
:10E51800054A064B125D104403EBC00010BD0020F5
:10E5280010BD00BF5871030864710308905E002095
:10E538002DE9F04F4A484B4B4B4C4FF090414FF070
:10E54800010A4FF002094FF004084FF0080C4FF091
:10E55800100E20274026802530F8022B12F0010FDC
:10E5680003D01960A3F804A0083312F0020F03D0F7
:10E578001960A3F80490083312F0040F03D019604F
:10E58800A3F80480083312F0080F03D01960A3F829
:10E5980004C0083312F0100F03D01960A3F804E088
:10E5A800083312F0200F02D019609F80083312F050
:10E5B800400F02D019609E80083312F0800F02D0FD
:10E5C80019609D80083312F4807F05D04FF4807B5A
:10E5D8001960A3F804B0083312F4007F05D04FF493
:10E5E800007B1960A3F804B0083312F4806F05D0DB
:10E5F8004FF4806B1960A3F804B0083312F4006F6D
:10E6080005D04FF4006B1960A3F804B0083312F476
:10E61800805F05D04FF4805B1960A3F804B008331D
:10E6280012F4005F05D04FF4005B1960A3F804B042
:10E63800083312F4804F05D04FF4804B1960A3F8CB
:10E6480004B00833D20B04D04FF4004219609A800A
:10E65800083301F58061A1427FF47EAFBDE8F08FF9
:10E6680058710308905E002000180048002867D001
:10E6780003682DE9F04F03F138445C4EA40A0125E4
:10E68800345D04F01F066409022C05FA06F558D01B
:10E69800032C00F0A580012C58D08088B0FA80F4B3
:10E6A800C4F11F04A4B2E50803EB850504F00704D0
:10E6B8002E6AA4000F27A74026EA07062E622E6AB4
:10E6C80001F00307A2407C1E3243012CC1F3810CE8
:10E6D800C1F300182A62C1F341113CD9C60700F101
:10E6E8008980850700F19580440700F1A38002071F
:10E6F80000F1B180C60600F1BF80850600F1CD802B
:10E70800440600F1DB80020600F1E980C60500F14D
:10E71800F780850500F10581440500F113810205A4
:10E7280000F12181C60400F12F81850400F13D81AB
:10E73800440400F14B81020400F15981BDE8F08FD7
:10E7480070472B4CA6693543A561A6E7284C666936
:10E7580035436561A1E7002422464FF0010E4FF0D2
:10E76800030904E00132102A04F10204E6D00EFA8B
:10E7780002F636EA0005F5D1D3F808A009FA04F53F
:10E78800ED430AEA050AC3F808A0D3F808B00CFA62
:10E7980004FA4AEA0B0AC3F808A0B3F804A01FFA5F
:10E7A8008AFA2AEA06069E80B3F804A008FA02F656
:10E7B80046EA0A06B6B29E801E682E401E60D3F84E
:10E7C80000A007FA04F646EA0A061E60D3F80CA071
:10E7D80001FA04F605EA0A0A46EA0A05DD60C1E715
:10E7E800034CE6693543E56157E700BF80700308CD
:10E7F800001002401A6822F003021A601A683A43AD
:10E808001A60DA6822F003020A438507DA607FF5A6
:10E818006BAF1A6822F00C021A601A6842EA870283
:10E828001A60DA6822F00C0242EA81024407DA60D0
:10E838007FF55DAF1A6822F030021A601A6842EA62
:10E8480007121A60DA6822F0300242EA0112DA602E
:10E8580002077FF54FAF1A6822F0C0021A601A68E3
:10E8680042EA87121A60DA6822F0C00242EA81128C
:10E87800C606DA607FF541AF1A6822F440721A6062
:10E888001A6842EA07221A60DA6822F4407242EAF9
:10E8980001228506DA607FF533AF1A6822F44062F8
:10E8A8001A601A6842EA87221A60DA6822F440621B
:10E8B80042EA81224406DA607FF525AF1A6822F41D
:10E8C80040521A601A6842EA07321A60DA6822F47B
:10E8D800405242EA0132DA6002067FF517AF1A6841
:10E8E80022F440421A601A6842EA87321A60DA68EB
:10E8F80022F4404242EA8132C605DA607FF509AF68
:10E908001A6822F440321A601A6842EA07421A600A
:10E91800DA6822F4403242EA01428505DA607FF57E
:10E92800FBAE1A6822F440221A601A6842EA87424B
:10E938001A60DA6822F4402242EA81424405DA6029
:10E948007FF5EDAE1A6822F440121A601A6842EA9E
:10E9580007521A60DA6822F4401242EA0152DA6079
:10E9680002057FF5DFAE1A6822F440021A601A68C1
:10E9780042EA87521A60DA6822F4400242EA815277
:10E98800C604DA607FF5D1AE1A6822F040721A60C8
:10E998001A6842EA07621A60DA6822F0407242EAAC
:10E9A80001628504DA607FF5C3AE1A6822F040621E
:10E9B8001A601A6842EA87621A60DA6822F04062CE
:10E9C80042EA81624404DA607FF5B5AE1A6822F043
:10E9D80040521A601A6842EA07721A60DA6822F02E
:10E9E800405242EA0172DA6002047FF5A7AE1A6863
:10E9F80022F040421A601A6842EA87771F60DA6894
:10EA080022F0404242EA8171D960BDE8F08F00BF30
:10EA1800002852D0036803F138422DE9F04F920ADA
:10EA2800504DAA5C02F01F0552090124022A04FA7B
:10EA380005F443D0032A00F09080012A43D001F066
:10EA480003077A1E012AC1F3810CC1F300188088DC
:10EA5800C1F341113CD9C60700F18880850700F150
:10EA68009480440700F1A280020700F1B080C60636
:10EA780000F1BE80850600F1CC80440600F1DA8002
:10EA8800020600F1E880C60500F1F680850500F170
:10EA98000481440500F11281020500F12081C604B9
:10EAA80000F12E81850400F13C81440400F14A8183
:10EAB800020400F15881BDE8F08F70472A4A956931
:10EAC8002C439461BBE7284A55692C435461B6E747
:10EAD800002422464FF0010E4FF0030904E00132F2
:10EAE800102A04F10204E6D00EFA02F636EA00050E
:10EAF800F5D1D3F808A009FA04F5ED430AEA050AA6
:10EB0800C3F808A0D3F808B00CFA04FA4AEA0B0ACA
:10EB1800C3F808A0B3F804A01FFA8AFA2AEA06067E
:10EB28009E80B3F804A008FA02F646EA0A06B6B2CE
:10EB38009E801E682E401E60D3F800A007FA04F6D7
:10EB480046EA0A061E60D3F80CA001FA04F605EAA4
:10EB58000A0A46EA0A05DD60C1E7034AD5692C437B
:10EB6800D4616CE780700308001002401A6822F034
:10EB780003021A601A683A431A60DA6822F003023C
:10EB88000A438507DA607FF56CAF1A6822F00C0239
:10EB98001A601A6842EA87021A60DA6822F00C02E0
:10EBA80042EA81024407DA607FF55EAF1A6822F014
:10EBB80030021A601A6842EA07121A60DA6822F00C
:10EBC800300242EA0112DA6002077FF550AF1A6894
:10EBD80022F0C0021A601A6842EA87121A60DA68DC
:10EBE80022F0C00242EA8112C606DA607FF542AF1F
:10EBF8001A6822F440721A601A6842EA07221A60F8
:10EC0800DA6822F4407242EA01228506DA607FF56A
:10EC180034AF1A6822F440621A601A6842EA8722FE
:10EC28001A60DA6822F4406242EA81224406DA6015
:10EC38007FF526AF1A6822F440521A601A6842EA31
:10EC480007321A60DA6822F4405242EA0132DA6086
:10EC580002067FF518AF1A6822F440421A601A6853
:10EC680042EA87321A60DA6822F4404242EA813284
:10EC7800C605DA607FF50AAF1A6822F440321A60D6
:10EC88001A6842EA07421A60DA6822F4403242EA15
:10EC980001428505DA607FF5FCAE1A6822F440224D
:10ECA8001A601A6842EA87421A60DA6822F4402237
:10ECB80042EA81424405DA607FF5EEAE1A6822F432
:10ECC80040121A601A6842EA07521A60DA6822F497
:10ECD800401242EA0152DA6002057FF5E0AE1A6896
:10ECE80022F440021A601A6842EA87521A60DA6807
:10ECF80022F4400242EA8152C604DA607FF5D2AEBD
:10ED08001A6822F040721A601A6842EA07621A60AA
:10ED1800DA6822F0407242EA01628504DA607FF51F
:10ED2800C4AE1A6822F040621A601A6842EA876222
:10ED38001A60DA6822F0406242EA81624404DA60CA
:10ED48007FF5B6AE1A6822F040521A601A6842EA95
:10ED580007721A60DA6822F0405242EA0172DA60F9
:10ED680002047FF5A8AE1A6822F040421A601A68B9
:10ED780042EA87771F60DA6822F0404242EA8171EE
:10ED8800D960BDE8F08F00BF10B1036882881A858A
:10ED9800704700BF10B1036882889A61704700BF4E
:10EDA80038B100298388026814BF002110218B40E4
:10EDB8009361704710B40A4B0A4A1C7801238340B8
:10EDC800234052F8200029B9B3FA83F149095DF8C4
:10EDD800044BE5E7191C18BF01215DF8044BDFE778
:10EDE800035C0020045C002030B1036882881B8A21
:10EDF8001A4214BF01200020704700BF2DE9F041DE
:10EE08000B4E346873691C400FD0DFF82880012747
:10EE1800B4FA84F3C3F11F0307FA03F558F8230083
:10EE280003689847AC437561F2D1BDE8F08100BF33
:10EE380000040140BC5B00202DE9F0410B4E346812
:10EE480073691C400FD0DFF828800127B4FA84F3D7
:10EE5800C3F11F0307FA03F558F82300036898471E
:10EE6800AC437561F2D1BDE8F08100BF00040140F8
:10EE7800BC5B00202DE9F0410B4E346873691C40DF
:10EE88000FD0DFF828800127B4FA84F3C3F11F03F9
:10EE980007FA03F558F8230003689847AC437561EF
:10EEA800F2D1BDE8F08100BF00040140BC5B002046
:10EEB8002DE9F0410B4E346873691C400FD0DFF820
:10EEC80028800127B4FA84F3C3F11F0307FA03F576
:10EED80058F8230003689847AC437561F2D1BDE840
:10EEE800F08100BF00040140BC5B00202DE9F04127
:10EEF8000B4E346873691C400FD0DFF82880012757
:10EF0800B4FA84F3C3F11F0307FA03F558F8230092
:10EF180003689847AC437561F2D1BDE8F08100BF42
:10EF280000040140BC5B00202DE9F0410B4E346821
:10EF380073691C400FD0DFF828800127B4FA84F3E6
:10EF4800C3F11F0307FA03F558F82300036898472D
:10EF5800AC437561F2D1BDE8F08100BF0004014007
:10EF6800BC5B00202DE9F0410B4E346873691C40EE
:10EF78000FD0DFF828800127B4FA84F3C3F11F0308
:10EF880007FA03F558F8230003689847AC437561FE
:10EF9800F2D1BDE8F08100BF00040140BC5B002055
:10EFA8000B490C4A0C4808B58B6943F001038B6187
:10EFB800136843F4805313600021402226F01DF8A3
:10EFC800064B4FF0FF321A60C3F8032008BD00BF9C
:10EFD8000010024000000140BC5B0020FC5B0020E8
:10EFE80003681B6A184700BF70B44E1C0568C272DC
:10EFF8008672AC69A44670BC604700BF2DE9F04139
:10F00800044618460D461646984623F0A9FE27687A
:10F01800E6722844A07229467D6943463246204656
:10F02800AC46BDE8F0416047036810B504461B686C
:10F038009847236820469B689847A37B0133A373AE
:10F0480010BD00BF03681B69184700BF10B50368EF
:10F0580004469B689847FF2301226373227310BDFF
:10F0680008B5FFF73FFA38B12D2282710022C2712C
:10F078002021BDE80840CBE408BD00BF0E4B9842F4
:10F088000AD0A3F57843984211D003F580639842DB
:10F098000FD04FF0FF3070470022084B03EB0213EC
:10F0A8005A89013292B25A81588980B27047012236
:10F0B800F3E70222F1E700BF00300140782A002080
:10F0C800427A02B9704710B504460368406804F1F3
:10F0D8000A0198470023637210BD00BF437A5A1C87
:10F0E8000344D2B242729972037A934200D802B9A9
:10F0F800704710B504460368406804F10A01984750
:10F108000023637210BD00BF98B10B4B012210B4ED
:10F1180002FA01F103F1750402E00333A34209D0B6
:10F128001A788242F9D15A780A42F6D001205DF85D
:10F13800044B70470020FAE75852030830B40A4DD0
:10F14800002305F16C0401E0272B0AD003EB4302EE
:10F158000133A15C8142F7D12A4430BC92F86E0099
:10F168007047002030BC7047EC51030870B54488E4
:10F1780006460D46C4F30B0422460021284625F016
:10F188003CFF3369094A934209D3094A934206D29C
:10F19800224628461946BDE8704024F09DBD23B19B
:10F1A80021462846BDE87040184770BDA4B503083D
:10F1B80090B60308064B07498B4202D30023184632
:10F1C80070471A88C2F30B029042F8D01433F3E761
:10F1D80030B10308A4B50308024A136823EA000003
:10F1E8001060704710880020F8B5174D2B78A52BB4
:10F1F80028D16B78BE2B25D1022229464FF6FF7005
:10F20800FEF70CFD114FAC1C22884AB1A618BE426D
:10F2180018D2052A16D92146FEF700FD3446F3E731
:10F2280021460222FEF7FAFC0222A118FEF7F6FC9C
:10F238000634074B641B1C8041F60F53C31A58420F
:10F248005841F8BD0020F8BD00F00308000004088C
:10F258002C2B00202DE9F04FDFF864914F4F8BB035
:10F268000326A7EB09071822002104A825F0C5FEEC
:10F278004B4BCDF8109005971A69120604D5494AE8
:10F288005A6002F188325A6001228DF82420342213
:10F29800DA60454B454C1B88ADF8003002226946C0
:10F2A80004A8FEF72DFD022269464FF6FF70FEF70F
:10F2B800B5FCDFF810A180464FF0000B544536D35B
:10F2C8000AAC002524F8245D0222214604A8FEF792
:10F2D80017FD022221464046FEF7A0FC40BAC04373
:10F2E800ADF80800022202A904A8FEF709FD079854
:10F2F80060B106ABC0F104022946184425F07DFE32
:10F30800069904A8FEF7A3FC079508909DF82430F9
:10F31800089A23B122490B6943F080030B61013E2F
:10F328002DD0002A9FD1FFF75FFF50B332E06588E8
:10F338008DF80DB0C5F30B05AB1DADF8083023886B
:10F34800C3F30B02ADF80A201B0B062202A904A87E
:10F358008DF80C30FEF7D4FC062202A94046FEF7D1
:10F368005DFC616880462A4604A8FEF7C9FC61680E
:10F3780040462A46FEF752FC143480469EE7002A8F
:10F38800D1D005201AF01EFC094B0A4A1A600A4B14
:10F398000A4ADA600BB0BDE8F08F00BF000004082D
:10F3A8000020024023016745CD52030830B103080D
:10F3B800FC9F0020EFBEADDE00ED00E00400FA0582
:10F3C80000F00308A4B503080378202B024600F1D7
:10F3D8000100F9D0092BF7D02D2B2CD02B2B03BFF4
:10F3E8005378B7EE000A0246B7EE000AA3F13001DF
:10F3F800C8B209289FED467A10D8F2EE046A07EEE3
:10F40800901AF8EEE77A12F8013FE7EE267AA3F1B0
:10F418003001C8B20928B0EE677AF0D92E2B4CD04B
:10F4280003F0DF03452B0BD0F7EE007A67EE276A6F
:10F4380020EE260A70475378BFEE000A0246D5E749
:10F4480010B451782D2959D02B290ABF9178501C16
:10F45800901C0024A1F13003092B53D8002303EB9F
:10F46800830301EB430310F8011FA1F13002092ABD
:10F47800A3F13003F3D9B3F59A7F28BF4FF49A73F9
:10F48800072B42D9DFED236A1A46F7EE007A083ACD
:10F49800072A67EEA67AFAD803F007032BB1F2EE33
:10F4A800046A013B67EEA67AFBD124B3C7EE276A4C
:10F4B8005DF8044B20EE260A70475378A3F130011B
:10F4C800C8B2092802F10102AAD8F2EE046AF0EEE5
:10F4D800665A07EE901AF8EEE77A12F8013F87EEBF
:10F4E800A66AA3F13001C8B2092866EEA56A37EE0C
:10F4F800067AEED994E767EE276AD9E7901C9178E7
:10F508000124A7E7F7EE007ACFE7F7EE007AC5E720
:10F518000000000020BCBE4CB5EEC00ADFED317A19
:10F52800F1EE10FACCBF30EE270A30EE670ADFEDB5
:10F538002E7A20EE270A30B5FDEEC07A87B017EE96
:10F54800904A054684EAE470002303A9A0EBE4701E
:10F558000193009302931FF075FC002CACBF20238D
:10F568002D2303A88DF8003023F0FAFB012803A906
:10F5780024D002282DD0032805BF302368466846CA
:10F588008DF8013025F041FD684623F0E9FB03388A
:10F59800C4B222466946284625F06EFD00232B5545
:10F5A800284623F0DDFB2E22431C2A540DEB0401D0
:10F5B800E81825F047FD284607B030BD30236846D7
:10F5C8008DF801308DF802308DF8033025F01DFDDF
:10F5D800DAE7302368468DF801308DF8023025F0DF
:10F5E80014FDD1E76F12033A00007A442DE9F04187
:10F5F800064615460846B6FBF2F43CB905FB14640A
:10F60800124B1B5D00F8013BBDE8F081B4FBF2F73B
:10F6180067B90E4B05FB174705FB1464DA5D00F864
:10F62800012B1B5D00F8013BBDE8F081B7FBF2F848
:10F63800B8F1000F02D04046FFF7D8FF05FB187855
:10F64800024B13F8082000F8012BE3E7A47A03081B
:10F65800104B2DE93048D3E9004554EA05020BD197
:10F668000346012200201871587198719A70DA7057
:10F6780018801881BDE83088074B1A6814EB020B14
:10F6880045F1000C5A466346FEF740F90120BDE8F3
:10F69800308800BFE01B0020385C0020F0B40288EE
:10F6A8008578164FC37804794179A2F2B27202F0D4
:10F6B800030606EB4606013D05EB860507EB450507
:10F6C800013BAE898579008940F2B557920807FB5E
:10F6D8000232931903EB430304EBC303C3EB031395
:10F6E80001EB8303C3EB031305EB830300214FF402
:10F6F8007A72C2FB0301F0BC704700BFEC510308EB
:10F70800FAB170B48E18044603E0101A14D1B1424D
:10F7180014D014F8012BA2F14103192B11F8013B65
:10F72800A3F1410598BF2032192D03F12000ECD92F
:10F73800D01A01D1002BEAD170BC7047002070BCF0
:10F7480070471046704700BF4FF0FF32FFF7D8BF31
:10F75800A0F16103192B98BF20387047A0F141032D
:10F76800192B98BF20307047202805D00938042865
:10F778008CBF00200120704701207047613819288C
:10F788008CBF002001207047413819288CBF002009
:10F7980001207047303809288CBF002001207047AD
:10F7A800A0F13003092B07D920F02000413819288F
:10F7B8008CBF0020012070470120704730B40268D8
:10F7C8001146531C036011F8024B0160D31C517899
:10F7D80003609378151D05601B0443EA0123D07864
:10F7E800234343EA006030BC704700BF0368591CDC
:10F7F8001A46016012F8021B0260587841EA00209C
:10F80800704700BF03685A1C02601878704700BF31
:10F8180038B504460068154624F05EFA22682A4482
:10F82800226038BD036810B40A0A5C1C04601A70B0
:10F8380003685A1C026019705DF8044B704700BFDA
:10F8480003685A1C026010B4197003680A0A5C1C29
:10F8580004601A7003680A0C5C1C04601A70036860
:10F86800090E5A1C026019705DF8044B704700BFFE
:10F8780003685A1C026019700368090A5A1C02605E
:10F88800197070472DE9F047002488B080460F466C
:10F898001E46A14605AD531C0393117839B325299B
:10F8A80033D1931CCDF810900393507830284ED064
:10F8B8004FF0000AA0F13003DBB2092B42D96C28C3
:10F8C80019D0642800F0938024D825281CD063D947
:10F8D800582876D063281BD131784046B847039A18
:10F8E800531C03931178043601340029D7D12046DC
:10F8F80008B0BDE8F087039B5A1C03921B78642B61
:10F908007CD02AD8252B54D1252140460134B8472C
:10F91800039AC0E7732833D044D975284FD106F12C
:10F92800040E30682B4600220A217646FDF7B6FF02
:10F93800049A0095534639464046FEF7A3F8039AC1
:10F948000444A8E704AA03A91BF02AFBB7E7D31CC1
:10F95800039390784FF0010AACE7732B10D05BD972
:10F96800752B3AD0782B96D1A3F15802B2FA82F2CD
:10F97800306852092B4610210436FDF78FFFD7E770
:10F988003368049A0093394600234046FEF77AF814
:10F9980004360444039A7EE70028B9D1204608B00B
:10F9A800BDE8F0876E28B3D1039A336804361C602B
:10F9B80071E72AD9582BD7D0632B8DD06BE77828DD
:10F9C800A6D1A0F15802B2FA82F2306852092B4649
:10F9D8001021FDF763FF0436AAE706F1040E30682C
:10F9E8002B4600220A217646FDF758FFA0E7331D73
:10F9F800306829461E46FDF723FF99E7331D306816
:10FA080029461E46FDF71CFF92E7002B7FF443AF03
:10FA1800204608B0BDE8F0876E2BC6D03BE700BF94
:10FA28000EB400B584B005AB019053F8042B064919
:10FA3800039301A8FFF726FF019B00221A7004B068
:10FA48005DF804EB03B0704781DA00082DE9F04750
:10FA580007468CB01E469246002A6AD115461446BF
:10FA68000A8840F2B1739A423AD98B78581E0B280B
:10FA780036D891F803E00EF1FF301E2830D891F8FF
:10FA880004C0BCF1170F2BD891F80590B9F13B0FC2
:10FA980026D888793B2823D8B1F80880B8F57A7F2A
:10FAA8001ED24FF00108002E34D109890491002C90
:10FAB800B4BF2D212B21002CB8BF644203900591BF
:10FAC8000795CDF80890CDF804C0CDF800E0384689
:10FAD80006942F49FFF7A4FF40460CB0BDE8F08715
:10FAE8000023012118468E46ADF824308DF82830C1
:10FAF8008DF829308DF82A30ADF82C3099469C467F
:10FB08001A4698468DF826108DF827100B4609A935
:10FB1800002ECAD00390CDF80890CDF804C0CDF8D7
:10FB280000E038461B49FFF77BFF40460CB0BDE8B4
:10FB3800F087194C84FB0234A318D417C4EB631460
:10FB4800C4EB0415A2EB85052DB2002D0846B8BFFD
:10FB58006D42FFF7A3FD4FF47A7200238046894671
:10FB680023F0C8FD3C230AFB030A4FF47A720023F2
:10FB78004046494623F0BEFD4FF47A7192B2002305
:10FB8800C1FB0A2309A8FDF7C1FE24B209A967E74A
:10FB9800EC7A0308CC7A0308898888880FB430B5D2
:10FBA80083B006AB0A490B4853F8042B0968006870
:10FBB8000193FFF767FE084C05462068FEF7E4F856
:10FBC8000028FAD0284603B0BDE8304004B070479A
:10FBD800482A00204C2A0020F81B0020DFED2B7A51
:10FBE800B4EEE70AF1EE10FA4ADDDFED296A9FED7F
:10FBF800297A01E0B0EE670AB4EEC70AF1EE10FA0E
:10FC080070EE667AF6DC9FED247AF4EEC77AF1EEB0
:10FC180010FA38D5DFED1E6A9FED207A01E0F0EE8C
:10FC2800407AF4EEC77AF1EE10FA37EEA60AF6D467
:10FC3800DFED1B7AB4EEE70AF1EE10FA14DDDFED22
:10FC4800137A37EEC00A60EE006A9FED166A9FEDE0
:10FC5800167ADFED167AA6EE867A20EE266AE6EEAA
:10FC6800877AA6EE270A7047DFED117AB4EEE70A25
:10FC7800F1EE10FA44BFDFED087A37EEC00AE2E78A
:10FC8800F0EE407ABFE7B0EE670AD1E7DB0F4940F4
:10FC9800DB0FC940E4CB1641DB0F49C0E4CB16C1EA
:10FCA800DB0FC93F92E741B99730083C15A82ABE37
:10FCB800DB0FC9BF09B909E0194690FBF1F301FB55
:10FCC80013030846002BF7D1084670470146FBE7A7
:10FCD80007EE901AF8EE677A9FED837A27EE800A8E
:10FCE80020EE070AFDEEC07A17EE903A2033402B3B
:10FCF80000F28C80DFED7D7AB4EEE70AF1EE10FABF
:10FD080040F3E880B0EE407A9FED796ADFED796ADA
:10FD180001E0B0EE677AB4EEE67AF1EE10FA77EE2B
:10FD2800467AF6DC9FED747AF4EEC77AF1EE10FAB3
:10FD380040F1CD809FED6E6ADFED706A01E0F0EE74
:10FD4800477AF4EEE67AF1EE10FA37EE867AF6D4D0
:10FD5800DFED6B7AB4EEE77AF1EE10FA51DCDFED05
:10FD6800697AB4EEE77AF1EE10FA44BFDFED627A11
:10FD780037EEC77A27EE076ADFED635ADFED637A5D
:10FD8800DFED636A9FED635AE6EE257A67EE065A61
:10FD9800E6EE276AF7EE007AA5EEA67AF0EE675A45
:10FDA800E7EE055AE7EE457A87EEA55ADFED547A75
:10FDB80030EE277AFDEEC76A16EE903A2033402BD4
:10FDC80029D99FED557AF6EE006AB7EE006AF7EE8C
:10FDD800004AC4EEA57A0023836143610362C361CC
:10FDE80080ED045A67EEA66A27EE866A27EE877AC0
:10FDF800C0ED006AC0ED026A80ED016A80ED037A09
:10FE08007047DFED3A7A37EEC77AB3E7B7EE005AB4
:10FE1800F0EE455ACAE7B4EEE70AF1EE10FA5FDDF4
:10FE28009FED336ADFED336A01E0B0EE677AB4EE36
:10FE3800E67AF1EE10FA77EE467AF6DC9FED2E7A46
:10FE4800F4EEC77AF1EE10FA47D59FED296ADFED97
:10FE58002B6A01E0F0EE477AF4EEE67AF1EE10FA5A
:10FE680037EE867AF6D4DFED267AB4EEE77AF1EE4D
:10FE780010FA27DCDFED237AB4EEE77AF1EE10FA18
:10FE880044BFDFED1D7A37EEC77A27EE076ADFED4C
:10FE98001E4ADFED1E6ADFED1E7AE6EE246A67EE83
:10FEA800064AE6EE267AB7EE006AA4EEA77AF6EEE0
:10FEB800006A36EE476AF8EE007A27EE277A66EE91
:10FEC800266A84E7DFED097A37EEC77ADDE7B0EE18
:10FED800677A3DE7F0EE407A24E7B0EE677AC2E74A
:10FEE800F0EE477AAAE700BF27D4D236DB0F4940A5
:10FEF800DB0FC940E4CB1641DB0F49C0E4CB16C188
:10FF0800DB0FC93FDB0FC9BF92E741B99730083C07
:10FF180015A82ABEF304353F0000008070B40668B7
:10FF28008E4217D90139751E002311F8014F082296
:10FF3800634013F0800F4FEA430318BF83F0D503E3
:10FF4800013ADBB2F5D18D42EFD1721C02603370F9
:10FF580070BC70470023F8E710B44C09012250F830
:10FF6800243001F01F0102FA01F10B4340F824305C
:10FF78005DF8044B704700BF4B0901F01F0150F8B2
:10FF88002320012303FA01F1114214BF184600206F
:10FF9800704700BF2DE9F84F314A137803F0FF048A
:10FFA800002BFAD12F4BDFF8CCA01868DFF8C8B0C7
:10FFB800DFF8C88001238AF80030FEF7E5FE052146
:10FFC8002948F0F77BFA21462748F0F777FA062107
:10FFD8002548F0F773FA21462348F0F76FFA9BF8A3
:10FFE80000502148042145F00105F0F767FA294639
:08FFF8001D48F0F763FAB8F8A8
:020000040801F1
:100000000030ABB11B4D1C4F194E95F801900721E4
:100010003046F0F757FA49463046F0F753FAB8F849
:10002000003015F8012F07F8012F01349C42ECDB5A
:1000300007210F48F0F746FAFF210D48F0F742FA82
:100040009BF800400A480421F0F73CFA2146084892
:10005000F0F738FA054B1868FEF7A0FE00238AF87F
:100060000030BDE8F88F00BF4D360020AC5D0020A9
:10007000003C00404F3600206F38002059380020E7
:10008000A83C0020F0010020F8B50D4F0D4DC1F146
:10009000030646EA80063868FEF77AFEF6B21024B8
:1000A000E1B22846F0F70EFA013431462846F0F75F
:1000B00009FA202CF4D13868BDE8F840FEF76EBE8E
:1000C000AC5D0020003C00400C4B1B78DB0700D5EA
:1000D00070470B490B68002BFAD04FF47A7202FB81
:1000E00003F39842F4D3074B1B781BB9064B9A686D
:1000F0001B69136000230B60704700BF0D3E00209A
:10010000CC220020C0220020AC22002008B511F033
:1001100083FC024B024ADA60FEE700BF00ED00E01C
:100120000400FA05024A034B127819780BF072BEEC
:10013000D01B0020D11B00208D4B1B7803B17047D2
:100140002DE9F0438B4D2B688BB013B90BB0BDE894
:10015000F083894E894A3378044601A8D75C0CF0B5
:1001600097FD736803F5C333A0339C4205D9032F71
:100170006AD8DFE807F054494010814B1B78DB0751
:10018000E4D42B68002BE1D01B681B68002BDDD06A
:1001900020469847DAE704AF38460CF079FD97E837
:1001A000070007AB03C39DF810101A8021B10DF1B1
:1001B0001D0107A80BF0FCFD0DF11E000BF0ECFD7E
:1001C00038460A2207A924F0F3FE6D4B1A78071C63
:1001D00018BF012702F001026A4933780878746079
:1001E000013393FBF0F100FB11333370002AC8D0C8
:1001F000002FC6D1AAE7DFF8888198F8002012F016
:10020000010230D00027E7E704A80BF0C5FD074640
:10021000002832D15A4B1A7802F00102DCE79DF82F
:100220000430002B34D1564B197801F00101554AA6
:10023000337810787460013393FBF0F200FB1233D3
:10024000337000299DD081E74D4A4E4933780978B3
:1002500010787460013393FBF1F201FB1233C10794
:1002600033708ED572E707A80BF08AFD68BB98F84B
:100270000020002702F00102AEE707A80CF008FDFD
:100280009DF81E009DF81030834212D10027C1E76F
:10029000DFF8EC8098F80030DA072FD5394A337848
:1002A00011787460013393FBF1F201FB1233337068
:1002B0004CE72B68002BADD09A798242AAD31B68F9
:1002C0001B69002BA6D09847A4E7272012F01EF93F
:1002D00007460028CBD0272012F0BCF89DF81C3030
:1002E000814600283BD0002BC1D101200BF06CFDD2
:1002F00098F800204F4602F001026DE704A90DF1C5
:1003000003000BF055FD20B998F8001001F0010131
:100310008DE707A80CF0BCFC9DF81C009DF803308D
:100320009DF81D10834203D19DF810308B42EBD015
:100330002B684BB11A79824206D35A798A4203D389
:100340001B68DB6803B198470E4A337811787460F4
:10035000013393FBF1F201FB1233337011E7002BF1
:1003600085D00BF031FD98F8002002F0010233E750
:1003700058380020103E0020581F0020D12A0020AD
:100380000D3E0020D52A00202DE9F04F2DED028BE7
:10039000A0F10A0389B00C46ED2B00F27686DFE867
:1003A00013F022017406740674067406740674064B
:1003B000740674067406740674067406740674066D
:1003C000740674067406740674067406740674065D
:1003D00074062F027406740674062C0674067406DE
:1003E000740699017406560174063E0174063301C1
:1003F00074062802740603027406EF01740674067C
:100400007406EA01E4017406D20174067406CC0194
:100410007406A5017406740674068A0474067406CC
:10042000740674066C047406020174063B06290502
:100430007406740674067406740674067406FD0465
:100440007406CF0474069C04740665057406600681
:1004500074067406740674060503F105EA05B90509
:10046000EE00740674062803A60274066F02E90201
:100470007406740674067406DE0274067406BD0201
:10048000740674067406AF02F303BB037A037406A2
:10049000740674066C03740674064C0374067406C2
:1004A000740674067406740674067406740674067C
:1004B00074067406740674067406050374067406DE
:1004C000740674067406740674067406740674065C
:1004D000740674067406740674067406740674064C
:1004E000740674067406740674067406740674063C
:1004F000740674067406740674067406740674062C
:10050000740674063E037406740674067406740654
:10051000740674067406740674067406740674060B
:1005200074067406740674067406740674067406FB
:1005300074067406740674067406740674067406EB
:1005400074067406740674067406740674067406DB
:1005500074067406740674067406740674067406CB
:1005600074067406740674067406740674066204CF
:100570003804740674067406740674060904AF4ED3
:10058000337853B1AE4F002537F8021F2046FFF7EE
:1005900073F933780135AB42F6DC012009B0BDECCC
:1005A000028BBDE8F08FA54E3378002BF5D0A54F18
:1005B0000025B846236817F81520591C21601A70C9
:1005C00098F8011001EB810101EB810101F2EE21AC
:1005D00089B22046FFF750F933780135AB4208F174
:1005E0000208E7DCD9E7984D284622F0BDFB002839
:1005F000D3DD2B460544226813F8011B501C9D4295
:1006000020601170F7D1C8E7904D05F1800655F8CC
:10061000041F2046FFF718F9AE42F8D1BDE78C4D14
:1006200005F14006B5F880102046FFF725F923684C
:1006300095F88220591C21601A70236895F8832050
:100640000435591CAE4221601A70EBD1A5E7814DEB
:100650000B682A7A591C21601A70A98B2046FFF773
:100660000BF9298B2046FFF707F9698B2046FFF726
:1006700003F92368EA7C591C21601A70A98C204672
:10068000FFF7FAF8E98C2046FFF7F6F82368AA7F0F
:10069000591C21601A70236895F82020591C21608C
:1006A0001A70698C2046FFF7E7F82368EA7A591C2C
:1006B00021601A70E9682046FFF7C6F823682A7C93
:1006C000591C21601A70236895F82120591C21605B
:1006D0001A7062E70B68604A581C11782060197024
:1006E00023685278591C21601A7056E70B685A4AE1
:1006F0005A4D11785A4A581C2060197011682046CA
:10070000FFF7A2F82368534A591C127A21601A7025
:1007100029882046FFF7B0F8A9882046FFF7ACF8F3
:1007200029892046FFF7A8F820460021FFF7A4F802
:1007300020460021FFF7A0F82FE708460822454988
:10074000FFF76AF829E70B68464A474990785D1C2D
:100750002560187023685278581C20601A7023682E
:100760000A79591C21601A7017E70B680122991841
:1007700021601A7011E708460021FFF765F80CE7C1
:100780003A4D3B4E05F1300795F90210394B93F97C
:1007900006208A4203F1080300F07A849E42F6D1D3
:1007A0000835BD42F0D1F8E6334B03F15A05226813
:1007B0005979501C2060117022681978501C2060F3
:1007C000117022685978501C206011702268997845
:1007D000501C206011702268D978501C2060117064
:1007E000226819790633501C9D4220601170DED1B9
:1007F000D3E60B68174A591C527D21601A70CCE66B
:100800001E4D05F1500628781FF0DCFC2368027AA3
:10081000591C21601A7023686A78591C21601A706B
:100820002368AA78591C21601A702368EA78043575
:10083000591CAE4221601A70E5D1AEE6E0420020BC
:1008400012640020C84400208A500020804B002001
:10085000844B00203C5D00208C320020B42A002014
:100860001088002044310020D41B0020685D002047
:10087000C459002094590020182E0020B8430020AD
:10088000AF4D0B682A68591C127821601A702B68CA
:1008900022689978531C2360002311702A6821680C
:1008A0001A4401335279481C032B20600A70F5D199
:1008B00023682A68591C127A21601A7023682A68F2
:1008C000591CD27821601A7023682A68591C127941
:1008D00021601A702B6820465989FEF7CDFF2A68DF
:1008E0002368527A591C21601A702A68F8E620465B
:1008F0000021FEF7A9FF20460021FEF7BDFF4CE6D0
:10090000904D08462988FEF7B7FF69882046FEF714
:10091000B3FFA9882046FEF7AFFF3EE68A4D05F1FA
:100920006006A9882046FEF7A7FFE9882046FEF763
:10093000A3FF29892046FEF79FFF2368AA7A591C46
:1009400021601A702368EA7A591C21601A7055F8E0
:100950000C1B2046FEF778FFB542E2D11DE67B492D
:1009600052232268501C2060137011F8013F002BA5
:10097000F7D112E6764800232268056803EB4301AD
:10098000561C6D5C26601570026825680A446E1C52
:10099000527826602A70026825680A4401339278EA
:1009A000691C0A2B21602A70E6D1F6E500258146F4
:1009B000DFF8C881DFF8C8B1049503950595069561
:1009C00001214FF6FF7A05E001350B2D00F07E8303
:1009D00018F9011F4F1C4AFA05F3F5D0DE07F3D5CD
:1009E000BBF800302B41D807EED505A8FFF7B8FAC1
:1009F000EAE7584D08462988FEF73EFF69882046F9
:100A0000FEF73AFFB5F90430534AD91782FB0323A6
:100A1000C1EBA301204689B2FEF72EFFBDE50B68AE
:100A20004E4A591C1278216005A81A70FEF714FE70
:100A300023685A1C22601870AFE50B68484F591C98
:100A40003A7821601A703B78002B3FF4A6AD002560
:100A5000EEB230460CF068F923684278591C2160E8
:100A600030461A700CF060F901892046FEF704FF49
:100A70003B780135AB42EBDC8FE53A4D0846298ADD
:100A8000FEF7FAFE698A2046FEF7F6FEA98A20469E
:100A9000FEF7F2FE81E5DFF8ECE00027FEB27146DA
:100AA00000232268501C206016702268501C2060B1
:100AB0001370226811F8010F0133551C062B2560B5
:100AC0001070EED10137062F0EF1060EE6D1264941
:100AD00000232268501C206017702268501C206080
:100AE0001370226811F8010F0133551C0B2B256080
:100AF0001070EED123681D4A581C07212060197020
:100B000023680021581C20601970236892F8F02097
:100B1000591C21601A7040E50B68154A1549107878
:100B2000154A5D1C2560187023688978581C206060
:100B3000197023689278591C21601A702DE500BF46
:100B4000D840002038460020602C0020D0520308F6
:100B5000D44000208040002067666666E2310020B5
:100B60002A3E002044560020674C0020844B002081
:100B70002054002024310020343100200053030889
:100B8000D0400020434C00200A68AC4BAC49187898
:100B9000551C2560107022685878551C256010700F
:100BA00022689B78501C206013702046C988FEF78D
:100BB00063FEF2E405A8FEF74FFD00283FF4EDAC1C
:100BC000BDF814102046FEF757FE23689DF8162046
:100BD000591C21601A7023689DF81720591C216048
:100BE0001A7023689DF81820591C21601A70236818
:100BF0009DF81920591C21601A7023689DF81A204D
:100C0000591C21601A702046BDF81C10FEF734FEF6
:100C1000C3E48C4B03F1700522681978501C2060E6
:100C2000117022685978501C2060117022689978E0
:100C3000501C206011702268D978501C20601170FF
:100C400022681979501C2060117022685979501C53
:100C500020601170226899790733501CAB422060E4
:100C60001170D9D199E4784D0846E989FEF704FE60
:100C7000A9892046FEF700FE8FE40B68734D591CCE
:100C80002A7921601A7023686A79591C21601A70C8
:100C900029882046FEF7F0FD2368AA79591C2160B7
:100CA0001A7069882046FEF7E7FD2368EA79591C27
:100CB00021601A7071E40B6800255A1C0A602046F6
:100CC00029461D70FEF7C0FD29462046FEF7BCFDF3
:100CD00029462046FEF7B8FD5FE45D4E0B68727949
:100CE0005C4D591C21601A702B682046198CFEF748
:100CF000C3FD2B682046D98BFEF7BEFD71892046C7
:100D0000FEF7BAFDB1892046FEF7B6FD2B682046F6
:100D1000598CFEF7B1FD2B682046998CFEF7ACFD8F
:100D2000F1892046FEF7A8FD318A2046FEF7A4FD92
:100D30002A68236892F82620591C21601A702CE436
:100D4000434EF378002B00F098820B680822591C60
:100D500021601A7023680122991821601A70236893
:100D60003D4D591C2A7921601A702368AA78591CB4
:100D700021601A7029882046FEF77EFDE989204609
:100D8000FEF77AFD2368F279591C21601A702368F6
:100D9000EA78591C21601A70FFF7FFBB0BF01EF8B0
:100DA000FF28054600F07A8208A8002300F80C3DD1
:100DB0000AF0E6FF2268294B511C21601570226859
:100DC0001978501C2060117022685978501C2060DE
:100DD000117022689978501C2060117022689DF86B
:100DE0001410501C2060117020469988FEF744FDB5
:100DF000FFF7D3BB0B681A4D591C012221601A70F2
:100E00002368AA78591C21601A7007F007FD23682F
:100E1000144A15495E1C26601870B1F90010B2F929
:100E20000000FEF74BFF23685A1C226018702988C7
:100E30002046FEF721FDFFF7B0BB00BF1C310020AC
:100E400038460020202D002024310020504600206C
:100E500020540020D440002044560020143E00209E
:100E6000EA630020822F0020882F002020460021E6
:100E7000FEF702FD20460021FEF7FEFC2046002181
:100E8000FEF7FAFC2368B14D00265A1C22601E7042
:100E900023682A68591C92F82C2021601A70236854
:100EA0002A68591C92F8362021601A7023682A6833
:100EB000591C92F8372021601A7023685A1C22604E
:100EC0001E7023685A1C22601E7023685A1C226000
:100ED0001E702B682046598FFEF7CEFC2B682046EB
:100EE000198FFEF7C9FC23682A68591C92F82E2036
:100EF00021601A7023685A1C22601E702B682046DD
:100F0000598EFEF7B9FC2B682046998EFEF7B4FC8B
:100F1000FFF743BB8E4D8F4E9FED8F8ADFF88082A7
:100F2000DFED8E8A05F120070EE0FCEEE77ACDEDCD
:100F3000017ABDF8041020460435FEF79DFCAF424F
:100F400006F118063FF429AB717C0029F3D0844BDD
:100F5000D5ED007A1B78012BE7D1824B1B68DB04AF
:100F600040F18181F5EE407AF1EE10FA40F0A9816E
:100F700040F2DC51DFE7084610227B49FEF74CFCCB
:100F8000FFF70BBB794B9B8AB3F5006F00F27381BF
:100F9000B3F5806F00F29381B3F5007F34BF012772
:100FA0000227734D05F10C0655F8041B91FBF7F170
:100FB000204689B2FEF760FCAE42F5D16D4D6E4F12
:100FC00005F10C06B5EC010AD7ED077A80EE270A89
:100FD00023F05AF881B22046FEF74EFCAE42F1D122
:100FE000664D05F10C0655F8041B204689B2FEF744
:100FF00043FCAE42F7D1FFF7D0BA614D08462988CD
:10100000FEF73AFCA9882046FEF736FC29892046DF
:10101000FEF732FCFFF7C1BA0A685A4D511C012392
:101020002160137095F824205749002A40F065810B
:101030002268501C20601370236841F2B4105A1CBF
:10104000085C226041F27812187089582046890A9B
:10105000FEF7FAFBA96A20464908FEF7F5FBFFF701
:101060009CBA0B68494A4A49D0784A4A5D1C2560B7
:10107000187023684979581C206019702368D27849
:10108000591C21601A70FFF788BA0020FFF786BA52
:1010900023685A1C2260197029882046FEF7ECFB51
:1010A0002368EA78591C21601A7023682A79591C30
:1010B00021601A702368AA79591C21601A7023686C
:1010C0006A79591C21601A70FFF76ABBDFF8D4A057
:1010D00000254FF0A8080135C5F1200208FA02F2F8
:1010E000A5F120032AFA05F6164328FA03F31E4356
:1010F000282D06F001024FF000030BD01343EAD075
:10110000E8B211F003FA0028E5D0294605A8FEF759
:1011100027FFE0E7204B1B78DA0700F1BA800025B3
:101120001E4E2F4602E00135282D3DD0294630467F
:10113000FEF726FF0028F6D0294605A8FEF720FF77
:10114000002840F08B800137EDE700BFD44000203D
:1011500054320020845500200000404200E08244C8
:10116000685600204454002044320020884000206B
:10117000B840002038540020A85100208C460020A0
:10118000B42A00206C840020546700202431002001
:101190002C660020343100200D3E002020860020E7
:1011A000DB9B914190E33FF46A4B6B4DB3F85010D9
:1011B0002046FEF761FB00212046FEF75DFB674BF2
:1011C00019684B0103F02002C1F340031343C1F33C
:1011D000800243EA4203C1F3C00243EA8203C1F33F
:1011E000401243EAC20301F0100119432046FEF702
:1011F00043FB03A904222046FEF70EFB236829784F
:10120000574A581C2060197011886429A8BF6421AE
:101210002046FEF731FBB9F1960F45D0002120465C
:10122000FEF72AFB2168B7F1190348BFA7F11203A3
:10123000A3F3C4034A1C226020461A460B7004A97B
:10124000FEF7EAFA2368474A581C112120601970FA
:1012500020461168FEF7F8FAFFF79FB9394603A850
:10126000FEF77EFE6FE7F4EEC87AF1EE10FA4CDA84
:101270004FF47A715FE6082793E60B68B1783A4A33
:10128000581C2060197023681278591C21601A704C
:1012900065E5059B43F00103059340E723685A1C6D
:1012A00022601870FFF779B923680322591C216066
:1012B0001A7023686A78591C21601A70B2E70427F3
:1012C0006FE6F4EEC87AF1EE10FA3FF551AEF4EEA7
:1012D000E87AFDEEE77AF1EE10FA17EE901A2BD8C5
:1012E0006FF4F973303903FB01F140F2E73391FBFE
:1012F000F3F101F2DB5189B21DE64B78022B16D0D7
:10130000032B0CBF0423012392E6FDEEE77A40F2A3
:10131000E73217EE903A303B02FB03F388FB0312EF
:10132000D917C1EB622101F2E93189B203E6042A3F
:1013300034BF022303237BE640F2F313A1F583615C
:1013400003FB01F140F2E73391FBF3F101F2DD51D0
:1013500089B2F0E5EC020020486000207C400020CB
:101360002E2B0020CC4000201831002038B5094D2C
:101370002B8823EA0000834228800AD0064B1421E0
:10138000FF220E2002241C7059709A701EF032FD4C
:10139000288838BDD0400020342F002038B5094DB2
:1013A0002B881843834228800AD0074B1421FF2240
:1013B0000E2002241C7059709A701EF01BFD2888A4
:1013C00038BD00BFD0400020342F0020024A1368EF
:1013D00018431060704700BFCC4000205B4B5C4856
:1013E00070B54C22012500211D7023F00AFE594AD8
:1013F00059495A4C5A4800230B60136002F03AFED8
:101400002946052002F0DAFE6579291C4FF0070015
:1014100018BF012102F0D2FEA679311C4FF008005E
:1014200018BF012102F0CAFEA37A002B66D04D4CF2
:10143000002D6DD1311C18BF01214B4E092002F047
:10144000BDFE3168CA0773D4454D11F0020161D168
:10145000003118BF0121032002F0B0FE434A444B83
:10146000128E93FBF2F3642BB8BF64230121042096
:10147000C5F8143102F0A2FE3E4B0620197802F0A6
:101480009DFE01210A2002F099FE21680B20C1F384
:10149000802102F093FE21684B0508D5364B1B7A5C
:1014A000083B012B9CBF4FF4FA63C5F84C32C1F3E3
:1014B00000410C2002F082FE21680D20C1F3804122
:1014C00002F07CFE01210E2002F078FE01210F20A7
:1014D00002F074FE0121102002F070FE274B196803
:1014E000B3F8464029B10AF0E1FA014608B9C4F35D
:1014F000C0011120BDE8704002F060BEE37A194CD3
:10150000002B95D1216811F4802196D0002D91D027
:10151000012192E70121022002F050FE184B3168B0
:10152000DB6A642BB8BF642301F00201AB678FE76D
:10153000144B0B4D1B68642B4FF00101B8BF6423A3
:1015400008466B6402F03AFE31687EE720230020F3
:10155000D422002024230020D0220020604000203C
:10156000EC020020445400207C400020685D0020F4
:1015700040420F00084400203C5D0020AC3C0020AD
:1015800088400020345400202DE9F04F2DED028BCF
:1015900093B005461BF0B0FFB24B1E7826B113B0D6
:1015A000BDEC028BBDE8F08FAF4F3B685805F6D518
:1015B000DFF81883D8F80020002A00F01B81AB4C1C
:1015C000D4F8283103F5F43348339D42C0F012813A
:1015D000A74994F82C310968C4F828510133DBB2CB
:1015E000890784F82C3101F11E81580701F05C80D5
:1015F000282BA04B029301F0AB815E2090479E4BBD
:101600001B78002B6BD0994C9C4AD4F83031EB1AE4
:10161000934200F2CD87DFF8B8A29AF80080B8F1C3
:10162000000F33D1DFF86492D9F80000FCF7BCFB5F
:10163000C0B201280ED90228914F41F095823B7823
:10164000002B41F0C483D4F83831EB1AB3F57A6F2C
:1016500081F071848B480768002F40D09AF80030E1
:10166000BBB9894BD9F800001B689B781E3B012B46
:101670004FF0020141F2B78304300CF09FF80122D1
:1016800000238AF8002084F8443126E07D4807686A
:101690002FB3D4F8403140F6B732EB1A93421ED93B
:1016A00094F83C31002B01F05682013BDBB284F808
:1016B0003C31002B01F0248117F8011B94F84421E0
:1016C000076094F8453171480A440133006884F892
:1016D000442184F84531FCF76BFBC4F840516C4A57
:1016E000029B12781B68012A03F101030A9300F0A0
:1016F000B086684B1B786BB1674F3B6853B1029B58
:101700005A4CD3F800B0D4F85831ABEB0303632B39
:1017100000F23F86DFF8BC8198F800A0BAF1020F12
:1017200001F0CA80564F97F87430032B00F086877B
:101730005A4B1B7873B15A4E33685BB14B4CF4F77C
:10174000C1F9D4F8643144F61F62C31A9342834648
:1017500000F2D480534B1B78002B4ED1524B1B7898
:1017600043B1424CD4F8B43203F50043E8339D4210
:1017700080F0E5864D4B1B78002B3FF410AF3B4EBD
:101780004B4C4C4D06F2BD272068FCF70DFB0028A2
:101790003FF405AF2068FCF7FFFA2B7880465A1E0D
:1017A00033B120682A70FCF7FFFA0028F2D1F6E680
:1017B00003223946781E23F00AFC96F8BC3296F8CC
:1017C000BD2286F8BF8283F47F4383F0FF039B1A18
:1017D0001FFA88F89BB2B8EB132FD5D196F8BE222A
:1017E000DBB29A42D0D1781E0BF01AFB2B7818444A
:1017F0002870C9E71F4B029301E72F4C2278002A7B
:1018000040F01E86DFF8D09099F80040002C65D19A
:101810002A4E3078002841F06582144C284ED4F8C6
:10182000AC223178274B93FBF1F313449D4295D3BF
:10183000254A94F8B032C4F8AC52D75CF90701F1EC
:10184000DC83BA0701F195837B0701F1F58294F8F7
:10185000B0323178013393FBF1F201FB123384F89B
:10186000B0327BE75838002044540020601F00202D
:101870007C400020385C0020D26400203F0D030033
:1018800020000020E8400020E4400020E04000204C
:10189000D3640020E0640020A0790020E8640020E8
:1018A000EC6400202C6500203D650020F2640020DF
:1018B000F8640020FC640020C4640020346500202B
:1018C0003C650020A086010038650020F040002023
:1018D000EC400020145B002035650020054E376E7B
:1018E000002F41F07080044B89F80070C3F8AC52AF
:1018F00034E700BF44650020601F002094F86A317F
:10190000002B41F00A80E04B1B6803F00802002A1C
:1019100048F603414AF60B404BF60F4249F607479B
:1019200004BF02460F4613F0040F4FF0190118BF11
:1019300017469A0684F86A1103D547F4804747F0A2
:10194000200702F007FAC7F30909002841F0A8832D
:10195000CE4B9B79002B41F09C83984664204FF03E
:10196000FF3A4FF0000C0A970B97ADF834C0CDF852
:101970003AC0CDF83EC0CDF842C0CDF83090ADF8B9
:101980003680ADF838A08DF846000AAF0FCFDFF8EB
:101990000CE384F805C0AEE80F0097E80F00AEE84E
:1019A00007002EF8023B71464FF0010C1B0CFE277E
:1019B0001F20C82201F81E39A770A27184F807C041
:1019C000E07094F87A01207180F0F10383EA031348
:1019D000DAB2130983F0E70343EA022383EAC2037E
:1019E0001BB283EA0312D2B2C3F3072383EA1213B2
:1019F00043EA022383EAC2031BB283F0C80282EAED
:101A00000212D2B2C3F3072383EA121343EA02237A
:101A100083EAC2031BB283EA0C0787EA0717FFB207
:101A2000C3F3072282EA171242EA072200EB0C03F3
:101A300082EAC7070EEB0C0084F87A31278011F890
:101A4000013B7B4083EA0313DBB21A0982EA1722C7
:101A500042EA032282EAC3031BB29FB2814227807B
:101A6000EDD183F07C0383EA0313DBB24FEA131E4C
:101A70008EEA172E8EEA032E8EEAC30E0FFA8EFE22
:101A80001FFA8EF9DFF818C2A4F800905FFA8EFEF4
:101A90004FEA192984F8289084F827E00CF5D178CA
:101AA00004F1220ADCF80000DCF80410DCF808205D
:101AB000DCF80C3047460FC70CF1100CD445B84683
:101AC000F0D1DCF800003860714F9CF8043088F8E1
:101AD000043007F1270884F8C9E184F8CA9117F89F
:101AE000011F3068FCF764F9B845F8D194F86B2110
:101AF000002A40F00D876749029B08781B680A217D
:101B000084F86B11002801F0DC80DFF898E10128EF
:101B1000BEF80010059141F208840228BEF8028048
:101B200001F0B483BEF804100491032801F0E883A7
:101B30000428BEF806A001F0F083BEF80810039157
:101B4000052801F0E6830628BEF80AC001F0EA8302
:101B50000728BEF80C1001D0BEF80E2094F87A01C8
:101B60000A93074687F0300383EA0313DBB24FEA98
:101B7000131E494806978EF07A0E4EEA032E00880F
:101B800027718EEAC303DFF820E1C0EB00208EFB53
:101B9000007E8644C017C0EB6E270797059F4FF065
:101BA000000967F30F09049F68F31F494FF000080D
:101BB00067F30F08039FCDF82C901BB24FF0000E77
:101BC00083EA031067F30F0E0027C0B261F30F071B
:101BD000C3F307236CF31F4E62F31F474FF0000C53
:101BE0009DF81C20CDF834E083EA10136AF31F48F7
:101BF000CDF830800E978DF83CC08DF83D2043EA3B
